:020000040000FA
:040000006FD00400B9
:101000006F00907E00000000000000009020002093
:10101000AA220020A9BDF9F56C23002000000000E1
:10102000000000006C230020902000200000000041
:101030000000000090200020000000009020002010
:101040000000000090200020902000209020002030
:101050009020002090200020582F00209424002071
:101060000000000090200020902000201E2400207E
:1010700090200020D22300209020002090200020EB
:101080009020002090200020902000209020002020
:101090009020002001A04111B7170040985F3AC688
:1010A000945F3247E39CE6FE3245410182800111A4
:1010B00013078008F337078093F787083EC20100C3
:1010C0000100B7170040930570052380B70413068D
:1010D00080FA2380C7040100010083C6B70493F699
:1010E000F60DA385D704238007049246F3A6068055
:1010F0000100010093760502D5CEF336078093F602
:10110000860836C4010001002380B7042380C70489
:1011100001000100B70614007D89558D88C70100C4
:1011200001000100010023800704A246F3A6068007
:101130000100010073370780137787083AC6010062
:1011400001002380B7042380C704010001000100CF
:1011500001003727004093061005A303D7802380A2
:101160000704B247F3A70780010001009307800836
:10117000F3B7078093F787083ECE01000100B71749
:101180000040130770052380E704130780FA2380CB
:10119000E7040100010003C7B70413670708A3852C
:1011A000E70423800704F247F3A70780010001004A
:1011B0000561828093760504BDC6F336078093F6F9
:1011C000860836C8010001002380B7042380C704C5
:1011D00001000100B7061400938606047D89558D31
:1011E00088C7010001000100010023800704C246F6
:1011F000F3A6068001000100733707801377870884
:101200003ACA010001002380B7042380C70401000B
:1012100001003727004093062005A303D7802380D1
:101220000704D24781B773370780137787083ACC12
:10123000010001002380B7042380C70401000100DE
:1012400098471367070C98C723800704E24719BF24
:101250000111814601468145114506CE97000000E7
:10126000E780605893078008F3B7078093F78708F3
:101270003EC601000100B717004013077005238028
:10128000E704130780FA2380E7040100010003C785
:101290006704136717002383E70423800704B2471A
:1012A000F3A7078001000100F2400561828041112F
:1012B000814601468145114597000000E780A05214
:1012C00013078008F337078093F787083EC40100AF
:1012D0000100B7170040130670052380C70493066A
:1012E00080FA2380D70401000100FD552396B70240
:1012F00023800704A245F3A5058001000100733790
:101300000780137787083AC6010001002380C704CD
:101310002380D7040100010003C767041367170087
:101320002383E70423800704B247F3A70780010063
:10133000010001A0B1473305F50201007D1575FDDF
:101340008280411122C426C206C6AA8401446317C2
:101350009400B24022449244410182800504130566
:10136000803E420497000000E78000FD4180C5B741
:101370009305000273A04580824573901534924016
:101380002242B2424243D2436244F2440255925551
:101390002256B2564257D2576258F25806499649D9
:1013A000264AB64A464BD64B664CF64C065D965DD1
:1013B000265EB65E465FD65F09617300203041113C
:1013C000B7170040985F3AC6945F3247E39CE6FE49
:1013D000324541018280B71700401307000323887C
:1013E000E702854717170000232EF74873002030C7
:1013F000411122C42D6426C24AC006C637190040D6
:101400001304A4AAB704002023208900976000E0F9
:10141000E780205B9C408297976000E0E780605AFD
:10142000E5B737370040834747009146BD8B639E41
:10143000D702B73600401306F00F973500009385AA
:10144000E5209737000083D7673003C7A6001377DE
:10145000F70F1DE3B7E70400BC4F09468945171590
:1014600000000345A5F8829731A099466394D70000
:10147000834757007300203003C786001377F70FA8
:10148000E365F6FC13851700AE9717380000231F9D
:10149000A82A2380E70075B7B787004003C7670015
:1014A000098B6309071003C77700930600031377BE
:1014B0000703630DD708173800000348387C173638
:1014C00000001306A6780547B30606012380E60050
:1014D00083C577001737000013074779429793F5C4
:1014E000F50F2300B70003C58700973500009385EB
:1014F000E576C2951375F50F2380A5000347070015
:1015000089451377F703630CB70C63E7E50A6306B5
:10151000071A8545630CB7129737000083C7177603
:101520003307F600034707001377F70F19CB85073A
:1015300093F7F70F3D476363F71A17370000A30FC0
:10154000F772B787004009472383E700B787004059
:1015500083C77700E207E18763DE0704973700005F
:1015600083C7D771173700001307476E3E9785462C
:101570002300D700173700001307476F3E979306E5
:1015800000032300D700173700001307276D3E978D
:10159000A14685072300D70093F7F70F3D47636403
:1015A000F71417370000A30BF76CB7870040094703
:1015B0002383E70073002030930610026300D70EE8
:1015C000930620026305D70693060002E316D7F4BC
:1015D00003C727021377C70F13672700D5A803C7D0
:1015E00067001377070465CB03C7A702173800000D
:1015F00013084847173500001305853E13470708B1
:101600002385E70203C7A7021377370F1367870005
:101610002385E702814713070004B305F5008C41D9
:10162000B306F80091078CC2E399E7FEF5B503C74E
:10163000A702134707042385E70203C7A70213770E
:10164000C70F136727002385E702F9B503C76700B3
:101650001377070449C303C767021738000013084C
:101660002834173500001305652B1347070823831B
:10167000E70203C767021377370F136787002383D7
:10168000E702814713070004B305F5008C41B30658
:10169000F80091078CC2E399E7FEBDBD03C767025E
:1016A000134707042383E70203C767021377C70FB3
:1016B000136727002383E70285B503C76700137705
:1016C000070411CB03C727021377370F136787006F
:1016D0002381E70291B5238006003DBD97370000C6
:1016E000A38E0758B9BD97370000A389075875BD69
:1016F0002303048015472303E48001002302A48010
:10170000828083076480E3CE07FE23030480828007
:1017100083076480E3CE07FE03454480828083070D
:101720006480E3CE07FE2302A4808280411126C498
:101730004AC24EC006C61377F50BAD47AA892E895B
:101740009544630CF700194597000000E78080FA84
:1017500097000000E78020FB8D444E859700000035
:10176000E78040F9FD59FD1463983401B240A2446A
:101770001249824941018280135509011375F50F01
:1017800097000000E780E0F92209F1BF011126CCA3
:1017900006CEB704080097000000E780C0F61545A4
:1017A00097000000E78000F597000000E78080F6D2
:1017B00097000000E78000F62AC697000000E78047
:1017C00080F432459377150089EB13651500137586
:1017D000F50FF240E24405618280FD14E9F0014515
:1017E000CDBF397126DC4ADA4ED852D656D45AD2F9
:1017F0005ED006DE62CE66CCB7E700E07D5783AAF6
:10180000070022C603AA470023A0E71823A2E7186F
:10181000B7170040130770052380E704130780FA09
:101820002380E70483C74704930B75FFB684E20760
:1018300093FBFB0F8546AA892E8B32893724004003
:10184000E187015763FA76016308D50089461307DB
:1018500000026313D5000157D98F93F7F70FB71C18
:1018600000402382FC0411472303E4801305F00F9A
:1018700097000000E78000E8094C97000000E7802F
:1018800080E863657C15B7050700DA9537870700A0
:10189000795563FEE504B3879500636AF704370B57
:1018A0000800A94733EB65016395F90881E8814495
:1018B00097000000E78020E5268515A8DA85094510
:1018C00097000000E780C0E605090345F9FFFD1415
:1018D000050B97000000E780C0E481C49377FB0FFD
:1018E000E5F797000000E780A0EA69F17D55B7179A
:1018F0000040130770052380E704130780FA238054
:10190000E70403C74704418B2382E704F250B7E79B
:1019100000E023A0571123A24711E2543244525948
:10192000C259325AA25A125B825B724CE24C21615C
:101930008280A547639BF90685691309F00FB306FA
:101940009900B3742B01B6941349F9FFB37499004D
:10195000856B33796901416B9387F9FFB3F72701F1
:1019600099E363FC340193D94900C147E3E637FFAB
:101970003DBF0569C1697D19D9B71305800D63881D
:101980006901130500026384790113051008CA85F3
:1019900097000000E780C0D997000000E78040DF93
:1019A00031D54E99B38434416DBFDA852D4597000A
:1019B0000000E780E0D7CA94E30B99EE0509970091
:1019C0000000E78020D5A30FA9FEFDB79387F9FF9C
:1019D00093F7F70F636DFC0C83C71C0413073008E3
:1019E0006315F706370708006361EB06B3079B0032
:1019F000B706100063FBD704334BEB0089476399AC
:101A0000F9068980D549E38404EADA850945970017
:101A10000000E780E0D111090327C9FF9147232087
:101A2000E48003076480E34E07FE23033481FD173F
:101A3000EDFBFD14110B81C49377FB0FE9FF9700B9
:101A40000000E780E0D461F155B5B717004003C747
:101A50005704B70708001377070219E3B787070091
:101A60007955E376FBE833079B00E3F9E7F841B5E6
:101A70008547E380F9F0DA852D4597000000E7807F
:101A800020CB9389F4FFE38404E297000000E78011
:101A900060C893F7390091EB83260480032709007F
:101AA00093074900E396E6E03E89CE84D9BFB54767
:101AB0006399F9001305900B97000000E78080C33D
:101AC000FDB3B1471305B00AE388F9FE9947639760
:101AD000F904B7050800B365BB002D459700000069
:101AE000E78000C581448D4BA14997000000E78045
:101AF00060C263967401832704802320F900850463
:101B0000E39534FF8327048013172B0163550700E7
:101B10002312F90069BB2322F90051BB9D47639F43
:101B2000F90281451305B00497000000E78040C02A
:101B3000BD442320090023220900FD59970000001D
:101B4000E78040BD93F77400CA9703C70700FD14F0
:101B5000398D2380A700E39334FF91BBA14763979E
:101B6000F90697000000E780A0C28144630D0B00D6
:101B70008D479304C0036308FB00930400056304CE
:101B80008B01930440041375C507E30295D21945F0
:101B900097000000E78000B697000000E780A0B63D
:101BA000054597000000E780E0B426859700000017
:101BB000E78020B7094597000000E78080B69700CE
:101BC0000000E780E0BCE31405CE0DB39147639FAE
:101BD000F9001305600697000000E780A0B19700A8
:101BE0000000E78040B213059009F9B5E38109CC04
:101BF000F1547DB9BD6601471736000013068625EE
:101C0000938606A685458347060093F7F70F91C391
:101C100082800507E3F9E6FE97370000238CB722A0
:101C2000DDB77D166206618693178601E18763D46E
:101C3000070001458280931726003307F500AE9711
:101C400018439C4363E7E7007D16E37FF7FC7D556F
:101C5000828005458280FD15E205E18513978501A7
:101C6000618793F7F50F63480700FD15139725006B
:101C70002A97584365D713851700620561858280CE
:101C80003308B5021C4283A80600B335B502C297DB
:101C900033B50701AE98469585486367B5006394F0
:101CA000A50063E3070181480C43C6950CC388C2B5
:101CB0001CC2828081471397870161876343B70005
:101CC0008280139727002A97232007008507E5B70E
:101CD0008147014793968701E18663C5B6001335B6
:101CE0001700828093962700AA9694428507558F05
:101CF000D5B793D755408A07AA979C430545331516
:101D0000B5007D8D828017F3FFDFE702833D2A84D3
:101D100097000000E78060F405C5931725003E9406
:101D20000327C4FF814711EB7D1516053E9542053B
:101D3000418517F3FFDF6700033D05838507E5B79E
:101D40000145C5BF81471397870161876343C7007A
:101D5000828013972700B386E50094422A9785076F
:101D600014C3D5B77D1662066186014793178601B5
:101D7000E18763D50700133517008280931726008B
:101D8000B306F500AE9794429C437D16B58F5D8FE8
:101D9000F1BF8A05AA9501476363B500828083A6D7
:101DA000C5FFF11593D71600D98F9CC11397F60183
:101DB000E5B72A830148014701456343D700828084
:101DC000B387050183A80700B30706019C43C697A4
:101DD000AA976384F80033B517010507B308030118
:101DE000620723A0F80061871108C1BF2A83014759
:101DF0008147014563C3D70082803388E50083288B
:101E00000800330EE600032E0E003388A840330886
:101E1000C8416384080133B508018507B308E300AE
:101E2000E20723A00801E1871107E9B717F3FFDFF5
:101E3000E702232B0111B286B2842E86AA850A8579
:101E400097000000E780C0FA2A84A6850A859700DB
:101E50000000E78020E833348000060413351500C5
:101E6000018D056117F3FFDF6700E32917F3FFDF3B
:101E7000E702A3244111AA89AE8A328BB68402C23A
:101E800002C402C60144131C8401135C8C416349E3
:101E90009C02939B1400FD1B0549138CF4FFF15C1D
:101EA00033048901620461846340740792478E049D
:101EB000CE9423AEF4FE410117F3FFDF67006323E6
:101EC00013192400B30B2B01014A93172A00D6974C
:101ED00083A50B0088437800340050009700000071
:101EE000E78040DA050A93178A01E187F11BE35E78
:101EF000FCFC92474E9905042320F900A2473EC2FC
:101F0000B24702C63EC441B7131A8901135A8A4127
:101F1000131D240093178A01E18763CF970092472E
:101F20000A044E941CC0A24705091379F90F3EC25A
:101F3000B24702C63EC4ADB7B3079A0313152A00D1
:101F400056950841780034005000050AEA97DA9760
:101F50008C4397000000E780E0D26DBF197106C284
:101F600012C416C61AC81ECA22CC26CE2AD02ED219
:101F700032D436D63AD83EDA42DC46DECAC0CEC2C9
:101F8000D2C4D6C6DAC8DECAE2CCE6CEEAD0EED2F9
:101F9000F2D4F6D6FAD8FEDA971500009385058EAE
:101FA0008841E700050092402242B2424243D243B8
:101FB0006244F244025592552256B2564257D257C5
:101FC0006258F25806499649264AB64A464BD64BBD
:101FD000664CF64C065D965D265EB65E465FD65F45
:101FE0000961730020300000972100209381810156
:101FF000175100201301018117F5FFFF1305C500DC
:102000009705002093850500171600201306C6FDCE
:1020100063FAC5008322050023A055001105910530
:10202000E3EAC5FE170502001305053097150020E9
:102030009385C5FB171600201306C66763FAC50013
:102040008322050023A0550011059105E3EAC5FE92
:102050001715002013050566974500209385852BED
:102060006377B500232005001105E36DB5FEFD4241
:10207000739002BC8D4273904280B722000093821D
:10208000828873900230970200209382A2F793E235
:1020900032007390523097520000938222A47390C2
:1020A00012346FB0F47573002030397101436EC67D
:1020B00019A0397141536AC866CA62CC5ECE19A0B4
:1020C000397101535AD056D252D44ED64AD826DA54
:1020D00022DC06DE33016140828241114AC026C201
:1020E00022C406C68282B24D4101024D924C224C5E
:1020F000B24B4101024B924A224AB2494101024984
:1021000092442244B240410182803D432A87637356
:10211000C3029377F700BDEFADE5937606FF3D8AE6
:10212000BA960CC34CC30CC74CC74107E36BD7FE30
:1021300011E28280B306C3408A0697020000969699
:102140006780A6002307B700A306B7002306B700E1
:10215000A305B7002305B700A304B7002304B70005
:10216000A303B7002303B700A302B7002302B700FD
:10217000A301B7002301B700A300B7002300B700F5
:10218000828093F5F50F93968500D58D9396050182
:10219000D58D61B7939627009702000096968682A8
:1021A000E78086FA9680C1171D8F3E96E374C3F8C8
:1021B000A5B73367B500FD530D8B79E7B7877F7FF0
:1021C0009387F7F710419441B372F6003363F6003A
:1021D000BE92B3E262006397720C6318D606504158
:1021E000D441B372F6003363F600BE92B3E26200EC
:1021F0006398720A631BD60410459445B372F600C7
:102200003363F600BE92B3E262006391720A631E0A
:10221000D6025045D445B372F6003363F600BE9241
:10222000B3E26200639A72086311D60210499449BE
:10223000B372F6003363F600BE92B3E262006393BA
:1022400072085105D105E30FD6F6131706019397CF
:102250000601631CF7001357060193D706013305E7
:10226000F7409375F50F91E982804183C18333056F
:10227000F7409375F50F91E182801377F70F93F78D
:10228000F70F3305F74082800346050083C605003B
:10229000050585056313D60065FA3305D6408280AF
:1022A00011059105E312D6FE014582802105A105A5
:1022B000E31CD6FC014582803105B105E316D6FC4E
:1022C000014582804105C105E310D6FC01458280AD
:1022D000B717004003C777051377E70FA38BE70411
:1022E000130700F8A38DE7043D47238CE704130789
:1022F0005003A38CE70403C7A7051377D70F238DDB
:10230000E7048280B717004003C7E7020D89411137
:102310001377C70F498F93068008F3B6068093F6AC
:10232000860836C601000100930670052380D70495
:10233000930680FA2380D704010001002387E70277
:1023400023800704B247F3A7078001000100410181
:10235000828041112A83014E930E407E130F001993
:10236000930F400663E56E129308001913034006AD
:10237000B3781503854E0D4FA14F337365020D8958
:102380001335150063EFBE121308F6FF79467298F5
:102390004208135808013307C70213D61700BE07B7
:1023A00032976146B3F6C60213068070B386C60242
:1023B0003697A166F58F42075D8FB716004083C739
:1023C000F60293F70708A303F1000346710083C7E1
:1023D000F60293F70708E394C7FE83477100B71628
:1023E000004093F7F70F6388071293078008F3B74D
:1023F000078093F787083EC401000100B71700402B
:10240000930670052380D704930680FA2380D704AF
:102410000100010023AA070383C6170393E60608F9
:10242000A388D70223800704A247F3A707800100EF
:1024300001001166B71700407D16D45BC85F938515
:102440004703A98EF18EF5FA93068008F3B606804D
:1024500093F6860836C601000100930670052380B6
:10246000D704930680FA2380D7040100010098C1A5
:1024700003C7170313670704A388E7022380070431
:10248000B247F3A7078001000100410182807D135C
:102490003368E3039308E016630E08003368F30320
:1024A0009308D016630808009378330093B8180097
:1024B0009388D81633081E01131E0801135E0E01FF
:1024C00055B56393E5030548638608000148630337
:1024D00003002A8871087298FD15131E0801C205B1
:1024E000135E0E01C18179BD13F8150063F4BF00BE
:1024F0007908D5B713381800E5BF83C7F60293F7FC
:102500000708A303F1000346710083C7F60293F79F
:102510000708E394C7FE8347710093F7F70FF1DFD5
:10252000E9B531714AD966CB06DF22DD26DB4ED70D
:1025300052D556D35AD15ECF62CD6AC96EC7AA8C26
:1025400002D897100000E78020B12A8993078008FD
:10255000F3B7078093F787083EDA01000100B71749
:102560000040130770052380E704130780FA2380D7
:10257000E7040100010003C7F7021377770FA38771
:10258000E70203C7F70213678700A387E7022380E8
:102590000704D257F3A70780010001000545970003
:1025A0000000E78060D6130780C13347E902116A53
:1025B00093070AE893065002BD69930BA004814A71
:1025C000014B13048008930470057D1AB347F90288
:1025D0003307D7023EC0FD873ECC938709A69309F7
:1025E000803E3347F7023AC27D873AC43347390306
:1025F0008549B399990193D93940B306D702B30BF2
:102600007703B3C6F602B3CBFB0236C6FD8636C8E7
:1026100093D6FB4136CEB7460F0093860624334946
:10262000D9028566938606FAB3969601B389E902C4
:10263000130760553309D90293060010B389E902E4
:102640003349D902B3C9F9029316390036CA37198A
:102650000040FD8636D0930D090493D7F9413ED250
:10266000F336048093F6860836DC010001009307F8
:1026700070052380FD00930680FA2380DD000100B1
:1026800001008346390593F6860FA309D9048346D2
:10269000390593E61600A309D90423800D00E256FC
:1026A000F3A6068001000100130C80FA116DF336C9
:1026B000048093F6860836DE01000100930770055A
:1026C0002380FD0023808D01010001008346390530
:1026D000216693E60602A309D90483560905B3E6E9
:1026E000A6012318D90483560905D18E2318D904CD
:1026F00023800D00F256F3A60680010001008346F8
:10270000390593F606026381061A03463905218AC4
:102710006DDE081897100000E7800098733604807B
:1027200013768608B2C20100010023809D00238039
:102730008D0101000100B717004003C6370513766D
:10274000F60DA389C70403C6370513660602A389DD
:10275000C704835609052166B3E6A6012318D904E8
:1027600083560905D18E2318D90423800D0096467F
:10277000F3A60680010001008346390593F60602A0
:10278000638B061483463905A18AEDFE970000206D
:10279000E7806090AA8636D497000020E780A08F5B
:1027A000A256E30AD5FE835609054255B3E6A601B3
:1027B0002318D90497100000E780C08F834639059D
:1027C000A18AEDDE03560905834629058247337643
:1027D000CA00B306DA0293D5F641B296B388F64042
:1027E000E24733B8C6002E983308F840A247B3B684
:1027F00016013308D84063C70701631DF8009247EC
:1028000063FA1701C247634FF80E63950701B24799
:1028100063EAF80E894663E9660FF24693151800DD
:1028200013D3F8015E8613951800B365B30042D642
:1028300046D497C00100E78060093258050B137B2E
:10284000FB0F63470001631A0838A25863870838F2
:1028500013081500B336A800B69513D6F5013298C3
:10286000B336C800AE9613581800FE06B3E606014C
:102870007336048013768608B2C6010001002380F7
:102880009D0023808D01010001000356C902B2960C
:10289000C206C1822316D90223800D00B646F3A6D4
:1028A00006800100010021B5F336048093F6860806
:1028B000B6C00100010023809D0023808D0101002E
:1028C00001008346390593E60602A309D904238053
:1028D0000D0086460DB5F336048093F68608B6C41F
:1028E0000100010023809D0023808D010100010073
:1028F0008346390593E60602A309D90423800D0017
:10290000A646BDB5E30B0BF0F336048093F68608BC
:10291000B6C801000100930680FA23809D00238041
:10292000DD00010001008346390593F5FC0F93F6A5
:10293000860FA309D90483463905CD8EA309D9048E
:1029400023800D00C646F3A6068001000100130592
:1029500080FA03463905930639051D8A631C9629BA
:102960007336048013768608B2CC0100010013068A
:1029700080FA23809D002380CD000100010003C662
:1029800006001376F60D2380C60003C60600136604
:1029900006022380C600835609051166D18E2318CE
:1029A000D904835609052166D18E2318D9042380C2
:1029B0000D00E646F3A6068001000100130680FA2A
:1029C0008346390593F60602638006268346390559
:1029D000130C3905A18AFDDA081897000000E7807A
:1029E000A06BF336048093F68608B6D00100010090
:1029F000930680FA23809D002380DD000100010002
:102A000083460C00116693F6F60D2300DC00834626
:102A10000C0093E606022300DC0083560905D18EE4
:102A20002318D904835609052166D18E2318D904A9
:102A300023800D008656F3A60680010001001306D0
:102A400080FA8346390593F60602638A0620834698
:102A50003905A18AEDFE97F0FF1FE780C0632A8C3D
:102A600097F0FF1FE7802063E30C85FF835609057D
:102A700011664255D18E2318D90497000000E780D3
:102A800060638346390513063905A18AFDDAF336FA
:102A9000048093F68608B6D401000100930680FAFC
:102AA00023809D002380DD00010001008346060095
:102AB00093F6F60D2300D60023800D00A656F3A64C
:102AC0000680010001008356090503462905D24707
:102AD000B376DA003306CA021305800C9355F6412B
:102AE0003696330DF6408257333CD6002E9C333653
:102AF000A601330CFC40330CCC40330885039256BE
:102B00004E86B335A5033305A503C29597C00100D2
:102B1000E780C0DB63468001631E0C16630C0D1654
:102B2000130615003335A6002E959356F5013696FB
:102B3000B335D600AA959396F50105828585D18E89
:102B40006346B000639D051A638B061A0356C902DB
:102B500015823305D6003336C500B2956348B00000
:102B6000639105241306F00F637DA622894663F363
:102B7000561593078008F3B7078093F78708BED6EA
:102B80000100010037170040930770052300F70488
:102B9000930780FA2300F704010001008356C7025F
:102BA00089678117D58FC207C1832316F7022300D7
:102BB0000704B657F3A7078001000100FA506A54D2
:102BC000DA544A59BA592A5A9A5A0A5BFA4B6A4C49
:102BD000DA4C4A4DBA4D296182801308F5FF33352E
:102BE000A800FD152E951356F5013298B336C8008E
:102BF000AA9695B9F336048093F68608B6CA010002
:102C0000010023809D002380AD0001000100834668
:102C10003905CD8EA309D90423800D00D646F3A62D
:102C200006800100010035B3F336048093F6860870
:102C3000B6CE0100010023809D002380CD0001005D
:102C400001008346390593E60602A309D9042380CF
:102C50000D00F646F3A606800100010095B3F33699
:102C6000048093F68608B6D20100010023809D00FF
:102C70002380CD00010001008346390593E606025A
:102C8000A309D90423800D009656F3A606800100FF
:102C9000010045BB9306F5FF33B5A600FD152E9543
:102CA0009355F501AE96B3B5B600AA951396F50106
:102CB000858269B5F336048093F68608B6D801009C
:102CC0000100930680FA23809D002380DD0001002F
:102CD00001008356C9020566011693F6F60FD18EE0
:102CE000C206C1822316D90223800D00C656F3A660
:102CF000068001000100850A93FAFA0F95B233E6C7
:102D0000B60045C20356C9023305D0403338A0008F
:102D1000B305B040B385054115826345B000D1E1EC
:102D20006371A608894663F0560593078008F3B7D8
:102D3000078093F78708BEDA01000100B71700404B
:102D4000130770052380E704130780FA2380E70444
:102D50000100010003D7C7027D8B2396E702238081
:102D60000704D65781BDF336048093F68608B6DC97
:102D700001000100930680FA23809D002380DD007E
:102D8000010001008356C9020566011693F6F60F8D
:102D9000D18EC206C1822316D90223800D00E656C9
:102DA000B9B793078008F3B7078093F78708BEDEAB
:102DB0000100010037170040930770052300F70456
:102DC000930780FA2300F704010001000356C702AD
:102DD00093975600B297C207C1832316F7022300C8
:102DE0000704F657C1BB914763EEB70217D701003E
:102DF0001307074B8A05BA959C41BA978287B71784
:102E0000004003A7470B1345F5FF698F23AAE70A84
:102E100003A7070B698F23A8E70A03A7070A798D81
:102E200023A0A70A8280B717004083A6470B134749
:102E3000F5FFF98E23AAD70A83A6070B558D23A881
:102E4000A70A83A6070A758F23A0E70A8280B7170F
:102E5000004003A7470B498F23AAE70A03A7070BE4
:102E60001345F5FF45BFB717004083A6470B13472F
:102E7000F5FF758F23AAE70A03A7070A598D4DB7F7
:102E8000B717004003A7470B498FEDB7914763EE93
:102E9000B70217D701001307E7418A05BA959C418D
:102EA000BA978287B717004003A7470D1345F5FF70
:102EB000698F23AAE70C03A7070D698F23A8E70CE6
:102EC00003A7070C798D23A0A70C8280B7170040B9
:102ED00083A6470D1347F5FFF98E23AAD70C83A6C7
:102EE000070D558D23A8A70C83A6070C758F23A06B
:102EF000E70C8280B717004003A7470D498F23AA2C
:102F0000E70C03A7070D1345F5FF45BFB7170040B2
:102F100083A6470D1347F5FF758F23AAE70C03A778
:102F2000070C598D4DB7B717004003A7470D498FC0
:102F3000EDB7797122D43714004026D24AD0035914
:102F400024028354040206D64209C2044ECE52CC57
:102F500056CA13590901C1802DE11379F9F793F489
:102F6000F49F4209C20413590901C18093078008E4
:102F7000F3B7078093F787083EC401000100930769
:102F800070052300F404930780FA2300F404010081
:102F90000100231124032310940223000404A247F8
:102FA000F3A7078001000100B25022549254025945
:102FB000F249624AD24A45618280B7F507008146EC
:102FC0003000B105194597000020E7808081A247B5
:102FD00013972701E34A07FC1369090893E40440A7
:102FE00093098008F3B7098093F787083EC0010072
:102FF0000100930A700523005405130A80FA230088
:10300000440501000100231124032310940223002E
:1030100004048247F3A7078001000100294597F0C7
:10302000FF1FE7802031F3B9098093F989084EC268
:1030300001000100230054052300440501000100A4
:103040008357040293E707202310F40223000404AB
:103050009247B9B7B7170040884742054181937737
:10306000050491EB9377F5013755E80113050580C9
:103070003345F50282809377050C130700046397AC
:10308000E7009377F50137459C1CCDB72165130503
:1030900005D0828037E700E01C435443A183E20659
:1030A000D58F1CC1FD572320F7182322F7188280E3
:1030B00013178500B7E700E023A0E710618123A282
:1030C000A7108280B7F700E08847CC47828081470D
:1030D00037370040A14663C4C7003285828003456C
:1030E000B740E38EA6FE3385F5000345050085074E
:1030F0002304A740CDB797070020938727EF9C4371
:1031000017370020130707213E95636EE500173738
:1031100000201307274F6368A70017070020232705
:10312000A7EC3E858280FD57EDBF8280411122C40D
:1031300006C62A8497000000E78000F22947B307FB
:10314000E502B2408D83B3D7870222449507B3D7F7
:10315000E70237370040C207C1832316F700410159
:103160008280411137150E0006C697000000E780E7
:1031700020FCB7370040130770F82381E7000D47A4
:10318000A381E70013070004A380E7000547238716
:10319000E700B24041018280B737004003C7170003
:1031A00019C9D98DA380B70003C70700136787002B
:1031B0002380E700828093C5F5FFF98DA380B700D7
:1031C0008280AE872A87B7360040214637380040D4
:1031D00089E717030000670083F583C8B600E30999
:1031E00016FF05078348F7FFFD17C20723041801E0
:1031F000C183F9BF411122C406C62A84970000008A
:10320000E78080E52947B307E502B2408D83B3D755
:10321000870222449507B3D7E70237370040C20739
:10322000C1832316F7404101828071654111130566
:10323000052006C697000000E78000FCB737004075
:10324000130770F82381E7400D47A381E740130778
:103250000004A380E74005472387E740B2404101CF
:103260008280CC41411106C6328503C6150083C554
:10327000050022064D8E42068D654186138875A293
:10328000630C0611634BC804138845A26300060D46
:10329000634AC800938535A26301B60823900600EF
:1032A00029464DA0138855A26305060D938565A296
:1032B000E316B6FE8D451D4663E6E5081146198EF8
:1032C00063F3C7003E86B7E704002390C600FC47BF
:1032D00097D50100938545009DA0138895A26303AF
:1032E0000611634E060D1388A5A26300061393858D
:1032F00005A5E315B6FA99451D4663E5E504198E63
:1033000063F3C7003E86B7E704002390C600FC477E
:10331000970500209385C5D71DA09D451D4663E3F5
:10332000E5022146198E63F3C7003E86B7E7040025
:10333000FC472390C6009705002093852538BA9551
:1033400082970146B240328541018280AD451D46DB
:10335000E3EAE5FE3146198E63F3C7003E86B7E720
:1033600004002390C600FC4797D50100938545F9DA
:10337000F9B7B1451D46E3E7E5FC3546198E63F321
:10338000C7003E86B7E704002390C600FC4797D5E8
:1033900001009385E5F765B78D451D46E3E4E5FA41
:1033A0001146198E63F3C7003E86B7E704002390E9
:1033B000C600FC4797D501009385C5F249B78D45F6
:1033C0001D46E3E1E5F81146198E63F3C7003E861A
:1033D000B7E704002390C600FC4797D5010093850A
:1033E000E5F4B1BFA5451D46E3EEE5F42946198E87
:1033F00063F3C7003E86B7E704002390C600FC478E
:1034000097D501009385C5EE1DBFB5451D46E3EB7D
:10341000E5F23946198E63F3C7003E86B7E704002C
:103420002390C600FC4797D501009385E5E901BFCD
:10343000B7E7040003A3071397060020938646C44A
:103440004146A54517050020130585BA02832D4581
:103450005DE703C505000947631FE50803A84500AC
:10346000411106C6034718003285034608002207AB
:103470004168518F930828FE6307170563E9E80048
:1034800005186303070323900600294591A8130636
:1034900048FE630AC7041518E31707FF15463E8761
:1034A000637BF600154701A8130600023E8763748C
:1034B000F60013070002B7E704002390E600FC477C
:1034C0001316070111A83E8691C30546B7E704000D
:1034D000FC472390C6004206CC45418282970145B5
:1034E000B24041018280130600083E87E375F6FC76
:1034F00013070008C9B72390060005458280828023
:10350000416779176304E504411122C406C6854763
:103510002A84639FF500B7E7040022852244B24065
:1035200003A3871397050020938585334101028308
:1035300089476399F500B7E7040083A7070B854522
:10354000829771D9B2402244410182808280797190
:1035500026D252CCAE842A8A97D50100938505DF06
:1035600017D50100130505E106D63AC622D44AD084
:10357000368432894ECE97C00100E7806080A285F4
:1035800017D50100130505E097B00100E780407FE3
:10359000294597C00100E780808383C7840093F7A3
:1035A0000702F9E383C9040089470545324763965A
:1035B000F908D44083C7160083C60600A207D58F3A
:1035C000C166138616FE638CC7028D16638FD706FD
:1035D0008D669386269029456391D706B7E7040048
:1035E000A286225403A34714B250F2494A86A68504
:1035F000025992545285624A8547456102832D459E
:103600000DEF93070002354563E98702B7E7040031
:10361000FC47C84413060002CA8582978149970770
:1036200000209387A7249C43014581CB9C4391C7ED
:103630004E852286CA8582970145B2502254925403
:103640000259F249624A456182802D457DF7930710
:10365000700F3545E3E387FEB7E70400FC47C84435
:103660002286CA85829765BF2145C1BF411122C408
:1036700037E404008327841326C2AA84416506C662
:10368000970500209385C51D7D1582978327C40A61
:1036900017050000130505E78588829795C0032369
:1036A00004132244B2409244970600209386C6AF8A
:1036B0004146C545170500201305059E41010283BB
:1036C000B2402244924401454101828019C59707C6
:1036D000002023ADA718014582804545828011470F
:1036E000636AA70A97D60100938606C50A05369530
:1036F0001841411106C63697AE87B2850287130777
:1037000000026145639DE700B7E70400FC4713062C
:103710000002170500201305E5FA82970145B24023
:103720004101828005476145E39BE7FEB7E704005E
:10373000FC470546170500201305C5FAF9BF130716
:10374000700F6145E39DE7FCB7E70400FC471306F3
:10375000700F17050020130525F9C1B713070008DE
:103760006145E39EE7FAB7E70400FC47130600084B
:10377000170500201305C5064DB715476145E390B1
:10378000E7FAB7E70400FC471546170500201305C4
:10379000650D61B709458280411126C2B7E4040076
:1037A00083A7C41322C44AC006C62E8497050020EE
:1037B0009385050B2A898297058905C597070020FF
:1037C0009387878D83D7A70BA28503A3440D23106E
:1037D000F4002244B24092444A8502490146410124
:1037E0000283B24022449244024949454101828009
:1037F00097070020238E07069707002023AC0706B3
:10380000B717004003A7070CB706C0FFFD16758F5A
:1038100023A0E70C03A7070DB7064000558F23A888
:10382000E70C03A7070C3D9B23A0E70C03A7070D9C
:103830001367070123A8E70C8280B717004003A590
:10384000470C83A7470C598113451500C18B058987
:1038500099E3136525009707002083C767016380FC
:10386000A702970700202385A70011C9970700200A
:103870009387470003A3070063030300028382804A
:10388000114517F3FFFF670003CA011122CC06CED2
:103890003714004026CA4AC84EC652C48344740531
:1038A000034AB405834984050349940597F0FFFF53
:1038B000E78040A28347A40593F4F40F137AFA0F2C
:1038C00093E71700230DF40493F9F90F1379F90F17
:1038D000B717004003C7A705058B6DFF03D5C705C4
:1038E000A38D4705238C3705A38C2705A38B97044D
:1038F000F2406244D2444249B249224A0561828080
:1039000041119397050122C406C626C2C1872E84A1
:1039100063DC0700B7E40400FC54829719C1BC546F
:1039200082972165218D15A893F7150013C5150001
:103930008DE793F725009DC797000000E78020F0F2
:10394000B7E70400BC4F1306000A8945170500209D
:103950000345C5F2829713452400B24022449244A5
:10396000410182809397250163D80702B7E40400E0
:1039700083A7C41E829797000000E780A0F0BC4C8C
:1039800037560700130606308965170500200345E2
:10399000E5EE8297096579B7939715010145E3DE56
:1039A00007FA17D501001305E5A597B00100E780D8
:1039B0000055B7E70400BC4F130600649165170576
:1039C00000200345A5EB82971165A9BF1D71A2CC0C
:1039D00037E404005C5C485886CE494697D5010020
:1039E0009385C59D829711E917D501001305459E62
:1039F00097B00100E780A05001A0B7F600E079572A
:103A000098CAFD57DCCA0567B7E700E023A0E710B6
:103A10001306F00290C223A0E71801000100370747
:103A2000002018471306000481459706002023A5AF
:103A3000E6E44157A38AE7403C4408088297971779
:103A40000020938727803EC88567138707409387A8
:103A500057D1231AE1002312F1021307B00F97F791
:103A6000FFFF938767662310E1023ED8154797074B
:103A700000009387C7E1B7F50700A30FE1003EDC24
:103A80000547970700009387E7DF81463000E1058F
:103A900019452301E1023EDE97F0FF1FE78060D465
:103AA00018088147994630003E9603460600850770
:103AB0000507A30BC700E398D7FEC24791C703577A
:103AC000410185676373F70001A0B7E7040083A78E
:103AD000470A08088297AA8511C917D5010013055E
:103AE000659097B00100E780A02901A0F6406644E8
:103AF00025618280411126C2B7E4040083A704082F
:103B000006C622C4170500001305C5DF82971704F7
:103B100000201304A4D62300A40097000000E7802F
:103B2000800297000000E780E0CC034504002244B7
:103B300003A38405B2409244130600328965410113
:103B40000283797106D622D413078008F3370780E1
:103B500093F787083EC201000100B71700409305A4
:103B600070052380B704130680FA2380C704010080
:103B7000010083C6F70293F6A60FA387D70223801E
:103B800007049246F3A60680010001007337078000
:103B9000137787083AC4010001002380B70423800B
:103BA000C7040100010003C7F70213672700A387BA
:103BB000E70223800704A247F3A707800100010062
:103BC000054597E0FFFFE780207497000000E7803D
:103BD00060CB014781468147054685451305407EF8
:103BE00097E0FFFFE780207737E404003C4468005B
:103BF000514681458297B707C0A83EC8B787E803FA
:103C0000938707D03ECA97E7FF1F9387477B3EC63F
:103C10007C5868008297B2502254456182804111DD
:103C200097D50100938505E217C50100130585743A
:103C300006C697B00100E780A01417D50100130550
:103C4000A5FA97B00100E780A013B24029454101D1
:103C500017B301006700A317411197D501009385A1
:103C6000A5DF17C501001305E57006C697B0010072
:103C7000E780001117D501001305C5F597B00100C5
:103C8000E7800010B2402945410117B301006700E9
:103C90000314411122C406C6834705002A849DC728
:103CA00097D50100938585E217C501001305856C42
:103CB00097B00100E780C00C4C4017D501001305F8
:103CC000A50797B00100E780A00B3DA058410DEF7C
:103CD00097D50100938585DF17C501001305856918
:103CE00097B00100E780C00917D50100130545060C
:103CF00097B00100E780C0082244B2402945410145
:103D000017B301006700A30CA1679386D703631361
:103D1000D70297D50100938565DB17C50100130510
:103D2000656597B00100E780A00517D50100130570
:103D300025037DBFED0797D50100938525D917C5CC
:103D4000010013052563631BF70097B00100E780AE
:103D5000200317D501001305E50159BF97B00100F5
:103D6000E78000024C4017D501001305A50291BF62
:103D7000411197D50100938565CF17C50100130543
:103D8000655F06C697B00100E78080FFB240294515
:103D9000410117B3010067008303797122D426D251
:103DA0004AD02E842A898145B2844800714606D6BD
:103DB00097E0FFFFE780A03597F7FF1F9387C76065
:103DC000DC4783D70700231421012313F100975008
:103DD0000000E78080119547A305F1009307401F7D
:103DE0003EC6FD572305A100230AF10097500000AD
:103DF000E780E0232686A285480097500000E780F0
:103E0000A011B2502254925402594561828041114E
:103E1000814617F6FF1F13066657854517050020D4
:103E20000355452706C697C00000E780206715C9DF
:103E300097D50100938505C617C501001305855365
:103E400097B00100E780C0F317D501001305C5EA5C
:103E500097B00100E780C0F2294597B00100E780E4
:103E600000F797D501009385E5C217C5010013053A
:103E7000655097B00100E780A0F017D50100130549
:103E8000E5E897B00100E780A0EF294597B0010071
:103E9000E780E0F397F7FF1F93870753DC47054759
:103EA00097D50100938505BF2390E70017C5010052
:103EB0001305454C97B00100E78080EC17D5010051
:103EC000130505E697B00100E78080EBB240294575
:103ED000410117B30100670083EF17250020035548
:103EE000E5869307E5FFC2072167C1839306D7FFE5
:103EF00063F5F6029707002083C7479997060020CD
:103F000083C6D698A207D58F9306E7FFFD8E1305CB
:103F1000001081C67D1733F5E7008280411126C26B
:103F2000B7E40400FC4406C622C44AC02A844146C1
:103F300097D50100938585E817F5FF1F1305054602
:103F4000829797000000E78080F917090020130985
:103F5000091E2310A90097D501009385E5B417C564
:103F600001001305254197B00100E78060E183550A
:103F70000900228617D50100130585E897B00100D6
:103F8000E78000E0294597B00100E78040E4228601
:103F9000224403A38405B24092440249170500203D
:103FA0000345458E894541010283011122CC06CE8D
:103FB00026CA4AC84EC693F715002E84A5CB970093
:103FC0000000E78000E5930710F817070020230D95
:103FD000F7169707002083D7A70B914517050020F8
:103FE0001305851617070020A300F716A1831707EE
:103FF0000020230CF71497070020A388071497606C
:104000000000E78020B597200000E780C04E0545FE
:1040100097600000E78000BD93441400F2406244C2
:1040200026854249D244B2490561828093F7250032
:10403000E9CF170700200357870F69C7AD64B71989
:1040400000409384A4AA23A0990097060020938699
:10405000660E944297D70100938787DE17060020EB
:104060000346060D814517F5FF1F1305253397708D
:104070000000E780605E23A0990097F7FF1F23915F
:10408000A7242A8941C197D501009385A5A917C501
:1040900001001305252E97B00100E78060CECA8588
:1040A00017C501001305C54497B00100E78040CD56
:1040B000294597B00100E78080D197070020239819
:1040C0000706930710F817070020230FF706970736
:1040D000002083D7E7FB17070020A307F706A1837B
:1040E000170700202303F70691458D471705002089
:1040F0001305850517070020A309F7049760000042
:10410000E78040A59344240011BF93F70510C5C371
:10411000AD64371900409384A4AA23209900171591
:1041200000200355A56297200000E7800068232047
:10413000990097000000E78080DA2A899700010043
:10414000E78040EA9344041031C51714002003545B
:1041500024636311240597D501009385A59C17C599
:1041600001001305252197B00100E78060C1A285F9
:1041700017C501001305853997B00100E78040C0DD
:10418000294597B00100E78080C497200000E780B0
:10419000803669B5B7E70400BC4F130600149305D9
:1041A000004017F5FF1F0345E56D829785BD93F726
:1041B000054091CFAD67371700409387A7AA1CC36E
:1041C00097E0FF1FE780C0089344044081BD8564E9
:1041D00093840480B3F7950099CFAD6737170040FB
:1041E0009387A7AAA18C1CC3C20497200000E78074
:1041F000803BC18025B593F705209DCFAD6737176C
:1042000000409387A7AA1CC397000100E78080DDC8
:1042100009CD854717070020230AF7F097700000A3
:10422000E780605393440420D5BB13050032970008
:104230000000E780E0CEFDB793F74500D1C397D5E6
:1042400001009385258E17C501001305A51297B0AF
:104250000100E780E0B217C501001305E52C97B017
:104260000100E780E0B1294597B00100E78020B662
:10427000930720F8170700202308F7EC9707002082
:1042800083D747E317070020A300F7ECA1831707A4
:104290000020230CF7EA854717070020A307F7EA59
:1042A00097500000E780A0D891451705002013051E
:1042B000A5E997600000E780E08993444400B9BB1A
:1042C00093F78500A9C797D501009385A58517C5E4
:1042D00001001305250A97B00100E78060AA17C501
:1042E00001001305A52597B00100E78060A92945C5
:1042F00097B00100E780A0AD9344840097070020A9
:10430000239707E297700000E780E04401BB93F732
:104310000501D1C38545170500200355A5D9976030
:104320000100E780E0FA97C501009385A57F17C5D6
:1043300001001305250497B00100E78060A417C5AC
:1043400001001305E52097B00100E78060A329452F
:1043500097B00100E780A0A7930730F81707002067
:104360002304F7DE9707002083D7C7D41707002060
:10437000A30CF7DC8D45A183170500201305C5DCD0
:10438000170700202303F7DC934404019750000033
:10439000E780407C61B193F70502D1C797C5010062
:1043A0009385457817C501001305C5FC97B001003A
:1043B000E780009D17C501001305C51B97B00100DC
:1043C000E780009C294597B00100E78040A0930753
:1043D00040F8170700202309F7D69707002083D756
:1043E000A7CB17070020A301F7D6A183170700204A
:1043F000230DF7D4854717070020A308F7D49707A4
:104400000020239B07C897500000E78040C29145D9
:1044100017050020130545D397500000E7808073EF
:1044200093440402E5BE93F70504FDC397C501005C
:104430009385456F17C501001305C5F397B00100BB
:10444000E780009417C501001305451497B00100DB
:10445000E7800093294597B00100E78040979707D0
:10446000002083C767CE1307700A6386E706130729
:10447000800A638CE7081307600A6393E7049307D5
:1044800060F8170700202301F7CC9707002083D797
:10449000C7C917070020A309F7CAA183170700207F
:1044A0002305F7CA854717070020A304F7CAB145BB
:1044B00017050020130545C997500000E780806963
:1044C00097500000E780A0B69344040497070020AB
:1044D000239D07C4A1B6930770F817070020230592
:1044E000F7C69707002083D747C417070020A30DFE
:1044F000F7C4A183170700202309F7C485471707CE
:104500000020A305F7C4994565B7930780F8F1B774
:1045100093F705088144E38307B097C501009385AD
:10452000656017C501001305E5E497B00100E78059
:10453000208517C501001305E50697B00100E78047
:104540002084294597B00100E78060889307A0F890
:1045500017070020230AF7BE9707002083D7C7BD9F
:1045600017070020A302F7BEA18317070020230E20
:10457000F7BC854717070020A309F7BC9707002061
:10458000239C07BA97500000E78060AA9145170561
:104590000020130565BB97500000E780A05B9344A3
:1045A0000408ADBC411122C497C501009385455351
:1045B0002A8417C501001305E5DB06C697A0010094
:1045C000E780007C4C4017C501001305657097A07B
:1045D0000100E780E07A294597A00100E780207F6D
:1045E000034704009307F00F631FF70297C501000C
:1045F0009385054F17C501001305C5D797A0010086
:10460000E78000784C4017C501001305656D97A041
:104610000100E780E0762244B2402945410117A31A
:1046200001006700C37AB2402244410182809707AB
:1046300000202391A7A697070020239BB7A48547B6
:10464000411117170020231DB71217C501001305CC
:1046500065D297C501009385E54217070020231A0C
:10466000F7A217170020230FF7FC06C697A001003A
:10467000E78000719715002083D5851017C50100CC
:104680001305857A97A00100E780806F294597A0E0
:104690000100E780C07397F7FF1F9387E7D2DC47DD
:1046A00003D70700C167FD176310F702B7E70400DF
:1046B000B24003A3870517F5FF1F0345A51C13068A
:1046C000000A854541010283B24041018280B1C1A7
:1046D000411122C417C501001305C5C92E8497C511
:1046E00001009385653906C697A00100E7804069FF
:1046F000A28517C501001305E56F97A00100E780AB
:1047000020682244B2402945410117A301006700F7
:10471000036C8280971700202394070697170020C8
:10472000238207F2B7E70400FC47411106C6414661
:1047300097C501009385856717F5FF1F130505C60B
:10474000829717070020034727A09307F00A6315F5
:10475000F7029307F0F88945170500201305C59E59
:10476000170700202302F79E97070020A38E079CBF
:1047700097500000E780003E97500000E780606996
:104780008145370504009707002023A5079A97075E
:104790000020239E079897070020238B07989707F0
:1047A000002023990790970700202397078E9707EB
:1047B0000020239C079697070020239F0796973099
:1047C0000000E78000C1014597500000E78080416C
:1047D0009707002083C787951305003299C797076D
:1047E00000202385079413050064B240410117F3AC
:1047F000FFFF6700E372B7E7040003A38705130612
:1048000000149305001017F5FF1F0345A507028349
:10481000B7E7040003A38705856513060014938595
:10482000058017F5FF1F0345E5050283797122D442
:1048300037E404005C5C06D6354697C501009385D5
:10484000E53B17D501001305E513829711E917C55C
:1048500001001305E5B797A00100E780406A01A0B9
:1048600097F7FF1F9387C7023ECCB7F50700856710
:1048700093870780814617F6FF1F1306E600E105C0
:1048800019453ECE97E0FF1FE780A0F57C4419460E
:1048900097F5FF1F938545FF170500201305C58178
:1048A0008297340817F6FF1F130606FE97D50100FE
:1048B0009385058B17D501001305058C97700000B3
:1048C000E78080AE2A841DCD97C50100938585249D
:1048D00017C50100130505AA97A00100E780404A0B
:1048E000A28517C501001305653297A00100E78076
:1048F0002049294597A00100E780604DB25022541D
:104900004561828097E00000E780801417C50100B0
:104910001305C52697600000E780C0A297A000009D
:10492000E780C06897600100E78040CD17F5FF1F62
:10493000130505A597600100E780E0B517C50100E4
:104940001305C52497600100E780C0CD2A849760D5
:104950000000E780000997100100E78020A59780FC
:104960000100E780403E97700000E780E0649760B8
:104970000000E780007F97300100E780806697C5E0
:1049800001009385251917C501001305A59E19C8B7
:1049900097A00100E780C03EA28517C5010013055E
:1049A0002529A1B797A00100E780803D17C5010028
:1049B0001305452A97A00100E780803C294597A070
:1049C0000100E780C04097300100E780604297F027
:1049D0000000E78020616309051485453705040060
:1049E00097300000E780E09E97C50100938585120F
:1049F00017C501001305059897A00100E78040380E
:104A000017C501001305852697A00100E7804037F0
:104A1000294597A00100E780803B97F7FF1F938708
:104A2000278983D7070017170020231BF7D4854752
:104A3000171700202308F7C097F7FF1F9387C79821
:104A4000DC4703D70700C167FD176316F70097F02F
:104A5000FFFFE780003C97700000E78000E013054F
:104A6000C51497700000E78000E097200000E78001
:104A7000A0BF97200000E78000A81715002003556D
:104A800025D097500000E78040E205459750000090
:104A9000E780401597F0FFFFE780604497170020FC
:104AA00083D707CE2AC6638CA70497C501009385D8
:104AB000650617C501001305E58B97A00100E78087
:104AC000202C32469715002083D585CB17C50100D1
:104AD0001305051C97A00100E780802A294597A0AF
:104AE0000100E780C02EB7E70400BC4F1306006446
:104AF0009305002017F5FF1F0345C5D8829797C57A
:104B000001009385250117C501001305A58697A00F
:104B10000100E780E02617C501001305251A97A0BC
:104B20000100E780E025F1B397500000E780800B9B
:104B30001305003297F0FFFFE780803EC9B74111AF
:104B400022C437E404008327041A06C682979750CC
:104B50000000E78040D98327040817F5FFFF1305FD
:104B60000545829797F7FF1F238EA7D017F5FF1FE4
:104B70001305858597400000E780007E2244B240FF
:104B80004101170300006700A3CAB7E70400FC4710
:104B90001171A2DDCAD986DFA6DBCED72E84328979
:104BA0002E86AA8517F5FF1F1305055A829717F75A
:104BB000FF1F1307675983470700930680029387F7
:104BC000E70793F7F70FE3ECF610BA898A0717C7E0
:104BD000010013076783BA979C43BA9782878D4772
:104BE00097C50100938545F517B501001305857834
:104BF000630FF40097A00100E780801817C501003B
:104C00001305C5B097A00100E7808017BDA497A049
:104C10000100E780E01617C501001305A5B097A0B5
:104C20000100E780E015294597A00100E780201AE0
:104C3000930720F8114697F5FF1F9385E5504A85A5
:104C400017F7FF1F2302F75097F7FF1FA38F074E99
:104C500097F0FFFFE780A0142A841DC997C50100C3
:104C6000938585ED17B501001305C57097A0010068
:104C7000E7800011A28517C50100130565AE97A056
:104C80000100E780E00F294597A00100E78020148C
:104C900097C50100938545EA17B501001305856D99
:104CA00097A00100E780C00D17C50100130585AC72
:104CB00097A00100E780C00C294597A00100E7807C
:104CC00000114165930730FA054697F5FF1F93855C
:104CD000A5477D1517F7FF1F2308F74697F0FFFF3D
:104CE000E780E00B2A841DC997C501009385C5E4C0
:104CF00017B501001305056897A00100E78040087B
:104D0000A28517C501001305A5A597A00100E7809E
:104D10002007294597A00100E780600BB7E7040052
:104D2000BC4F0566130606C8A14517F5FF1F0345CE
:104D300065B58297FE506E54DE544E59BE591161CE
:104D4000828091476303F40297C501009385C5DE15
:104D500017B501001305056297A00100E780400226
:104D600017C50100130545A471BDB7E70400FC4F4A
:104D7000914517F5FF1F0345E5B0829797C50100E0
:104D8000938585DB17B501001305C55E97A001006B
:104D9000E78000FF17C501001305C5A297A0010019
:104DA000E78000FE294597A00100E7804002974078
:104DB0000000E780C027914535A485476303F402CE
:104DC00097C50100938545D717B501001305855A8E
:104DD00097A00100E780C0FA17C50100130505A0E0
:104DE00015B597F7FF1F2397272DB7E70400056632
:104DF000BC4F130606C8C1450DBF8D476303F402BF
:104E000097C50100938545D317B501001305855655
:104E100097A00100E780C0F617C501001305C59DE6
:104E2000D5B3930740F8114697F5FF1F9385C53119
:104E30004A8517F7FF1F2309F73097F7FF1FA3864F
:104E4000073097F0FFFFE78080F52A84E30405EE42
:104E500097C50100938545CE17B50100130585510F
:104E600097A00100E780C0F1A28517C501001305D6
:104E7000258F97A00100E780A0F0294597A00100A9
:104E8000E780E0F445BD9147E31CF4F6B7E7040082
:104E9000FC4F9305000217F5FF1F0345A59E82975F
:104EA00097C50100938545C917B501001305854CC9
:104EB00097A00100E780C0EC17C5010013054595D8
:104EC000F1BD894763E3870297C501009385C5C695
:104ED00017B501001305054A97A00100E78040EAD5
:104EE00017C501001305059431BB97F4FF1F83C458
:104EF000C42597F7FF1F83C7372597C50100938502
:104F0000A5C3A20417B501001305C546DD8C97A003
:104F10000100E780E0E6A28517C501001305C591F1
:104F200097A00100E780C0E5C204294597A00100D1
:104F3000E780E0E9C1849305D4FF93960401C18220
:104F40004A8693F5F50F17F5FF1F130515209720D7
:104F50000000E780C04BE35F90DC930750F817F741
:104F6000FF1F2303F71E83C73900228697F5FF1F13
:104F70009385851D85074A8517F7FF1FA307F71C33
:104F800097F0FFFFE780A0E12A84E30505DA97C5E3
:104F90000100938565BA17B501001305A53D97A0DB
:104FA0000100E780E0DDA28517C50100130585E358
:104FB000C9B5894763E3870297C501009385C5B7E3
:104FC00017B501001305053B97A00100E78040DB02
:104FD00017C501001305058835B197400000E7802B
:104FE0000005A28517F5FF1F130505169750000051
:104FF000E78040B681B38D476303F40297C5010093
:10500000938585B317B501001305C53697A0010038
:10501000E78000D717C5010013058585E5B6B7669B
:1050200002000146B7750200054597D0FF1FE780D3
:10503000407B930760F817F7FF1F2307F71097F7D8
:10504000FF1FA38407109307000617F7FF1F230F06
:10505000F70E894717F7FF1FA30AF70E97F7FF1FF1
:105060002387070E97F7FF1FA383070EC14717F784
:10507000FF1F230FF70C930720F917F7FF1FA30952
:10508000F70C314697F7FF1FA385A70C97F5FF1F75
:105090009385850B4A8597F7FF1F238C070A97F0A6
:1050A000FFFFE780C0CF2A84E30605C897C501004B
:1050B000938585A817B501001305C52B97A001009E
:1050C000E78000CCA28517B501001305E57B55B339
:1050D000B1476303F40297C501009385E5A517B5B1
:1050E00001001305252997A00100E78060C917B5C5
:1050F00001001305257B39B6B7E70400FC4F930583
:10510000000417E5FF1F0345E577829797400000ED
:10511000E780E0F1B145F9B5914763E3870297C5B0
:105120000100938565A117B501001305A52497A07B
:105130000100E780E0C417B5010013056578D9B414
:1051400097F4FF1F83C4840097F7FF1F83C7F7FFFF
:10515000A204DD8C8E04B77702006D14BE94228603
:10516000A68517B501001305E57697A00100E78035
:1051700020C1B7E70400FC47228697F5FF1F9385FF
:10518000F5FC2800829793160401C1823000A685A1
:10519000094597D0FF1FE780C0642A8409C917B565
:1051A00001001305E57497A00100E78040D593073F
:1051B00070F8194697F5FF1F938505F94A8517F78B
:1051C000FF1F2303F7F897F7FF1FA38187F897F0D6
:1051D000FFFFE780C0BC2A84E30E05B497C5010039
:1051E0009385859517B501001305C51897A0010093
:1051F000E78000B9A28517B501001305657095B960
:105200009947630BF41297C501009385E59217B592
:1052100001001305251697A00100E78060B617B5B9
:1052200001001305656FF9BA914763E3870297C5DB
:1052300001009385659017B501001305A51397A08C
:105240000100E780E0B317B501001305656E5DBA94
:1052500097F4FF1F83C484EF97F7FF1F83C7F7EE10
:10526000A204DD8C8E04B77702006D14BE942286F2
:10527000A68517B501001305E56C97A00100E7802E
:1052800020B0B7E70400FC47228697F5FF1F9385FF
:10529000F5EB2800829793160401C1823000A685A1
:1052A0000D4597D0FF1FE780C0532A8409C917B561
:1052B00001001305E56A97A00100E78040C4930749
:1052C00080F8194697F5FF1F938505E84A8517F77B
:1052D000FF1F230BF7E697F7FF1FA38987E697F0D9
:1052E000FFFFE780C0AB2A84E30605A497C5010051
:1052F0009385858417B501001305C50797A00100A4
:10530000E78000A8A28517B501001305A56695B62C
:1053100099476303F40297C501009385E58117B5AA
:1053200001001305250597A00100E78060A517B5CA
:1053300001001305A565F9B0B7E70400FC4F93051C
:10534000000417E5FF1F0345E553829797400000CF
:10535000E780E0CD994579B18D476303F40297B5B5
:1053600001009385657D17B501001305A50097A081
:105370000100E780E0A017B501001305A56259B050
:1053800017B501001305056397A00100E78020B75A
:105390001305C01297D0FF1FE780A0FA014597E0E0
:1053A000FFFFE78060CF0D4597100000E78080A0E9
:1053B000294597D0FF1FE780C0F897D0FF1FE780EF
:1053C00020E98DBA99476303F40297B501009385EC
:1053D000A57617B501001305E5F997A00100E78050
:1053E000209A17B501001305A55D29B817F7FF1F0F
:1053F0000347D7D597F7FF1F83C747D522075D8F90
:105400009166BA96C2061166C1821306F6EF8D4701
:105410006365D60297E7FF1F938707FB9C4B17F640
:10542000FF1F034696D29386C7002DC203D60700FE
:1054300069CA8907E39CD7FE89471307A0F811467C
:1054400097F5FF1F938545D04A8597F6FF1F238D5B
:10545000E6CE17F7FF1FA30AF7CE97F0FFFFE7800E
:1054600000942A84E308058C97B501009385C56CE8
:1054700017B50100130505F097A00100E7804090E3
:10548000A28517B501001305E554E5B203D6070060
:10549000630EE60A8907E39BF6FE8D4779BF9147C5
:1054A0006304F40297B501009385056917B50100FF
:1054B000130545EC97A00100E780808C17B501002B
:1054C0001305C5526FF00FF4B7E70400FC4F9305C6
:1054D000000817E5FF1F0345E53A8297C9B897B55D
:1054E00001009385656517B501001305A5E897A030
:1054F0000100E780E08817B501001305A5506FF0A3
:105500006FF02390E70017E5FF1F1305E5EB9730D9
:105510000100E78060B397B501009385E56117B599
:105520000100130525E597A00100E780608517B508
:1055300001001305254E97A00100E78060842945EE
:1055400097A00100E780A0888147C5BD2390070090
:1055500017E5FF1F130545E797300100E780C0AE50
:1055600097B501009385455D17B50100130585E0EA
:1055700097A00100E780C08017B501001305054B17
:105580005DBF411122C406C6834705002A849DC71A
:1055900097B501009385055617B50100130585DD04
:1055A00097900100E780C07D4C4017C501001305AE
:1055B000258A97900100E780A07CC9A85841B707C9
:1055C000CF009387777D6312F70897B50100938525
:1055D000655217B501001305E5D997900100E780E2
:1055E000207A1C448356E4008355C40003C6070098
:1055F00017C501001305458797900100E7804078A3
:10560000294597900100E780807C0357E4009707C5
:10561000002083D7E716630EF7008355C4000844C3
:105620008547170700202302F71297300000E78014
:10563000A03F0356E4008355C40008442244B2400E
:10564000410117F3FFFF67008354B707CC0093872E
:10565000777D6315F70497B501009385A54917B5C4
:105660000100130525D197900100E78060711C446B
:105670008356E4008355C40003C6070017B5010034
:105680001305857E97900100E780806F2244B24029
:10569000294541011793010067006373B707CE00E6
:1056A0009387777D6304F70297B50100938585445E
:1056B00017B50100130505CC97900100E780406CF9
:1056C0004C4017B501001305E56CE5B5B240224426
:1056D00041018280B7E70400FC4741112E8606C6CF
:1056E00022C426C24AC02E842A89AA8517F5FF1F24
:1056F000130585A5829797B501009385A54517B534
:105700000100130525C797900100E780606797F5B2
:10571000FF1F83C565A317B50100130525EA979000
:105720000100E780E065294597900100E780206A45
:1057300097F4FF1F938444A183C7040041479387D4
:10574000070693F7F70F636EF75A17B701001307B1
:10575000E7D58A07BA979C43BA9782879D47630724
:10576000F40297B501009385E53E17B501001305D6
:1057700065C097900100E780A06017B50100130590
:1057800065E497900100E780A05F8DA497F7FF1F65
:1057900083C7979BDDCB17F7FF1F0347179B97F72F
:1057A000FF1F83C7879A22075D8F97F7FF1F83C765
:1057B000E799C2075D8F97F7FF1F83C73799E20705
:1057C000D98F17F7FF1F2327F79683C7640097B574
:1057D00001009385253817B501001305A5B917F702
:1057E000FF1F2307F79497900100E780605997F710
:1057F000FF1F938727948C4317F6FF1F034646939A
:1058000017B501001305C5DD97900100E7804057EB
:10581000294597900100E780805B97F7FF1FA385DC
:1058200007922244B24092440249930700F817F7C6
:10583000FF1F230BF7909D4517F5FF1F1305C5901C
:105840004101174300006700E33097600000E780E4
:10585000000097F7FF1F238AA78E9357850017F73D
:10586000FF1FA304F78E935705012A8417F7FF1F24
:10587000230EF78C93578501014517F7FF1FA307E8
:10588000F78C97600000E780E00097F7FF1F238008
:10589000A78C97B501009385E52B17B5010013057B
:1058A00065AD97900100E780A04D17F6FF1F0346F6
:1058B000068AA28517B50100130505D4B1B7CD47F7
:1058C0006303F40297B501009385C52817B501005D
:1058D000130545AA97900100E780804A17B501009B
:1058E000130505D379BD37E404007C44414697F5A0
:1058F000FF1F9385758517E5FF1F130525AA82975E
:1059000097F7FF1F83C7678517F7FF1F0347D784E4
:10591000A20703238405D98F17F7FF1F2319F780E8
:105920001306000A89452244B2409244024917E511
:10593000FF1F034525F5410102838D476303F402F0
:1059400097B501009385052117B50100130585A2C0
:1059500097900100E780C04217B50100130505DBF1
:105960000DB517E4FF1F0344447E97E7FF1F83C76D
:10597000B77D97B501009385E51D220417B5010099
:105980001305459F5D8C97900100E780603FA285DD
:1059900017B50100130545C997900100E780403E07
:1059A000294597900100E78080420D4697E5FF1F4B
:1059B00093858579228597E0FFFFE780403EAA84A2
:1059C00021C197B501009385E51817B501001305AE
:1059D000659A97900100E780A03AA68517B5010067
:1059E0001305C5C597900100E78080392244B24075
:1059F0009244024929454101179301006700233D64
:105A000097E7FF1F2398876AB7E70400116603A38F
:105A10008705130606E8914539B78D476303F402FD
:105A200097B501009385051317B5010013058594FB
:105A300097900100E780C03417B501001305C5DB5E
:105A400089B317E4FF1F0344447097E7FF1F83C720
:105A5000B76F97B501009385E50F220417B50100D4
:105A6000130545915D8C97900100E7806031A28518
:105A700017B501001305C5BD97900100E7804030C0
:105A8000294597900100E78080340D4697E5FF1F78
:105A90009385856B228597E0FFFFE7804030AA84DD
:105AA0001DC197B501009385E50A17B501001305DF
:105AB000658C97900100E780A02CA68517B50100A2
:105AC000130545BA05B797E7FF1F2397875CB7E72C
:105AD0000400116603A38705130606E89305000278
:105AE00099B5894763E3870297B5010093858506D9
:105AF00017B501001305058897900100E78040283D
:105B000017B50100130505D2ADB997E4FF1F83C493
:105B1000C46397E7FF1F83C7376397B50100938579
:105B20006503A20417B501001305C584DD8C9790A9
:105B30000100E780E024A68517B50100130505B430
:105B400097900100E780C023294597900100E780E6
:105B50000028228697E5FF1F9385055F268597E03D
:105B6000FFFFE780C0232A84630E051A97B5010062
:105B7000938545FE17A501001305C57F9790010089
:105B8000E7800020A28517B50100130565B099BD17
:105B9000854763F98718834519002244B24092442F
:105BA0000249B335B00097E7FF1F238FB75017B5F1
:105BB0000100130525AF4101179301006700431C45
:105BC000A2852244B24092444A850249410117030A
:105BD00000006700632499476303F40297B501004E
:105BE000938545F717A501001305C5789790010027
:105BF000E780001917B50100130585DC59B617E4D5
:105C0000FF1F0344845497E7FF1F83C7F75397B5DB
:105C10000100938525F4220417A50100130585755D
:105C20005D8C97900100E780A015A28517B5010053
:105C30001305C5A897900100E78080142945979027
:105C40000100E780C018194697E5FF1F9385C54FEF
:105C5000228597E0FFFFE7808014AA841DC197B5D5
:105C60000100938525EF17A501001305A5709790F6
:105C70000100E780E010A68517B50100130505A512
:105C800095B397E7FF1F2399874AB7E7040011668A
:105C900003A38705130606E89305000869B1854745
:105CA00097B50100938505EB17A501001305856CD9
:105CB000630BF40097900100E780800C17B501009A
:105CC000130505A27DBC97900100E780600B17B516
:105CD0000100130565A297900100E780600A29453D
:105CE00097900100E780A00E2244B24092440249FE
:105CF00097E7FF1F239D07424101176300006700DC
:105D000083A597B501009385E5E417A50100130568
:105D1000656697900100E780A00617B5010013059E
:105D200065CE85B4B240224492440249410182804A
:105D3000411106C622C497E0FFFFE780400621CD4F
:105D400097E7FF1F83D7673885072A8417E7FF1F68
:105D5000231DF73697B50100938545E197E7FF1FAF
:105D60002396A73617A501001305C560979001007B
:105D7000E7800001A28517B501001305A5069790DD
:105D80000100E780E0FF2244B2402945410117931A
:105D900001006700C30397E7FF1F83D74733B24073
:105DA0002244850717E7FF1F2313F7324101828042
:105DB000411122C491462A8417E6FF1F13060647A5
:105DC0009D652D4506C697D0FF1FE78080A1B7F7D8
:105DD000070003C70701A5476313F70001A0930657
:105DE000001001469D65254597D0FF1FE780609F05
:105DF00097E7FF1F238C87422244B240914617E663
:105E0000FF1F1306A6429D652945410117D3FF1FB9
:105E10006700239D1171CED7B7E9040083A7C90499
:105E2000CAD917E9FF1F13092932A2DD2E8686DFA2
:105E3000A6DB2E84AA854A85829797E7FF1F83C732
:105E4000A7301307700A6385E710636DF700130727
:105E5000600A6385E704FE506E54DE544E59BE5905
:105E6000116182801307800A6385E7161307900A81
:105E7000E393E7FE8D476306F41C97B50100938515
:105E8000250A17A501001305E54E97900100E7804C
:105E900020EF17B501001305E50525A08D47630C1C
:105EA000F40297B501009385A50717A50100130516
:105EB000654C97900100E780A0EC17B50100130531
:105EC000A5FC97900100E780A0EB29459790010081
:105ED000E780E0EF49B7854717B50100130585FC5A
:105EE00017E7FF1F2302F71E97900100E7802001AC
:105EF000B7750200B76602000146054597D0FF1F3F
:105F0000E780208E930760F817E7FF1F230EF72224
:105F100097E7FF1FA38B07229307002617E7FF1FB2
:105F20002326F722E5779387072117E7FF1F231121
:105F3000F722B14597E7FF1F238D072097E7FF1F43
:105F4000A389A7204A8597000000E780E01621B7C3
:105F5000914763E3870297B50100938565FC17A518
:105F600001001305254197900100E78060E117B516
:105F70000100130525F5B1B797E4FF1F83C4041D85
:105F800097E7FF1F83C7771CA204DD8C83A7C90492
:105F90006D14228697E5FF1F9385551B2800829775
:105FA0008E0493160401B7750200C1823000A695D5
:105FB000094597D0FF1FE780C082930770F817E765
:105FC000FF1F2303F718994597E7FF1FA380A71822
:105FD00095BF914763E3870297B50100938545F428
:105FE00017A501001305053997900100E78040D9F6
:105FF00017B50100130585EEE9B597E4FF1F83C4CB
:10600000E41497E7FF1F83C75714A204DD8C83A70E
:10601000C9046D14228697E5FF1F93853513280068
:1060200082978E0493160401B7750200C182300076
:10603000A6950D4597C0FF1FE780A07A930780F8CB
:10604000BDBF17B50100130525EC97900100E7804F
:1060500000EB930790F82304F100834719008D4566
:106060002800A304F100834729002305F1009700CD
:106070000000E78060041305C01297C0FF1FE7808F
:10608000402C014597D0FFFFE78000010D459700A8
:106090000000E78020D2294597C0FF1FE780602AD3
:1060A00097C0FF1FE780C01A7DB397E7FF1F23A7A4
:1060B000A718828097E7FF1F9387471803A307005D
:1060C000630303000283174300006700A3A8411184
:1060D0004AC097F6FF1F83D6A66A328917F6FF1FBC
:1060E0000356C66622C426C206C62A84AE8497001A
:1060F0000000E780A06235C12DC0994763FF970477
:106100008347140003470400A207D98F1397870021
:10611000A183D98FC2073167C1831307C755639E17
:10612000E70297F7FF1F83D76762A301F400A183FB
:106130002302F40097F7FF1F83D7876491C7A30258
:10614000F400A1832303F400A68517B5010013050D
:1061500025E197900100E780A0C297F7FF1F83C752
:10616000674EB9CF97F5FF1F83D5455E17B5010080
:106170001305C5E097900100E78080C02686A285C0
:1061800017F5FF1F0355855C97000000E78080BA74
:106190006301090497E7FF1F83C7870A9DCB95C852
:1061A00097E7FF1F83C747F28DE722852244B2405D
:1061B0000249A68592444101174300006700839974
:1061C00017B50100130585DC97900100E78020D307
:1061D000C1B7B240224492440249410182808347C0
:1061E00055008345450017B50100130525D6A207C4
:1061F000DD8D179301006700A3B817B501001305E3
:10620000E5D317930100670083CF8D4763FBB70A7F
:10621000011126CA06CE22CC0344350097E4FF1FA5
:1062200083C4140297B50100938505D7B337800066
:1062300017E7FF1FA306F70009C497B50100938570
:1062400065D617B50100130565D697900100E78064
:1062500020B397E7FF1F83C7B7FE6386970097E0D9
:10626000FFFFE780205B97E7FF1F83C777FD8DC7A0
:1062700085472306F100B7E7040083A7471770009E
:10628000854513055030829717B50100130505D3D6
:1062900097900100E780A0C69967938757EE231671
:1062A000F100680085479145A30781002307F100AD
:1062B00097000000E78040E0F2406244D24405616C
:1062C00082808280894763F8B70A011122CC06CE0A
:1062D0008347250005472A846393E706914763FCBB
:1062E000B7048347450003473500A207D98F17F746
:1062F000FF1F0357A745630AF70017F7FF1F231770
:10630000F74497E0FFFFE780404F9967938767EE78
:106310002314F10085472305F10083473400A305CA
:10632000F10083474400954528002306F1009700BB
:106330000000E78060D8F240624405618280E5FF9A
:1063400097F7FF1F83D787409386E7FFC206216731
:10635000C18275176376D70097F7FF1F83D747422F
:106360001967130767EEA305F1002314E100230565
:106370000100A1834DBF82800111996722CCD517FE
:1063800017F4FF1F1304042C2314F10083470400A7
:1063900026CA97F4FF1F9384A43E2305F10083D7F8
:1063A000040028009545A305F100A18306CE23062D
:1063B000F10097000000E78020D003D60400834559
:1063C000040017B501001305E5C097900100E780B0
:1063D000209BF2406244D244056182809D677971BE
:1063E000D9172316F10097F7FF1F83C7A72506D6F5
:1063F0002307F100A9C3B7E70400FC47414697D53E
:10640000FF1F9385A5F91305F10082976800CD451C
:1064100097000000E78040CA97F5FF1F83C58522DB
:1064200017B50100130505BE97900100E780409560
:10643000B25045618280B7E70400BC4741468145C0
:106440001305F1008297D9B745C5411106C622C48C
:10645000930750FA2300F5009307A005A300F50069
:1064600089472301F5009147A301F5009307200315
:10647000A302F50097F7FF1F9387C71C83C7070088
:10648000230205002A842303F50097E7FF1F938763
:1064900037DB83C70700414697D5FF1F938505F07B
:1064A000A303F50097F7FF1F83D7872D2304F5007B
:1064B000A183A304F50097F7FF1F83D7272923059E
:1064C000F500A183A305F500B7E70400FC473105FB
:1064D00082972285F14597000000E7802020230E57
:1064E000A4002181A30EA400B24022444101828075
:1064F00082805D710A8586C6A2C497000000E7808D
:10650000E0F437E404007C448A85081079468297D9
:106510003C441305E1030946814582971010930519
:106520000002014597D0FFFFE780A01BB64026443C
:1065300061618280011122CC2D6426CA4AC84EC6F0
:1065400052C456C25AC006CEB71400401304A4AABF
:1065500080C037E900E0B70940002A8AAE8A328B52
:1065600023203919010001008566AA8501462545C9
:1065700097C0FF1FE780E026DA865686D285294538
:1065800097C0FF1FE780E0252320391180C0F2402B
:106590006244D2444249B249224A924A024B0561BE
:1065A00082800111B7C7A55A22CC9387C73317E45D
:1065B000FF1F1304F4C83EC4834704002C00214687
:1065C000196506CE3EC697000000E780E0F68345D9
:1065D000040017B50100130565B197800100E7803D
:1065E000207AF2406244056182800111A1463000A8
:1065F00099652D4522CC06CE97C0FF1FE780601E0F
:10660000A24737C4A55A1304C43363958702B24521
:1066100017B50100130545A1B335B00097E7FF1F7B
:10662000A380B7C297800100E7808075F240624482
:10663000056182809165A1463000938505F02D4566
:1066400097C0FF1FE780E019A247E38287FC8547D8
:1066500017E7FF1FA306F7BE854517B50100130511
:10666000E59EC9B77971D146700091652D4522D458
:1066700006D697C0FF1FE780C016B24737C4A55A99
:106680001304F43563988702B7E70400FC4717D575
:10669000FF1F1305A5D041460C08829717B50100CE
:1066A000130545A097900100E7806085B250225401
:1066B000456182809165D1467000938505E82D453E
:1066C00097C0FF1FE780E011B247E38F87FA17B545
:1066D00001001305259FF9B7C16769768146FD174B
:1066E00005061397060141836364B7003E858280E7
:1066F0003307D50003470700B98F214713F8170068
:10670000858363050800B18FC207C1837D171377A6
:10671000F70F6DF78506F1B741C5A547054763F249
:10672000B70883471500034705003168A207D98FD2
:1067300013978700A183D98FC207C1831308C85557
:10674000054763900707411106C622C426C20344C9
:106750002500914763F087049307540063ECF5022A
:10676000A301C50021822302C5009304340091C611
:10677000A302D500A1822303D5002A84A685970011
:106780000000E780A0F526942300A4002181A30047
:10679000A4000147B240224492443A8541018280DC
:1067A00005473A8582800111B7C7A55A22CC938745
:1067B000E7342A842AC62C002146156506CE3EC43D
:1067C00097000000E78040D7A28517B501001305A8
:1067D000E59397800100E780A05AF240624405618A
:1067E00082800111A146300095652D4522CC06CE50
:1067F00097C0FF1FE780E0FEA24737C4A55A1304E5
:10680000E43463958702B24517B501001305058688
:1068100097F7FF1F239CB7F2C205C1819780010043
:10682000E7800056F2406244056182809165A1468E
:106830003000938505EE2D4597C0FF1FE78060FA75
:10684000A247E38287FC17B501001305258497F75B
:10685000FF1F239D07EE97800100E780406AD9B7AC
:1068600097B701009387878E13D7C5003E970347DC
:1068700007001105230EE5FE13D785003D8B3E97DB
:1068800003470700A30EE5FE13D745003D8BBD89E6
:106890003E97AE970347070083C70700230FE5FE27
:1068A000A30FF5FE8280011122CC06CE26CA4AC86B
:1068B0004EC693F715002E84638E0716AD67938737
:1068C000A7AA371700401CC397F7FF1F83C7E7E746
:1068D00099EF97F7FF1F83C7C7EA850793F7F70F6D
:1068E0001D47636AF70217F7FF1F230CF7E8B7E7A6
:1068F0000400BC4F13060019854517D5FF1F03453B
:10690000A5AE829713451400F2406244D244424936
:10691000B2490561828097F7FF1F238407E6B757C6
:1069200020419304D0039387777497F5FF1F83D595
:1069300025E517F5FF1F1305F5E11309000217F709
:10694000FF1F2327F7E097F7FF1F238597E09700A6
:106950000000E78020F12300250197F7FF1F83C780
:1069600067CEB337F00093870703A301F5009309BF
:10697000000593072004A30035012301950023029D
:106980002501A302F5002303950097D5FF1F83D5AA
:1069900065A31D0597000000E780C0EC23002501DA
:1069A000A3003501930750042301F500A3019500CE
:1069B00097D5FF1F83D5C590110597000000E7808C
:1069C00060EA9307B0042300250123019500A3008A
:1069D000F50097D7FF1F83C7679CA20797D5FF1FB6
:1069E00083C5D59BDD8D0D0597000000E78080E70E
:1069F00097D7FF1F83C7A79AA20797D5FF1F83C505
:106A0000159ADD8D97000000E780C0E5B5472300AB
:106A1000F500A947A300F5009305250017F5FF1F12
:106A2000130505D3898DC205C18197200000E78039
:106A3000C00875BD93F7250081CB97F7FF1F2395FD
:106A400007D013C52500C9B593F745000145E38D6F
:106A500007EA17A501001305256D97800100E7805F
:106A6000004A97300000E780803C1345440069BD30
:106A7000411122C437E404005C5C06C6354697A584
:106A800001009385A51717B501001305A5EF82979F
:106A900011E917A501001305E56997800100E7805A
:106AA000004601A08327041C82972A84054597C0CD
:106AB0000000E78040F997600100E780607E976002
:106AC0000100E780605397B00000E780C00A22858C
:106AD000B2402244410182804111054506C622C4CC
:106AE00026C297C0FFFFE78000451305A00497B0BA
:106AF000FF1FE780C05B757585457D1597C0FFFF5B
:106B0000E780A02E7D7585451305F53697C0FFFFFC
:106B1000E7800038371400408327840A8D45130529
:106B2000002093E707202324F40A97C0FFFFE780A3
:106B3000C02BB7E4040097C0FFFFE780406FC85840
:106B400097800100E780A03B17B50100130585E39E
:106B500097800100E780A03A8327840C8545414552
:106B600093E707082324F40C97C0FFFFE780403227
:106B70008D451305000897C0FFFFE780603197C07F
:106B8000FFFFE780405E37A507001305051297C099
:106B9000FFFFE780E0599D45014597C0FFFFE78073
:106BA000E05FB7E700E03707000423A0E718010023
:106BB000010097D0FFFFE780A0E197D0FFFFE780BB
:106BC000A0F397000000E780E0EA97000000E7806C
:106BD00000A297000000E78000C197E0FFFFE78078
:106BE00040F697000000E780A02597000000E780AE
:106BF000801083A7040817050000130505CB8297B2
:106C000097C7FF1F2382A77EBC4C130600648545EF
:106C1000829797B0FF1FE780A07D01458280AD6716
:106C2000371700409387A7AA1CC3B7E700E03707D0
:106C3000400023A0E71801000100B7F7070003C7D1
:106C40000701A5476316F7009397450191C301A07B
:106C50004111AE860146AA85254506C697C0FF1F8D
:106C6000E78020B8B240B7E700E03707400023A034
:106C7000E710410182804111B2862E86AA852D45FA
:106C800006C697C0FF1FE780C0B5B240014541016D
:106C900082809307000463ECC7041D71A2CC2A8490
:106CA0000808A6CACAC886CE32C697800100E78007
:106CB000C001AD67371700409387A7AA1CC3B7E48C
:106CC00000E03709400023A0241901000100B2466A
:106CD0001008A285294597C0FF1FE78080B0F640C5
:106CE000664423A02411D644464925618280395543
:106CF000828041110D658D4506C697C0FFFFE78074
:106D0000C00EB71700408D6623A6D70A17F5FF1FE0
:106D1000130545A71387C70A9387870A1CC15CC55B
:106D2000856689675CC958C114C518C9B7E70400EE
:106D3000B24003A3871E410102838145B307B5001A
:106D40008387070089E7172300006700E3CD8505E7
:106D5000C205C181E5B797A701009387A75D1357C7
:106D6000C5003E9703470700011106CE2304E1004A
:106D7000135785003D8B3E9703470700230601000C
:106D8000A304E100135745003D8B3D893E97AA9728
:106D90000347070083C7070028002305E100A30578
:106DA000F10097000000E78080F9F24005618280E1
:106DB000411126C2E97797F4FF1F938424AD22C4C2
:106DC0009387A7552E842381B4002E86AA8517F5B4
:106DD000FF1F1305E5AB06C62390F400A381040052
:106DE00097800100E78060EE93052400C205C18111
:106DF00017F5FF1F1305A5A997000000E780008E77
:106E0000B38784002382A7002181A382A700930572
:106E100064002244B24026859244C205C1814101EA
:106E200017230000670043C009C99307800263E687
:106E3000B700170300006700E3F7828097F7FF1F92
:106E400083C7A7A799EF411106C697200000E780E6
:106E500080B5B240854717F7FF1F2300F7A6410111
:106E60008280828063040556638205565D71A2C4E8
:106E7000A6C286C6CAC04EDE52DC56DA5AD85ED6E4
:106E800062D466D26AD0B9472A84AE8463F9B70661
:106E9000394697A501009385E53297800100E78088
:106EA00060E031ED8347E400130710036394E702C9
:106EB000854717F7FF1F2309F79C17A50100130546
:106EC000653197F7FF1F2390079C97000000E7802C
:106ED00000E771A01307000317A501001305853211
:106EE000E395E7FE97F7FF1F2380079A97F7FF1FA9
:106EF000239B079817A501001305452FF9B797F7AE
:106F0000FF1F83C7679863890722BD6AB96B938C9B
:106F1000FA55014A17FBFF1F130B8B88138CEB6587
:106F2000938AFA6605A8B307440183C6070097F75A
:106F3000FF1F83D74795B1E39307A005639BF60036
:106F4000854717F7FF1F2310F79497F7FF1F238933
:106F5000D784050A93170A01C183E3E697FCB6407C
:106F6000264496440649F259625AD25A425BB25BB1
:106F7000225C925C025D61618280054D639BA70388
:106F80009307500A639EF600894717F7FF1F231CDB
:106F9000F78E930750FA17F7FF1FA303F78055BF2B
:106FA0009307A005E387F6FA97F7FF1F239D078C49
:106FB0004DB7138717004207DA9741832380D70024
:106FC00017F6FF1F2311E68C8D47E3F4E7F817E966
:106FD000FF1F0349197D97E7FF1F83C7877C22099D
:106FE0003369F9009307F9FFC207C1839306F00DD7
:106FF000E3ECF6FA93076900C207C183E31BF7F4D9
:1070000093052900C205C18117E5FF1F13056579A6
:1070100097F0FFFFE780806C33072B018347570011
:1070200003474700A207D98F17F7FF1F231D0784C7
:107030006319F50E8149630DA90197E9FF1F83C903
:107040006976A20997E7FF1F83C7D775B3E9F900EF
:1070500017050000130585DD97F0FFFFE780200589
:1070600063878907636D3C039387EB556382F9045B
:1070700097E7FF1F83C7077305476389E70681CB3F
:107080001387A7051377F70F8D4663F2E6081307FA
:10709000F0072300E100A300F10089459DA0638271
:1070A0009905E39759FD97F0FFFFE780603311A83A
:1070B000CA8517E5FF1F1305E56E97F0FFFFE78010
:1070C0000015014597F0FFFFE78060FE59B5CA85BE
:1070D00017E5FF1F1305056D97F0FFFFE780C01E42
:1070E000CDB797F0FFFFE7806029E1BF930710F865
:1070F000130511002300F10097F0FFFFE780003532
:10710000FD450A8597000000E780C0CA5DBFCA85BB
:1071100017E5FF1F1305056997F0FFFFE780C0CF54
:107120004DB79307F00789450A852310F1009700B2
:107130000000E78020C831BDBD4763F99722414672
:1071400097A501009385450E228597800100E78071
:1071500060B5631C051417A501001305250E9700E3
:107160000000E780C0BD17E5FF1F0355656197006C
:107170000000E78080BE97E7FF1F83C7A74C17A5D5
:1071800001001305250389E717A501001305050371
:1071900097000000E780A0BA17A501001305850B32
:1071A00097000000E780A0B917C5FF1F0355852190
:1071B00097000000E78060BA17A501001305C50914
:1071C00097000000E780A0B717E5FF1F035505589B
:1071D00097000000E78060B817A501001305450877
:1071E00097000000E780A0B517D5FF1F035525EED7
:1071F00097000000E78060B617A501001305C506DB
:1072000097000000E780A0B317D5FF1F0355E5EBFB
:1072100097000000E78060B417A50100130545053D
:1072200097000000E780A0B117D5FF1F035505EABE
:1072300097000000E78060B217A5010013058503E1
:1072400097000000E780A0AF17C5FF1F0355450753
:1072500097000000E78060B017A501001305050244
:1072600097000000E780A0AD97C7FF1F83C70713F3
:10727000A20717C5FF1F034575125D8D970000001B
:10728000E780A0AD97C7FF1F83C76711A20717C587
:10729000FF1F0345D5105D8D97000000E780E0AB30
:1072A000179501001305856B0DB1414697A50100A7
:1072B000938505FD228597800100E780A09E5DE50E
:1072C000C114C20493060401C180510401498D45D3
:1072D0002545154663FC9500639F86001307E9FF6B
:1072E0004207A1674183F51763FAE70417A5010078
:1072F000130545FAD9BE83C70600138707FD137728
:10730000F70F637CE5001387F7FB1377F70F636EC6
:10731000E600938797FC13F7F70F12093369E9002A
:10732000420913590901850675B71387F7F91377D1
:10733000F70FE36DE6FA938797FAF1BF97E7FF1F20
:1073400083D7C740638A270197E7FF1F2390274110
:1073500097D0FFFFE780604A17A501001305C5F528
:1073600097000000E780A09D4A853DB7C147E3F83C
:1073700097BE414697A50100938545F522859780E4
:107380000100E7802092E31C05BC8347040113073A
:107390001003639CE700854717E7FF1F2300F740B2
:1073A00017A501001305C5F30DB61307000317A5B4
:1073B00001001305E5F5E39AE7B097E7FF1F238F78
:1073C000073C17A50100130525F301B68280411182
:1073D00026C2AE848D4522C406C62A8497C0FFFF0C
:1073E000E78000ABB717004099C803A5C70C418DD3
:1073F00023A6A70CB240224492444101828003A5F7
:10740000870C418D23A4A70CF5B7834705000347DC
:107410001500A207D98FC2076177C18713072720FC
:10742000639AE70083452500370504001703000031
:10743000670023FA828017E6FF1F1306664881471C
:10744000B2861303F00FA9483308F600034808007A
:1074500013F7F70F6307A80C630668008507E39529
:1074600017FF2947B387E6002380A70097E7FF1F90
:107470009387C7455DA8411113D7650013471700CF
:1074800006C693F63500058B954791CA0546994780
:107490006387C60009469D476383C600A14713F66C
:1074A00045003336C00093F68503050685C2A14525
:1074B000638BB604E145638AB60493058002638852
:1074C000B604930580036393B600914697E5FF1FCA
:1074D0002383F56697E5FF1F238EC56497E5FF1F9D
:1074E000A38AD564BE8517A501001305A5E897807A
:1074F0000100E780E088B240854717E7FF1FA30C33
:10750000F762410182808546D1B78946C1B78D4671
:1075100075BF17A50100130565E817830100670013
:10752000238617E7FF1F1307673ABA972380B70030
:10753000E147E302F5F493077002E30CF5FC828067
:107540002A8723800500814717E5FF1F130545376C
:107550001308F00F2946B306F50083C606006396AC
:10756000E60297E6FF1F93866636B69783C7070045
:1075700005452380F5009947636EF7029D4763FD3B
:10758000E700E147630DF700828063850601850708
:10759000E393C7FC0145C5B7238005008280B73758
:1075A000004003C7370083C7050093F70704D98F4E
:1075B0002380F50082805D7152DC56DA5ED6716AF6
:1075C00097EBFF1F938B4B688D6AA6C24EDE62D489
:1075D00086C6A2C4CAC05AD866D26AD06ECEC14985
:1075E0005E8C97E4FF1F9384242F130A0A20938A4A
:1075F0007ADC17E9FF1F03492968B3872B0183C78A
:10760000070093F7F70FC9EFB787004003C767007C
:10761000058BE310077C03C76700118BE30D077E22
:1076200083C75700918B99E36F10200317E7FF1F63
:107630000347A76485476304F7006F10400197E78D
:10764000FF1FA38AE74E97E7FF1F2387073497E7BB
:10765000FF1F2385074097E7FF1F2383074C97E70A
:10766000FF1F2380074C97E7FF1FA387073297E789
:10767000FF1FA385073E97E7FF1FA383074A97E7EE
:10768000FF1FA380074A97E7FF1FA387074A97E7D3
:10769000FF1FA384075EB787004011476F00707714
:1076A0009307190093F7F70F3D476364F70617E751
:1076B000FF1F2303F75C97E7FF1F9387E75ACA97DB
:1076C00083C707001307100293F7F703638EE71EC3
:1076D0006366F70405446385871CE38C07620947EA
:1076E000638EE71013070002E384E74EB7E700E07C
:1076F0003707400023A0E71801000100629923002A
:107700000900FD1923A0E71093F9F90FE39309EE9F
:10771000E5BD97E7FF1F2381075671BF13073002AE
:107720006388E70C63E8E71613074002638CE70AF7
:1077300013070003E39CE7FA97E7FF1F9387C751FE
:10774000CA9703C70700A1471377F70FE31BF71486
:1077500083C7640097E6FF1F2386F63C97E7FF1F69
:1077600083C7F71791C7FD5797E6FF1F238CF63A9B
:1077700097E5FF1F83C5551697E7FF1FA384B73A08
:1077800097E7FF1F83C7471513FB070893060004FD
:1077900093F70706639FD74C9307A009638DF516EF
:1077A00063EAB7129307F0056386F54A9307500919
:1077B0006384F52A014497E7FF1F83C7B73615474F
:1077C000E392E736B7E700E03707400023A0E71869
:1077D00001000100B786004023808602130680FC6A
:1077E0006F00500EFD5717E7FF1F230CF732FDBD4A
:1077F000FD5717E7FF1F2305F732CDBD17A5010081
:10780000130545CB97700100E780606F97E7FF1F76
:1078100093878744CA9703C40700014B97ECFF1F67
:10782000938C0C241374F40F17AD0100130D0DC9C4
:1078300063478B04294597700100E78040598547CD
:1078400017E7FF1FA30CF72017E7FF1F2309872067
:1078500017E7FF1F2302F72E37E700E0B7064000C7
:107860002320D71801000100378600408347A60275
:1078700093F7370F2305F6022320D71085BDB38772
:107880006C0183C507006A85050B97700100E780CE
:10789000204F79BF854717E7FF1F2301F71CB9B5B4
:1078A00017E7FF1F1307473B4A970347070097E671
:1078B000FF1FA383F60E97E6FF1F2380E60E17E750
:1078C000FF1F230BF7261DB5854717E7FF1F23056D
:1078D000F70C29BD9307400A6389F5349307200B01
:1078E0006384F5369307100AE396F5EC838724004A
:1078F0000144E3D207EC97E7FF1F83C717FE93F617
:107900003700638A061A0546638AC62209466395CC
:10791000C61A1D4755A217E5FF1F034505FCC947B9
:1079200097ECFF1F83CC7CFB97E5FF1F83C505FB0E
:1079300017E4FF1F034494FA6315F510CD476392D3
:10794000FC1093077008639CF5021307300FB717FC
:107950000E006308E4001307900DB7B7040063142A
:10796000E40817E7FF1F2325F71CBE8517A50100B4
:10797000130545B597700100E780804025BD93074A
:107980008008639DF500B307804013F4F70FB777C5
:107990004600938787CDB3D78702E1B79307900856
:1079A000639AF500B307804013F4F70F916793874C
:1079B000C766D5B79307A008639BF500B30780405F
:1079C00013F4F70FB7173D0093870790E9B79307B4
:1079D000B008639AF500B307804013F4F70F91677E
:1079E000938797D04DBF93F5F5078D47639BF500BF
:1079F000B307804013F4F70FB7975B00938707D85E
:107A000059BF8947639BF500B307804013F4F70F14
:107A1000B7770B009387071BBDBF8547639AF500B7
:107A2000B307804013F4F70FDD67938767E3A5B7CB
:107A3000D28785F9B307804093F7F70FB3D7FA02DF
:107A40000DB797000000E780409FA28566859700EC
:107A50000000E780809EB9BB9305610017E5FF1F1A
:107A60000345A5E717E4FF1F034434E79700000030
:107A7000E78040AD93057100228597000000E78004
:107A800060AC3C0017E7FF1F232EF71A8347610005
:107A90002304F10083477100A304F100894717E72D
:107AA000FF1F2301F7088357810017E7FF1F2315E6
:107AB000F7E2094409B3154793F64700B336D000FF
:107AC00093F78703850685C32146638BC706614606
:107AD000638AC706130680026388C70613068003FD
:107AE0006393C700914717E6FF1F2305D60497E667
:107AF000FF1FA381F60497E7FF1F238EE70217E716
:107B0000FF1F0347A7DD9376070497E7FF1F83C78F
:107B1000F7DC8DEE1377770C93067008630CD702B1
:107B20001377F7078D466312D70CB307F040B7956C
:107B30005B0093F7F70F938505D849A81947ADBFA8
:107B4000854755B7894745B78D4771BF930670087C
:107B50006311D7021307300FB7150E006389E702D0
:107B60001307900DB7B504006383E702130770088D
:107B700045BF9306800C6311D702B307F040B77579
:107B8000460013F7F70F938785CDB3D5E70297E744
:107B9000FF1F23AFB7F8D9BB9306900C631CD70027
:107BA000B307F04093F5F70F91679387C766B3D596
:107BB000B702F1BF9306A00C631DD700B307F040D6
:107BC000B7153D0093F7F70F93850590B3D5F502F0
:107BD0007DBF9306B00CE315D7F4B307F04093F5DF
:107BE000F70F9167938797D0D9B78946631BD70062
:107BF000B307F040B7750B0093F7F70F9385051B9C
:107C0000F1B78546631AD700B307F040DD6593F7F7
:107C1000F70F938565E35DBFD28535FBB305F04073
:107C200093F5F50FB3D5BA029DB783C72400C18B76
:107C300099C7854717E7FF1F2309F7EEA5BE97E70A
:107C4000FF1F238407EEBDB6854717E7FF1FA30478
:107C5000F7EE8DB63C0017E7FF1F2325F7FE094717
:107C6000930700032314F10097E6FF1F238CE6EA35
:107C70002DBD63940756A94763E5B74217970100E6
:107C80001307876C8A05BA959C41BA97828717E4D7
:107C9000FF1F034494C4894C6306940D63E68C066D
:107CA00085476303F4089307F00F17E7FF1F0347A7
:107CB00067E763F6E70017E7FF1F2305F7E697EC92
:107CC000FF1F83CC2CE69307000413F4FC0F63F42E
:107CD00097011304000497E7FF1F9387A7F603ADEE
:107CE000070022862685EA85B38C8C40229D9770FA
:107CF0000100E78080FD97E7FF1F238597E397E763
:107D0000FF1F23A1A7F545BC8D47630CF40A9947D3
:107D1000E31BF4F8979701009387876917E7FF1F24
:107D20002322F7F2A94751B717E7FF1F0347E7F4EC
:107D300097E7FF1F938707E14946979501009385D1
:107D4000257063068700979501009385656B3E85D6
:107D500097700100E78060F717E7FF1F2324A7EE65
:107D6000C947A1B797E6FF1F83C626F1054797E7E6
:107D7000FF1F938727DD6394E6023E85130670029A
:107D8000979501009385456997700100E780E0F3BE
:107D900017E7FF1F2328A7EA9307700239B73E852C
:107DA0001306300497950100938545619770010093
:107DB000E780A0F117E7FF1F2326A7E89307300409
:107DC000EDB597E5FF1F83C545B117950100130574
:107DD000A57097700100E780A0FA054D97EDFF1F91
:107DE00083CDADE997E5FF1F83C525AF179501004A
:107DF0001305856E6398AD0B97700100E78040F81E
:107E000097E7FF1F83C767ADB5CBE36EF4E8179420
:107E1000010013042467638CB70117940100130455
:107E2000E46663869701179401001304A467228512
:107E300097700100E780E00D1375F50F93071500AB
:107E4000860717E7FF1F230FF7CE8D4717E7FF1FA2
:107E5000A30AF7CE97E7FF1F9387C7CE0147BE86D9
:107E60001376F70F89076365A60297E7FF1F23AB19
:107E7000D7DC97E7FF1F83C7E7CC05BD97970100C5
:107E80009387475917E7FF1F232EF7DA914731BD34
:107E90003306E40003460600A3800700050723809D
:107EA000C7007DBF97700100E78080ED97E7FF1F57
:107EB00083C7A7A2E1D7E368F4DE17940100130497
:107EC0006459638CA7011794010013042459638635
:107ED0009701179401001304E4592285977001005B
:107EE000E78020031375F50F93071500860717E742
:107EF000FF1F2309F7C48D4717E7FF1FA304F7C42B
:107F000097E7FF1F938707C40147BE861376F70FD5
:107F10008907E37CA6F43306E40003460600A38049
:107F2000070005072380C700D5B797E5FF1F83C566
:107F3000C59A179501001305E55A97700100E7806F
:107F400020E497E7FF1F83C7B7BF93E7470017E712
:107F5000FF1FA307F7BE83C7240017E7FF1FA30F68
:107F6000F7BC89B8179501001305055997700100F2
:107F7000E780E0F897E7FF1F938747BC83C70700B8
:107F800017E7FF1F230AF79417E4FF1F034484B980
:107F9000333480000DB017950100130525579770F5
:107FA0000100E780C0F597E7FF1F83C777B993E724
:107FB000070117E7FF1FA305F7B883C7240017E7DA
:107FC000FF1F230DF7B66FF0EFFE179501001305A5
:107FD000255597700100E78080F203C704007D8B70
:107FE00051EFB787004003C767021377C70B1367CA
:107FF00027002383E70203C7A7021377C70B136782
:1080000027002385E70203C7E7021377C70B13672F
:1080100027002387E70203C727031377C70B1367DC
:1080200027002389E702854717E7FF1F2306F796F6
:1080300017E7FF1F2304F7A217E7FF1F2302F7AE7E
:1080400017E7FF1F230FF7AC97E7FF1FA3860794DF
:1080500097E7FF1FA38407A097E7FF1FA38207AC42
:1080600097E7FF1FA38F07AA97E7FF1FA38607AC19
:1080700097E7FF1FA38307C06FF0CFF38947631211
:10808000F70297E7FF1F83C767859146638CD70880
:1080900063E0F604638EE70C6369F70A05476380C3
:1080A000E70EFD5717E7FF1FA30EF7A6370740009F
:1080B000B7E700E023A0E71801000100B786004001
:1080C0001306F0FC2381C60223A0E7106FF00FE235
:1080D000130720086382E7086362F702130710089A
:1080E000E391E7FC378700408347670293F7C70BAC
:1080F00093E727002303F7026FF0CFEB1307300855
:108100006389E70213074008E39DE7F837870040DB
:108110008347270393F7C70B93E727002309F70249
:108120006FF04FE9378700408347270393F73707FE
:10813000F5B7378700408347E70293F7C70B93E70C
:1081400027002307F7026FF0EFE6378700408347E9
:10815000E70293F73707F5B7378700408347A70251
:1081600093F7C70B93E727002305F7026FF08FE41F
:10817000378700408347A70293F73707F5B737875C
:1081800000408347670293F73707ADB717950100A3
:108190001305053A97700100E78060D697D7FF1F57
:1081A000238C0772D5B317950100130565399770B5
:1081B0000100E780C0D497D7FF1F239F077097E780
:1081C000FF1F9387279603C40700894763F387003F
:1081D00009441374F40F6FF00FDE13070002E392EB
:1081E000E7EC631B0B0A638FF500930720026383A0
:1081F000F508179501001305253897700100E780F1
:1082000020B845B517950100130545349770010056
:10821000E780E0CE0144179D0100130D6D34A14CA1
:10822000B387840083C507006A8505049770010041
:10823000E78000B5E31694FF178501001305057864
:1082400097700100E780A0CB17D4FF1F0344046997
:1082500001E897D7FF1F23830766014B6FF0AFD567
:108260008947E310F4E4854717D7FF1F2308F76415
:108270006FF04FD417D6FF1F0346366697D5FF1F02
:1082800083C5A565179501001305052E977001009C
:10829000E78000AF6FF00FD26380F50693071002FE
:1082A000E399F5F497D5FF1F83C545631795010042
:1082B0001305852D97700100E78080AC97E7FF1FBD
:1082C00023A2979897E7FF1F93878786944383D7C6
:1082D000470017E7FF1F0347078617D6FF1F232D09
:1082E000D65E1D4497D6FF1F239AF65E97D7FF1FD1
:1082F0002387E75E6FF02FCC97D5FF1F83C5055E00
:10830000179501001305C52997700100E78040A764
:1083100097D7FF1F2384075A97D7FF1F239E075A1B
:108320006FF02FF92547638FE7C8994637870040DC
:108330006394D70223008702B7E700E0B706400046
:1083400023A0D71801000100130600FC2301C70277
:1083500023A0D7106FF08FB99306100A639FD70040
:1083600023008702B7E700E0B706400023A0D71834
:1083700001000100130680FCD1BF9306A009E38130
:10838000D7FE9306400AE38DD7FC93062002639D37
:10839000D700B7E700E0B706400023A0D7180100D8
:1083A000010023008702F9B78546E384D7FE9307CF
:1083B0000008E300FBFEB7E700E0B706400023A09B
:1083C000D71801000100130620FC23008702BDBF5F
:1083D00017D7FF1F034717756302F71E63E7E7020E
:1083E00095476300F7109947630AF704B786004082
:1083F00023800602B7E700E03707400023A0E71814
:10840000010001001306A0FC75B99307F005630A8B
:10841000F700930750096306F70093071002E3176C
:10842000F7FCB7E700E03707400023A0E71801009A
:108430000100B7860040130620FC69B117DBFF1F5F
:10844000034B4B6E930700045A8D63F46701130DC1
:10845000000497D7FF1F9387E77E83AC0700137450
:10846000FD0F2286E685268597700100E780E0856E
:10847000B3078B40669417D7FF1F2305F76A97D77A
:10848000FF1F23A1877CB7870040630C0B0223806A
:10849000A703B7E600E03706400023A0C618010096
:1084A000010003C72702134707042381E70203C71C
:1084B00027021377C70F2381E70223A0C6106FF0AE
:1084C000EFA22380070237E700E0B7064000232031
:1084D000D71801000100130620FC2381C7026FF0AA
:1084E000AFB9378700408347370097D6FF1F83C651
:1084F000F66493F70708D58FA301F700B70640008D
:10850000B7E700E023A0D718010001001306A0FC84
:1085100035BD97D7FF1F93872774CA9783C7070076
:1085200093F7F70FC1CF97D7FF1F83C70775D9E719
:1085300017D7FF1F0347175F930700026310F70861
:1085400083AD040017DDFF1F034D4D3997DCFF1F7E
:1085500083CCDC3817DBFF1F034B6B38E6876A8759
:10856000DA866E8697D5FF1F83C5453517950100BE
:108570001305850497700100E780808097D7FF1F5F
:1085800023A8B75B97D7FF1F2386A75B97D7FF1F4B
:10859000A382975B97D7FF1F238F675997D7FF1F3A
:1085A000A38D8730B7E700E03707400023A0E71826
:1085B00001000100B78600406FF04FA2B7E700E06E
:1085C0003707400023A0E71801000100B7860040EC
:1085D00015BD97D6FF1F83C6466A0547639CE60410
:1085E00029472381E70209472383E7022385E7021E
:1085F00097D7FF1FA382075497D7FF1FA38F076644
:10860000B7870040A381070017D7FF1FA3080752B1
:1086100005472383E700B640264496440649F259AD
:10862000625AD25A425BB25B225C925C025DF24DAE
:108630006161828029472381E70209472383E7029A
:108640002385E7022387E7022389E70255B717D777
:10865000FF1FA304F7266FE01FFF854717D7FF1FF3
:10866000230CF73217D7FF1F230AF73E17D7FF1F38
:108670002308F74A17D7FF1F2305F74A6FE0BFFE0D
:10868000854717D7FF1F2309F73017D7FF1F230789
:10869000F73C17D7FF1F2305F74817D7FF1F230203
:1086A000F74817D7FF1FA309072E17D7FF1FA307E8
:1086B000073A17D7FF1FA305074697D7FF1FA382C7
:1086C00007468280411106C697000000E78080FBC4
:1086D000B787004023800700130740FC2386E7008C
:1086E0001307C004A386E70017D7FF1F1307C71E91
:1086F0002398E70017D7FF1F13070722239AE700E5
:1087000017D7FF1F1307872D239CE70017D7FF1FDD
:1087100013070739239EE70029472381E70209470A
:108720002383E7022385E7022387E7022389E70201
:10873000A3810700930600F8A380D7009306900258
:108740002380D700FD562383D7002381E7009306BB
:10875000000537E700E0230BD740B7064000232091
:10876000D71003C7170013671700A380E700B240B4
:1087700097D7FF1F2394073C41018280411106C611
:1087800097000000E78000F0B787004023800700D3
:10879000130700FC2386E7003147A386E70017D7BD
:1087A000FF1F130767132398E70017D7FF1F13074F
:1087B000A716239AE70017D7FF1F13072722239C2A
:1087C000E70029472381E70209472383E70223853E
:1087D000E702A3810700930600F8A380D700930661
:1087E00090022380D700FD562383D7002381E70022
:1087F0009306000537E700E0230BD740B70640009B
:108800002320D71003C7170013671700A380E700C2
:10881000B24097D7FF1F2393073241018280F1674F
:108820009387072017D7FF1F2324F730854717D7D3
:10883000FF1F2311F730A14717D7FF1F230DF72E76
:1088400097D7FF1FA389072E97D7FF1F2386072ED1
:1088500097D7FF1F2384070697D7FF1FA38F07040F
:10886000814717D5FF1F1305A505FD5517D6FF1F17
:108870001306C6052947B306F5002380B600B306E4
:10888000F600238006008507E397E7FE97D7FF1FD2
:10889000A38B072897D7FF1FA389072897D7FF1F08
:1088A0002384072897D7FF1F238F072697D7FF1FFB
:1088B000238E072697D7FF1FA388072697D7FF1F6A
:1088C00023850726814717D6FF1F1306E637414742
:1088D000B306F600238006008507E39BE7FE82804F
:1088E00017D7FF1F0347673985476316F70017033C
:1088F00000006700E3E8170300006700E3DC4111B4
:1089000022C406C617D7FF1F0347273785472E8681
:1089100013F4F50FAA856317F70417D5FF1F130586
:10892000E50F97600100E780403A97D7FF1F238744
:108930000712B787004023848702B7E600E03706B6
:10894000400023A0C6180100010003C7A702137747
:10895000C70F2385E702B240224423A0C610014579
:108960004101828017D5FF1F130505FF97600100A5
:10897000E780A03597D7FF1F23800702B787004005
:1089800023828702B7E600E03706400023A0C6181E
:108990000100010003C767021377C70F2383E702B3
:1089A0005DBF411106C697000000E78080E7B24036
:1089B0004101170300006700E3F2411106C697F07A
:1089C000FFFFE78080BF97D7FF1F83C7F7FCA1CBCE
:1089D00097D5FF1F83C565FC89C917D5FF1F1305F0
:1089E000E5FB97E0FFFFE780204897D7FF1FA385AF
:1089F00007FA97D7FF1F2381071437E700E0B70670
:108A000040002320D718010001003786004083472B
:108A1000660293F7370F2303F6022320D710B240E4
:108A20004101828041C9D9C597D7FF1F83C707116C
:108A3000D1C3011122CC4AC84EC656C25AC006CE76
:108A400026CA52C42E89AA890144930A0004371BFE
:108A5000030063772403B3078940C207C183BE8440
:108A600063F4FA0093040004C204C180130A1BD407
:108A700097D7FF1F83C747F29DE37D1A631C0A0047
:108A8000F2406244D2444249B249224A924A024BDD
:108A90000561828097F0FFFFE78020B2D1BF338568
:108AA00089002694A685420497000000E78060E5CF
:108AB000418045B78280411106C622C429C12E8457
:108AC00095C997D7FF1F83C7670795CB97D7FF1F18
:108AD00083C787EC8DC713070004AE876374B700A4
:108AE00093070004139407014180A28597000000BA
:108AF000E78020E12285B240224441018280014486
:108B0000D5BF97D7FF1F9387E71A18429C4383D698
:108B100045000345070083C5C7000356460063961A
:108B2000A50083D5E700638DD502011106CE23860B
:108B3000A7002397D700B705CF00DC4B9385757D41
:108B400005077D162EC2230001003AC42316C1007A
:108B50002317D10099C30A858297F240056182806C
:108B60008280DC4DDC4B81CFB7E70400904503A346
:108B70008705914517D5FF1F0345051402838280A1
:108B80006D713C083EC6B707E500232291103EC830
:108B9000AA843C083285232611103ECA2324811062
:108BA000232021112E8997300000E780C0672A8496
:108BB000979501009385C5A3177501001305857B63
:108BC00097600100E780C01BA2851795010013057F
:108BD000A5B297600100E780A01A294597600100BF
:108BE000E780E01EB705CB009385757D6800971080
:108BF0000000E780406DA285680097300000E780A4
:108C0000E054014781467000CA8526859720000000
:108C1000E780C09005CD2A84979501009385459DF6
:108C2000177501001305057597600100E780401571
:108C3000A285179501001305E5AC97600100E78058
:108C40002014294597600100E78060188320C11037
:108C50000324811083244110032901105161828073
:108C600097D7FF1F9387070518429C43797122D439
:108C700006D60348070083C807012A8483D6450027
:108C8000035546006396080183D82701638DD802F7
:108C90002388070105072399D7003708CC00DC4B50
:108CA0001308787D3ACC1307F5FF42CA2308010068
:108CB000231EE100231FD10099C7080832C62EC425
:108CC00082973246A245228597000000E78080EB1C
:108CD000B2502254456182806D713C083EC0B70796
:108CE000E5003EC23C083EC4232611102324811017
:108CF00023229110231701002318010023190100DA
:108D0000231A0100231B010097A7FF1F83D7477079
:108D100099E3C167FD172316F10097A7FF1F83D7BB
:108D2000476F91EB97D7FF1F9387C7F89C439C43EE
:108D3000DC4783D7070017A4FF1F1304646D584C4A
:108D40002317F10083574400484B2318F10031E109
:108D5000979501009385C5901775010013058561EE
:108D600097600100E780C001179501001305859009
:108D700097600100E780C000294597600100E78007
:108D800000058320C1100324811083244110516108
:108D9000828097A7FF1F83C7176889EBB7E7040096
:108DA000BC5782975C4C23AA0700E1BFFD1797A62A
:108DB000FF1FA382F66603560701834704014C4751
:108DC0000A85230BF10097300000E780403597D7E4
:108DD000FF1F938727EE9C430147814688430A86FD
:108DE0006C0097100000E7806073AA8429C19795F2
:108DF00001009385E586177501001305A557976057
:108E00000100E780E0F7A685179501001305458767
:108E100097600100E780C0F6294597600100E78070
:108E200000FB584CB7E70400BC57484B9DBF97A7C1
:108E3000FF1F83C7575EF5D7B7E70400BC4F104448
:108E4000854517D5FF1F034525E782971DBF5C4E5B
:108E5000DC4BB9CFB1CD411122C417750100130508
:108E600065512E84978501009385C57D06C6976060
:108E70000100E780E0F0A285179501001305058346
:108E800097600100E780C0EF294597600100E78007
:108E900000F4B7E704002244B24003A3870517D5C6
:108EA000FF1F034565E1130640069145410102831A
:108EB0008280411122C417A4FF1F130424531C4CA9
:108EC00006C689C7DC4399C34C488297584CB7E71C
:108ED0000400BC57484B82975C4CB240224423AA02
:108EE00007004101828017A7FF1F130727528347FE
:108EF00007009306F00B850793F7F70F63E9F60079
:108F000097A6FF1F2384F65003450700828093072E
:108F100000F8FDB7835745006386071001114AC862
:108F200017A9FF1F1309C94E52C4032AC90106CE4F
:108F300022CC03274A0126CA4EC656C2F15735E352
:108F40001307D00DFD57636EC704B7E9040083A76C
:108F500009072A841305860042054181B284AE8A3E
:108F60008297232AAA000325C9015C49A9E79785AE
:108F700001009385256B177501001305A53F9760C8
:108F80000100E780E0DF178501001305657A97602F
:108F90000100E780E0DE294597600100E78020E3DB
:108FA000DD57F2406244D2444249B249224A924AD1
:108FB0003E850561828093874400B705CF00231961
:108FC000F5009385757D310597100000E780A02F8F
:108FD0000325C90183456400310597300000E7800F
:108FE000E0160325C9012686D68531059730000095
:108FF000E780E0127146A2854A8597600100E7800C
:10900000C0CC504419CA83A78905854517D5FF1FD1
:10901000034585CA8297814769B797000000E780BA
:10902000E0CBD5BFFD573E858280411126C297A473
:10903000FF1F9384E43DD84C22C437E404003C5421
:10904000484B06C68297DC4C0323C4052244B24039
:10905000924423AA070017D5FF1F0345E5C58545A0
:1090600041010283411126C297D4FF1F938484C417
:109070009C4006C622C44AC0D5C3DC43C5C35CC1FC
:109080002300B5002A84978501009385E554177560
:1090900001001305252E97600100E78060CE294569
:1090A00097600100E780A0D29C4023A4070023A280
:1090B000070097A7FF1F93876733DC4FDC4B91C7EF
:1090C000295597000000E78000DF97A7FF1F9387CF
:1090D0002734DC4FDC4B89C797000000E78020F580
:1090E00037E904008327C905894517D5FF1F0345C4
:1090F000A5BC82978327C905914517D5FF1F034556
:10910000A5BB82979C4003A3470163090300228506
:109110002244B2409244024941010283B2402244B7
:1091200092440249410182800111328506CE22CC4F
:1091300026CA2E8497300000E780E00EAA84978527
:1091400001009385A54C177501001305A5229760B2
:109150000100E780E0C203078400035664008355E2
:109160004400A68617850100130545569760010047
:10917000E78000C1294597600100E78040C597A7B7
:10918000FF1F83C70727639D9700014597000000D5
:10919000E78060D281450A8597000000E780C0EC37
:1091A000F2406244D244056182806D7123248110B3
:1091B000232611102322911093F745002E846387F4
:1091C00007143C083EC0B707E5003EC23C083EC459
:1091D000231701002318010023190100231A01009D
:1091E000231B010097A7FF1F83D7472099E3C1677F
:1091F000FD172316F10097A7FF1F83D7471F91EB99
:1092000097D7FF1F938707AB9C439C43DC4783D7CB
:10921000070017A7FF1F1307671D2317F100544FFF
:10922000835747002318F100DC4AA1E79785010026
:1092300093850542177501001305C513976001005A
:10924000E78000B4178501001305C542976001004F
:10925000E78000B3294597600100E78040B71345D8
:1092600044008320C11003248110832441105161E4
:10927000828097A7FF1F83C7D7172555D9C3FD172E
:1092800017A6FF1FA307F61603D60601834707019B
:10929000CC460A85230BF10097300000E78020E8D8
:1092A00097D7FF1F938707A19C4317A7FF1F13079B
:1092B000E713978601009386E63E88430A866C0092
:1092C00097100000E7808025AA8451D99785010076
:1092D00093850538177501001305C50997600100CE
:1092E000E78000AAA68517850100130565399760F8
:1092F0000100E780E0A8294597600100E78020ADE4
:10930000268597000000E78000BB91BF93F72500FA
:109310009DC7B7E70400BC474146814528088297AE
:10932000255597000000E78000B928089305F00F45
:1093300097000000E78040D3134524001DB793F742
:109340001500014599DF97000000E780209913453B
:10935000140001BF5C4D411106C688C317D7FF1F1B
:10936000232AF794B7E7040083A70708170500002E
:109370001305E5E38297B24097D7FF1F238EA7928C
:1093800001454101828001113335A000A307A100EE
:10939000B7E7040083A7471706CE1306F1008545FB
:1093A000130550308297F24005618280828041111E
:1093B00022C406C697D7FF1F83C78791014489EF50
:1093C00097B7FF1F83C7D7E7054499E717B4FF1F77
:1093D000034404E713441400228597000000E7804B
:1093E000C0FA178501001305A53F09E417850100A0
:1093F000130505402244B240410117630100670094
:109400002398797122D4A30F010037E40400832745
:10941000841726D24AD006D6AA842E891305503046
:109420009305F10132C6829732468347F1019315C5
:109430000601C18185CB01452EC697000000E7805B
:10944000C0F483274417B2454A862685829705458E
:1094500097000000E78060F3B25022549254025902
:1094600045618280832744174A8626858297EDB717
:1094700041119397050122C406C626C2C1872E84D6
:1094800063D40702B7E40400FC5417A5FF1F03458B
:1094900025FB829719C1BC5482972165218DB2406A
:1094A000224492444101828093F715008DC7B7E7AB
:1094B000040083A7471A17A6FF1F130666F797D560
:1094C000FF1F9385258017A5FF1F034565F782972A
:1094D00013451400E9B793F7250099CFB7E70400C7
:1094E000BC4F13060064894517A5FF1F034545F5CA
:1094F00082971345240065B793F7850085CF97C7FA
:10950000FF1F83C7A77D85E7B7E7040003A8871A75
:109510001307401F97A7FF1F83C787F281461306D3
:109520004006994517C5FF1F0355C57A0298134594
:109530008400B5B793F745000145B5D3B7E40400FF
:1095400083A7041817C5FF1F0355C5788297BC4C25
:1095500013060064914517A5FF1F034565EE82972A
:10956000134544002DBF97C7FF1F83D7A776639885
:10957000A70217C7FF1F2310B77617C7FF1F231DAA
:10958000C77417C7FF1F231AD7742E8617850100CB
:109590001305852CBE85175301006700637E178570
:1095A00001001305E52C176301006700439503577D
:1095B000450097C7FF1F83D7E771631EF704C16794
:1095C0004111F91722C417C7FF1F2325F77037E48D
:1095D000040097C7FF1F23A1077097C7FF1FA38928
:1095E000076E97C7FF1F238B076E7C4C06C6894505
:1095F00017A5FF1F0345C5E482977C4C914517A52D
:10960000FF1F0345E5E382972244B240410117035F
:109610000000670003DA178501001305652517634D
:1096200001006700C38D7D15954763E2A71C17876E
:109630000100130767190A053A951C41011122CC54
:1096400006CEBA972E848287178501001305C5229E
:1096500097600100E780A08AA1A203C7250099476F
:109660006311F7022E8597000000E78080F48345A0
:109670006400178501001305252197500100E7803C
:10968000207097B7FF1F238D07BA178501001305B8
:1096900065217DBF03C7250095476319F702C167A0
:1096A00017C7FF1F03570763F91703D5A500630901
:1096B000F702B7E7040083A7C71782971785010051
:1096C0001305451F97600100E7806083854717B742
:1096D000FF1F2307F7B617850100130525208DBF4F
:1096E00097C7FF1F2398A75E83D7E50097C6FF1F84
:1096F0002393F65E83D7050197C6FF1F239EF65C72
:1097000083D7250197C6FF1F2399F65C97C7FF1FD4
:10971000A380075C631BE502B7E70400BC4F096642
:1097200013060690A14517A5FF1F034565D1829733
:109730000356E4008355A400178501001305C518DE
:1097400097500100E780C06351B79307700F23164D
:10975000F100B7E7040083A7870D17A6FF1F034694
:1097600026CE6C0082974DF9854717C7FF1FA301CE
:10977000F7565DB71785010013050517D1BD83C5E1
:10978000250091476392F5021785010013054517DF
:1097900097500100E780A07697000000E78060C145
:1097A000F24062440561828099476392F502228506
:1097B00097000000E780E0DF834564001785010023
:1097C0001305850C97500100E780805BD1BF95475A
:1097D000639AF50083471400E1F317850100130530
:1097E0006514BDB51785010013054514E1BF8280DE
:1097F0000111B7F5070030008146E105194506CE95
:109800009790FF1FE780E0FD8347C1000347D10029
:10981000B7562D47A207D98F938676D517A7FF1F76
:10982000130747C314C3B736302D9386360354C38A
:109830009566938676742314D7009306D002230589
:10984000D70013D6C700978601009386A6FD3696EB
:109850000345060013D687003D8A369683450600E9
:1098600013D647003D8ABD8B3696B69783C6070050
:109870000346060097A7FF1F938747BFA305A700CE
:109880002306B700A306C7002307D700A3070700D6
:10989000A386A7002387B700A387C7002388D70024
:1098A000F24005618280411106C697000000E78002
:1098B00060F4B7E7040083A7871417A6FF1F1306F9
:1098C00066B9D54501458297B240694697A5FF1F05
:1098D0009385C5B913057030410117030000670077
:1098E00083B261712324811A37E4040083270408BA
:1098F0002326111A2322911A2320211B232E3119EA
:1099000017050000130505B7829717A9FF1F130954
:1099100029B3994785442300A900231CF1009785AA
:109920000100938525EF9307400617750100130585
:1099300065A4231CF1082308910097C9FF1F938990
:1099400029E497500100E780A04383D509001785DB
:109950000100130525EB97500100E780604229457F
:1099600097500100E780A04603D509008969970058
:109970000000E78020E88327441710088545130579
:10998000503082978327441717A6FF1F130606AE91
:10999000E9451305703082978327441717A6FF1FE8
:1099A000130646AAB54513056030829783274417EE
:1099B00030088945130510318297832744173009F1
:1099C0008945130520318297832744159385099093
:1099D0000D458297832744159385099011458297F9
:1099E000A30591002306910002CD23080100230C5A
:1099F0000100832784163009914513057040829732
:109A0000832784161306B10085451305004082970D
:109A1000832784167000854513051040829783279D
:109A200084163008854513052040829783278416C5
:109A300010088545130550408297832704157D55EE
:109A40008297832744137D5582977D5597A0FFFF0A
:109A5000E78000C28327440C829797A0FFFFE7802E
:109A6000609D8327841417A6FF1F1306A69ED54565
:109A70000145829789471306700F814528092306FF
:109A8000F1009780FFFFE78080688D47130600088C
:109A900081452808230CF1089780FFFFE7802067A5
:109AA0009147230CF100976701009387277E984325
:109AB00083C747003AC8230AF10097D0FFFFE78029
:109AC00080A370008545054597A0FFFFE78060C132
:109AD00030099305700F094597A0FFFFE78060C02C
:109AE0003008930500080D4597A0FFFFE78060BF91
:109AF00010089545114597A0FFFFE78080BEC1671C
:109B000017C7FF1F1307071DF9171CC323220700E0
:109B100017A5FF1F1305859297A0FFFFE78040BBA5
:109B20008327C41D17C5FF1F1305451982973C489D
:109B300003450900854582978320C11A0324811AB1
:109B40008324411A0329011A8329C1195D61828086
:109B5000C16717C8FF1F0358E817F9176301F80812
:109B60003DCDB5CD011126CAB7E4040083A7841208
:109B700022CC2E862315B10006CE2A8401478146C9
:109B8000ED45428582972AC611ED17850100130520
:109B9000A5CA97500100E7808036F2406244D24463
:109BA00005618280FC440356A100A28582972C00A7
:109BB00017C5FF1F0355051297A0FFFFE78000BEE2
:109BC00069DD17850100130565C897500100E7801E
:109BD000003383A7C412ED45280082977DBF8280A1
:109BE0000DC5854717A7FF1FA303F78697A7FF1F7C
:109BF00023800786354697A5FF1F9385A584130507
:109C00006030170300006700038097A7FF1FA38041
:109C10000784E9BF97C7FF1F83C7470CA9EFC16738
:109C200017C7FF1F0357070BF9176306F704411106
:109C3000854722C417C7FF1F2302F70A37E4040031
:109C40007C4C06C6A1451795FF1F0345657F82978B
:109C50000323841A2244B2409797FF1F83C7477E8D
:109C600017C5FF1F035505071307401F81463146DF
:109C700099454101028382806D712324811023263E
:109C8000111023229110328401CD8947630AF50215
:109C90008320C110032481108324411051618280EC
:109CA00017850100130545C9AE8497500100E78070
:109CB0000025A285268597C0FFFFE780E0A1C9BFE8
:109CC000B7E70400FC4728008297178501001305B9
:109CD00065C797500100E78080228347810039C41F
:109CE0001307000B6380E7021387A7051377F70FAD
:109CF0008D4663EDE602A285280097C0FFFFE7804E
:109D0000A01179B78547E3F587F88345910017756A
:109D1000010013052599B335B00097A7FF1F2385D0
:109D2000B73A97500100E780A0059DB7034791001F
:109D3000A207D98F35671307D7556385E70863688E
:109D4000F7022D671307B7556387E70631671307D7
:109D5000C755638AE70429671307A7556394E70289
:109D6000A285280097C0FFFFE780604915B73967D3
:109D70009306E7656381D70863E9F6001307E755A3
:109D80006384E706A28528003DB73D679306F75533
:109D9000638AD7061307F766E396E7FE97C0FFFFCF
:109DA000E7800064F5B50146A285280097C0FFFF53
:109DB000E7802032F1BDA285280097C0FFFFE78031
:109DC0004042F9B58947E3F587EC97000000E7804A
:109DD000A0E49305E4FFC205C1811305A10097909B
:109DE000FFFFE780403E6DB5A285280097C0FFFFCA
:109DF000E780E04171BDA285280097C0FFFFE780A2
:109E0000A04C79B597C0FFFFE780405751B5C167B7
:109E100017C5FF1F035505ECF9176307F500B7E7F2
:109E2000040003A3C71702838280854717C7FF1F5B
:109E30002300F7EA014517F3FFFF67000355178377
:109E4000FFFFE70223282A8408452E89B28919C911
:109E500000C1971500009385A58661059730010024
:109E6000E780200581447D5A97100000E780E039A3
:109E700063C7A404814497100000E780003A63C8D8
:109E8000A40497C7FF1F9387A7E59C43DC47B3074C
:109E9000F94091872302F400638309048327C900F2
:109EA000B307F4409587A302F4001C4C89C79C4774
:109EB00099C3228582971783FFFF6700E3235C44E1
:109EC000139714008504BA972390470171BF1C486B
:109ED000139714008504BA972390070069BF83275E
:109EE00089000547B307F4409587A302F400835720
:109EF0000400638EE7028DC309476384E7040D47BE
:109F0000E395E7FA97870100938787F61CCC97873C
:109F100001009387E7F611A8978701009387C7BCD4
:109F20001CCC97870100938727BD5CC8BDBF97876E
:109F30000100938767A81CCC978701009387C7A867
:109F4000EDB797870100938767F71CCC97870100CF
:109F50009387C7F7D9BF95E51783FFFFE70223185B
:109F6000004618448347940075839D8B6317F70060
:109F700097100000E78060B448C41783FFFF6700B4
:109F8000431882801783FFFFE702C313138935004C
:109F9000C16442094111AA890144F114135909010C
:109FA000054A2EC697100000E7802026B245634878
:109FB000A400014541011783FFFF6700E31383A756
:109FC000090013171400BA9783D707006388B700F6
:109FD0006394970063742A010504E1B70545D9BF6E
:109FE0001783FFFFE702230DAA892E89328BB684DF
:109FF0003A8ABE8A97A00000E780C0FE71C9268514
:10A0000097200000E780C00C8D4763E7A7007D55CF
:10A010001783FFFF6700A30D83DB44009710000048
:10A02000E780A0242A8497100000E780402593074A
:10A03000740031443305850263CDA70297100000F8
:10A04000E780A02297100000E78020222A84971042
:10A050000000E780C0229307740031443305850275
:10A0600063C3A70497100000E780202093074500F2
:10A0700029A897100000E780802033058502130788
:10A08000F0179307C017E35FA7FA2D55E3C277F9DE
:10A0900063040B02D6865286A6854A859720010066
:10A0A000E780C0BDB5B797100000E780401D3305BD
:10A0B00085029307C5FFD1BF832749001385C900D7
:10A0C00083D5270097000000E78000EC61F581B799
:10A0D00069553DBF97C7FF1F2396A7C097C7FF1FAE
:10A0E000938707C0904381470C463307F50042072A
:10A0F00041836393B70082805446139847008507D5
:10A10000C2962390E600D5B797C7FF1F938747BD38
:10A110009C4303C58700828017C5FF1F035585BC7C
:10A1200082801783FFFFE70283FBC1671387D7FF96
:10A13000630BE502636AA700F1176300F5020145AE
:10A140001783FFFF6700E3FB1387E7FF6302E50266
:10A15000FD171D8D13351500E5B797500000E780FA
:10A16000602A7D15C5BF97500000E780E0FED5BF8F
:10A1700097500000E78000FDEDB71783FFFFE7026F
:10A1800003F64111AA8401442EC697100000E7800F
:10A19000C008B2456348A400014541011783FFFF91
:10A1A000670023F69C48131514003E95835705005D
:10A1B000E385B7FE0504C9BF03485500814693F700
:10A1C000F60F63E5070181473E85828058459397E6
:10A1D0005600BA9703D727006316B70003D70700C6
:10A1E000E304C7FE8506E1BF834645000147937738
:10A1F000F70F63E4D700814711A81C4513165700D9
:10A200000507B29703D60700E313B6FE3E858280AA
:10A210001783FFFFE70203EB93170501C18797CA76
:10A22000FF1F938AEAAB635BF00883A70A00C0476D
:10A230009C4703570400198D420541816368F5006E
:10A24000014422851783FFFF670003EB12052A9460
:10A25000CDBFDC4713944900014A3E948347440034
:10A260006341FA02014A834754006349FA028509AF
:10A27000C20993D9090183A70A009847E3EBE9FCD7
:10A28000C1B71C4413195A00A6853E994A85970008
:10A290000000E780C0EE05E1050AC9B75C44131968
:10A2A0005A00A6853E994A8597000000E78020ED78
:10A2B00019E1050A4DBFE30C09FA61B7AA84814987
:10A2C0005DBF1783FFFFE70283E11C452A8481E716
:10A2D0009307C5001CC51C44231204001CC093072F
:10A2E000F00F63EDB70093F5F50F2285972000007E
:10A2F000E780C0E51783FFFF6700A3E093940501A3
:10A30000C167C18063F9F500A6852285972000000A
:10A31000E780E0E8C5B7C18193F5F50F2285972066
:10A320000000E780A0E2A685228597200000E78054
:10A33000E0E3C9B797C7FF1F9387879A8843828056
:10A340001C4599C797C7FF1F23ACA798014582807A
:10A350007D55828097C7FF1F9387879898438347CF
:10A360004500484792073E9582801783FFFFE7022A
:10A3700003D7617100451C183EC6B70780013EC86F
:10A380001C183ECA8357440002CE02D002CC231EC2
:10A39000F100834784002A8902D22301F1023C089C
:10A3A0003ED402D697000000E78000FB83570500EB
:10A3B0002316F10297500000E78000C82307A1028E
:10A3C0005C4003556400F18313F717008347F102E3
:10A3D00052055181F99BD98FA307F1029710010013
:10A3E000E780207939CDAA840355050097A00000A5
:10A3F000E78020C083D704002AD26800231CF10024
:10A4000083D72400231DF1001C4803D647008C434A
:10A4100097200000E780A0D08347B400CA86177653
:10A4200001001306E6528117A305F4006C004810E2
:10A4300097200100E78080845D611783FFFF67003C
:10A4400043CC2155D5BF1C45B1CF03C5A7008946D4
:10A4500013576500630BD7028D46630ED7028546FE
:10A460006300D702130740063305E50203C7B700B0
:10A47000418B15CB83C7B700BD8B3355F540828028
:10A480001375F5031307803EC5B709671375F50308
:10A4900013070771D1BF372709001375F503130799
:10A4A000077CD9B7014582801783FFFFE70223C3EA
:10A4B00003A98500630C09048347B900AE8493F7B0
:10A4C000070E85C303459900930520030D810505FB
:10A4D000B305B5028844610597300100E78080AD7F
:10A4E00035A02E8597000000E78020F62A8419CD3C
:10A4F00097000000E780605C8325C900B307B54082
:10A5000063FA87002E94B305A440E9F51783FFFF93
:10A51000670023BF85457DBF1783FFFFE70223BC8C
:10A520002A8403D50500011132C636C43AC22EC0B2
:10A5300002CA02CC02CE97A00000E78080AB824521
:10A540002ACA22852ECC97000000E780E0E003575E
:10A550000500231EE10097500000E780E0ADA24611
:10A5600032469247230FA10036874C08B2862285D7
:10A57000014697000000E780E0A605611783FFFF12
:10A58000670023B81783FFFFE70263B561711C18EA
:10A590003EC6B70780013EC81C183ECA3C080045AD
:10A5A0003ED4AA8402CC02CE02D002D202D69700B8
:10A5B0000000E78060DA8357050035592316F10261
:10A5C00097500000E78040A72307A10209C48357E2
:10A5D000440081EB21594A855D611783FFFF6700C5
:10A5E00043B2035564005205518197100100E78082
:10A5F00040582A8965D18347B40093F7070E99C75D
:10A600001305840197300100E780009D83574400C3
:10A61000231EF100834784002301F1025C400355AF
:10A620000900D98313F7070883471102231CA100EF
:10A6300093F7F707D98FA300F10283572900231D51
:10A64000F1005C40F18313F717008347F102F99B97
:10A65000D98FA307F10297A00000E78080992AD242
:10A6600035D9834794006800139757008347B40097
:10A67000FD8BD98FA305F4001C4803D647008C43FB
:10A6800097200000E780A0A9A6871777010013078D
:10A69000272C740005464C10268597000000E780A3
:10A6A00060942A890DD98347B400A685FD8BA30544
:10A6B000F40097000000E78060DF31BF1783FFFFE1
:10A6C000E702E3A1832485FE2A84411126859700B1
:10A6D0000000E78080D7834734FF93F7070E8DCBC8
:10A6E0002AC6268597000000E78060C809CD834709
:10A6F00034FFB245FD8BA309F4FE91C52285973046
:10A700000100E780208B41011783FFFF6700639FF3
:10A710007DD98327C4FF2685829775F5834734FF4B
:10A7200093F7070E91C7228597300100E780C08A12
:10A73000032584FE97000000E78000E5E9B7178352
:10A74000FFFFE702C3969C4141112A8903C7070016
:10A7500089472E84935667006380F6040D4663880C
:10A76000C6049307F0076304F7022E8597200000C4
:10A77000E78060ABAA848149C16B130C490097B78D
:10A78000FF1F9387E7559C43984763E4E904410121
:10A790001783FFFF6700639503D745008547E3F8FC
:10A7A000E7FE2E8597200000E78040ADE1B703D794
:10A7B0004500E3FEE7FC2E8597200000E780A0A679
:10A7C000AA84228597200000E78000A8C204C98CD3
:10A7D0005DB7DC470355A900139A49003E9A9317C9
:10A7E0000501C187635DF00083570A006397A702E4
:10A7F00063E774038327CA00034D5A002DA0A167A5
:10A800002167A98F1307F7EFE374F7FE6397090039
:10A8100097000000E780209161FD85098DB78327AF
:10A820008A00034D4A00835DA90003576900216A2D
:10A83000138BC7003AC6814A33CA4D01631E5D01BE
:10A8400097B7FF1F9387474A9C43E1DBA286628646
:10A85000814526858297D1B7A1679387F7EF930C3F
:10A860004BFF63F24703B2455A8597F0FFFFE7803D
:10A87000A0710DC103278B00104709CE10436382DE
:10A88000C4023107D5BFEE85668597000000E780DA
:10A89000008F71F993861A0093FAF60F130B0B02CF
:10A8A00071BF835644005C43E3E9F6F622853AC65D
:10A8B00097200000E7802081A1679387D7042A8A28
:10A8C000035D4400324763E897008347D90093E76C
:10A8D00007F8A306F9001C4766852286E285829761
:10A8E000C1670844FD17337AFA00529508C0231255
:10A8F000A40125B797B7FF1F9387873E98438147E9
:10A9000015C31447814763FFD500939745004C4713
:10A91000BE9519C903C7550081476375E600DC453C
:10A920001606B2973E85828003C745008147E37BC8
:10A93000E6FE16069C45F5B71773FFFFE70283781E
:10A94000AA892E8A814497BAFF1F938A6A3983A7FE
:10A950000A00984763E6E4001773FFFF6700C379B6
:10A96000DC471394440001493E9413BB1400834711
:10A970004400634BF900014913BB140083475400A2
:10A98000634FF9008504E1B70844931759005287D3
:10A99000DA860146A2853E9582990509C9BF4844D9
:10A9A000931759005287DA860546A2853E9582990B
:10A9B0000509E9B71773FFFFE7026372814517F5D1
:10A9C000FFFF1305054897B7FF1F239D073097002A
:10A9D0000000E780A0F61773FFFF6700837297B748
:10A9E000FF1F9387E72F9C4395C31773FFFFE70271
:10A9F000036F814517F5FFFF1305A544970000007D
:10AA0000E780C0F31773FFFF6700A36F828017739F
:10AA1000FFFFE702236B37E4040083278412411110
:10AA20002315E100AE893289368A3A86814601478C
:10AA3000ED45AA8482972AC621C90356A100D28572
:10AA400097400100E78060288327C413CE852685C0
:10AA50008297058905C98327440D231421010146E6
:10AA60002C00268582972A8401C9B7E7040083A7B2
:10AA7000C712ED4528008297228541011773FFFF19
:10AA8000670083674944D5B76554FDB75C41FD173E
:10AA90005CC182801773FFFFE7026364B7E70400BD
:10AAA000FC5F829795473305F50281450D81177349
:10AAB000FFFF670003651773FFFFE7024362B7E715
:10AAC0000400FC5F829795473305F5020D811773EB
:10AAD000FFFF670003631773FFFFE7024360B7E7F9
:10AAE000040083A7870B0355050082971773FFFFA8
:10AAF000670023611773FFFFE702635E03550500DC
:10AB00003287AE861796FF1F0356E69C97B5FF1F48
:10AB10009385C51D97000000E780A0EF1773FFFF26
:10AB20006700235E1773FFFFE702635BB7E704006C
:10AB300083A7C71782971773FFFF6700835C17739C
:10AB4000FFFFE702C359B7E7040083A7871397B550
:10AB5000FF1F9385A519829701451773FFFF6700B3
:10AB6000435A1773FFFFE7028357B7E7040083A731
:10AB7000C71F81451795FF1F0355E59182971773EE
:10AB8000FFFF670003581773FFFFE7024355B7E75E
:10AB9000040083A7871397B5FF1F93852516829717
:10ABA00001451773FFFF6700C3551773FFFFE702E7
:10ABB0000353B7E7040083A7C71F81451795FF1FFD
:10ABC0000355659382971773FFFF670083531773CD
:10ABD000FFFFE702C3502E8597800000E78080B317
:10ABE00097800000E78080F01773FFFF67006351D4
:10ABF0001773FFFFE702A34E97800000E78080FAFB
:10AC00001773FFFF6700E34F5C49E1175CC95CC540
:10AC100083572501A1072319F50083570501A107D3
:10AC20002318F5008280F1473305F50297B7FF1F1F
:10AC30009387C70E9C433E9582808D476315F60827
:10AC400003D74600854763F0E7081773FFFFE70265
:10AC50000349368536842E8997100000E780A05C72
:10AC600029C98357440093140501C18063E3970405
:10AC7000228597100000E780005BFD1423129400EA
:10AC80009307A0026300F5029307B0026307F50281
:10AC900093079002631FF500228597000100E7806B
:10ACA000608901A80146CA85228597A00000E78037
:10ACB00000B41773FFFF6700C3442285971000009C
:10ACC000E7806007FDB7828097B6FF1F9386460531
:10ACD0009C42014599CF9843D44217B6FF1F2321C8
:10ACE000E6046396D70097B6FF1F23ADE6021385EF
:10ACF000C7FE82801773FFFFE702633E97000000E4
:10AD0000E780A04B71443305850291459790000080
:10AD1000E780C0EC11E565551773FFFF6700633EE0
:10AD200097B7FF1F23AAA7FE97000000E780E0481F
:10AD300033058502914597900000E78020EA61DDA8
:10AD400097B7FF1F23ACA7FC97000000E780E04601
:10AD500097B7FF1F239CA7FA97000000E780E04504
:10AD600097B7FF1F2395A7FA97770100938787C3AB
:10AD700017B7FF1F2320F7FA97070000938707E90B
:10AD800017B7FF1F2326F7F8014579B71773FFFFA1
:10AD9000E702E334AA8517B5FF1F130525F79710BF
:10ADA0000000E780605F1773FFFF6700833517734C
:10ADB000FFFFE702C33297000000E78060FD9710B5
:10ADC0000000E780E05E97B7FF1F938767F59C431D
:10ADD00091CF1387C7FE19CB83D5C7FF17B5FF1FC8
:10ADE000130585F497200100E780C01C1773FFFF4F
:10ADF000670023311773FFFFE702632E97000000FF
:10AE0000E780C0EC09CD834785002A8493F70704C7
:10AE100099EB0355E50097000000E78080F9177370
:10AE2000FFFF6700032E8347C5009304450117B950
:10AE3000FF1F1309E9EE85E3832709005CC997B773
:10AE4000FF1F23AF97EC83274900F1FB97B7FF1F44
:10AE500023AA97ECE9B7FD172306F5006105978053
:10AE60000000E78060DA8307840063CB0704834730
:10AE7000840093E707F82304F400B7E704009C5F1D
:10AE800082974205A94741813375F50283478400C3
:10AE900093F707FCC98F2304F4008347D4003E9541
:10AEA0001C402318A40089CF984319CB8347C400C2
:10AEB0005040814585073305F502420541810297DF
:10AEC000832709005CC897B7FF1F23AB97E483274C
:10AED000490089E797B7FF1F23A697E48347C4007B
:10AEE0009DDF8355040117B5FF1F1305E5E3972088
:10AEF0000100E780200C25B71773FFFFE702231E30
:10AF000097B7FF1F938787079C4701448583858BED
:10AF100085E3AE84B2853A8697100000E780204F23
:10AF20002A8419C597100000E7806045829408CCF8
:10AF300022851773FFFF6700C31C1773FFFFE7022B
:10AF4000631841112E8932C6AA8997000000E78054
:10AF5000C031324713060502CA8697050000938563
:10AF6000C5CC17B5FF1F130565DA97000000E78011
:10AF7000E0F82A8425C99304C50097000000E78003
:10AF8000E0411946AA85268597100000E780201920
:10AF90008545268597100000E7800015177501008C
:10AFA0001305059E4E9583450500268597100000E4
:10AFB000E780C0195C4831468145A1075CC85CC484
:10AFC00083572401E1172319F40083570401E11783
:10AFD0002318F4001C4C3E859770FFFFE780201378
:10AFE000A3042501228541011773FFFF6700C310E9
:10AFF0001773FFFFE702A30E4111AA842EC632C4C5
:10B0000097100000E780003A004DB2452246834782
:10B0100084000CC050C093F7F70393E707042304A0
:10B02000F40023180400268597100000E7802035DF
:10B0300083479400A9462317A40013D737000507B8
:10B040003307D7029D8B85072306F400A306E4008F
:10B0500083C70401D8488507230FF7FE17B7FF1FE2
:10B06000130707CC5843232A04009307440129E31C
:10B0700017B7FF1F2328F7CA17B7FF1F2322F7CAE6
:10B0800017B4FF1F130444CA228597200100E780EC
:10B09000A0E41C44858B5D8D19E5814522859720B0
:10B0A0000100E78020F141011773FFFF670063058E
:10B0B0001CC317B7FF1F2327F7C6D9B71773FFFFA6
:10B0C000E702E30197050000938565B70145970006
:10B0D0000000E78000B001451773FFFF67006302BF
:10B0E0001773FFFFE702A3FF97000000E78080B01F
:10B0F0001773FFFF6700E3008347C500A5E31773DD
:10B10000FFFFE702C3FD2A840355E5009700000016
:10B11000E78000C821C18347840093F7F7FB23042D
:10B12000F4001C4091C7DC4381C74C400145829725
:10B1300097000000E78080B917B5FF1F1305C5BE53
:10B1400097200100E78040E90355E40097000000E4
:10B15000E78020C61773FFFF6700A3FA828017738A
:10B16000FFFFE702C3F797B7FF1F938767BB9705FA
:10B170000000938565C817B5FF1F1305E5BA23A026
:10B18000070023A2070097200100E78080D21773F1
:10B19000FFFF670003F71C4D91CFDC4381CF17738E
:10B1A000FFFFE702C3F38345070082971773FFFF92
:10B1B000670023F5828097B7FF1F938727B99C43C9
:10B1C00003C50700828097B7FF1F938727B89C436A
:10B1D00003C51700828097B7FF1F938727B79C434B
:10B1E00003C52700828097B7FF1F938727B69C432C
:10B1F00003C54700828097B7FF1F938727B59C43FD
:10B2000003C53700828097B7FF1F938727B49C43FD
:10B2100003C55700828097B7FF1F938727B39C43CE
:10B2200003C56700828097B7FF1F938727B29C43AF
:10B2300003C57700828097B7FF1F938727B19C4390
:10B2400003C58700828097B7FF1F938727B09C4371
:10B2500003C59700828097B7FF1F938727AF9C4352
:10B2600003C5A700828097B7FF1F938727AE9C4333
:10B2700003C5B70011E11D45828097B7FF1F938773
:10B28000E7AC9C4303C5C700828097B7FF1F938735
:10B29000E7AB9C4303C5D700828097B7FF1F938716
:10B2A000E7AA9C4303C5E700828097B7FF1F9387F7
:10B2B000E7A99C4303D50701828097B7FF1F9387B7
:10B2C000E7A89C4303C52701828097B7FF1F938798
:10B2D000E7A79C4303D54701828097B7FF1F938759
:10B2E000E7A69C4303D56701828097B7FF1F93872A
:10B2F000E7A59C4303D58701828097B7FF1F9387FB
:10B30000E7A49C4303C5A701828097B7FF1F9387DB
:10B31000E7A39C4303C5B701828097B7FF1F9387BC
:10B32000E7A29C4303C5C701828097B7FF1F93879D
:10B33000E7A19C4303C5D701828097B7FF1F93877E
:10B34000E7A09C438857828097B7FF1F938707A089
:10B350009C4303D5C702828097B7FF1F9387079F3F
:10B360009C4303D5E70219E11305800C828097B74F
:10B37000FF1F9387A79D9C4303C50703828097B750
:10B38000FF1F9387A79C9C43C85B828097B7FF1FD2
:10B390009387479B8843828097B7FF1F9387C79AFD
:10B3A0008843828019E17D558280F5DE984265DF11
:10B3B000FDD917B7FF1F130767BC1847AA87715538
:10B3C000058B631D072403C507001547E37DA7FC14
:10B3D00003C737001305F0057D171377F70FE364F4
:10B3E000E5FC03C35700E30003FC83C86700E38C5C
:10B3F00008FA03C77700494579171377F70FE36415
:10B40000E5FA03C7A70011481305F7FF1375F50FF9
:10B41000E36BA8F803CE97000D481305FEFF1375E4
:10B42000F50FE362A8F803C8B700630908006518C0
:10B430001378F80F1305600DE36705F703C5C70020
:10B44000794879151375F50FE36FA8F403C8D70091
:10B450000D457D181378F80FE36705F503D807014C
:10B46000930E40175118420813580801E3ED0EF3EC
:10B4700003C8E7007D181378F80FE36605F303C8E7
:10B4800027017D181378F80FE36F05F103C88700D3
:10B49000C54E75181378F80FE3E70EF103D867016E
:10B4A000856E938EBEE06D18420813580801E3ECD8
:10B4B0000EEF03D847016D18420813580801E3E462
:10B4C0000EEF03D887017918420813580801E36C7E
:10B4D00005ED03C8A7017D181378F80FE36505EDA6
:10B4E00003C5B7011D487D151375F50FE36DA8EA77
:10B4F00003C5D701714879151375F50FE365A8EAFF
:10B5000003D5E7011308E00F7D1542054181E36C87
:10B51000A8E803C50702494879151375F50FE364D8
:10B52000A8E8C85301C937C834005915130858BFD3
:10B53000E36BA8E603A8870237C53400130555BF9F
:10B540005918E36205E717A5FF1F232FC57E03C621
:10B55000050117A5FF1F232BF57E0545E375C5E4FF
:10B5600003D82501D04933760603E31E06E203C65D
:10B570001501E30A06E217A6FF1F2325B67C83C543
:10B58000270001466387A50003C61700F14533066F
:10B59000B60283C707039305C00272971A07130701
:10B5A000C70516031A9796084697B387B702415501
:10B5B0003E973297420741836362E8061773FFFFA5
:10B5C000E702E3B1368597800000E780406C970082
:10B5D0000100E780C04B2A8497A00000E780205E2E
:10B5E0002A9497F00000E780002A2A9497900000A0
:10B5F000E78040852A9497F0FFFFE780E06F2A9468
:10B6000097400000E78000972A9497700000E78039
:10B6100040A022951773FFFF6700A3AE82801773C7
:10B62000FFFFE702C3AB4111A307A10097A00000F1
:10B63000E78040C99305F100170500001305E5B543
:10B6400097F0FFFFE780802F014541011773FFFF4F
:10B65000670023AB1773FFFFE702E3A517B4FF1FD3
:10B660001304C4910328840079599368180097B48F
:10B67000FF1F23A914911378180063100802BA84DD
:10B68000BE89368B328A2E89AA8A97F0FFFFE7801F
:10B69000E0A77D15269519E531594A851773FFFFF7
:10B6A0006700E3A497F0FFFFE78040A67D1526958D
:10B6B000A167E353F5FE97B7FF1F938727C398430E
:10B6C0003E8C814B01CB014597F00000E780C047DD
:10B6D000933B15004A85DA865686D28597900000FE
:10B6E000E78060512A8911CD1C44F99B17B7FF1FD1
:10B6F000232AF78883270C00CDD3E3800BFA8297A7
:10B7000069BF268597B7FF1F23AC078697F0FFFF19
:10B71000E780809C4146CE8517B5FF1F1305858FB6
:10B7200097300100E780605A97D00000E780E09CE6
:10B730000325040B97D00000E780A0A0054597D013
:10B740000000E780A0A7054597000000E78060EDB6
:10B75000A9B797B7FF1F938767829C47858BEDC773
:10B760001773FFFFE702A39717B5FF1F1305C588DF
:10B7700097B7FF1F23A4078097B7FF1F23A2078057
:10B7800097B7FF1F23A0078097200100E780C084A0
:10B7900097500000E78080F997100100E780405043
:10B7A00097100100E780405697A7FF1F9387877B7C
:10B7B0009C4391C7054597800000E780E02397A749
:10B7C000FF1F9387E7639C4399C741657D15977079
:10B7D0000000E780E0A597F00000E780804197D067
:10B7E0000000E780209397B7FF1F9387278E9C4325
:10B7F000139717016356070097F00000E780A0B089
:10B8000097B7FF1F23A8078097B7FF1F23A60780BE
:10B8100097B7FF1F23A4078097B7FF1F23A20780B6
:10B8200097000000E780008C97000000E780A0757B
:10B8300097F0FFFFE780401897F00000E780E0D91D
:10B840001773FFFF6700E38B828097A7FF1F938723
:10B85000E7728843828097A7FF1F93872772C843A8
:10B860008280B7E7B0009387075063E1A70297A7EC
:10B87000FF1F9387A770D843FD576367E50097A71D
:10B88000FF1F23AFA76E81473E858280B957EDBF6A
:10B890001773FFFFE702A38497800000E7806075BD
:10B8A00097800000E780C0771773FFFF670063850C
:10B8B0001773FFFFE70203812A8493041402011126
:10B8C0002E85B289A685214636C63A899730010071
:10B8D000E780403D0DE9B24638082686CE8513053F
:10B8E000940497500000E780604121462C084A8567
:10B8F00097300100E780003B1335150005611763A1
:10B90000FFFF6700637F0145D5BF1763FFFFE702B5
:10B91000037D9305450617A5FF1F13056543971083
:10B920000100E78020691763FFFF6700837D1763CD
:10B93000FFFFE702C37A41112EC697F0FFFFE780B1
:10B94000C017B24588C141011763FFFF6700637BE1
:10B950001763FFFFE7020377AA842E849780000015
:10B96000E780006CAA898545228597000000E78062
:10B97000E07D83C7E4011389940899E313890403E4
:10B98000CE85228597000000E780407C2146930504
:10B990001902228597000000E780607897A7FF1FB3
:10B9A0009387C75D8C43228597100000E780C08293
:10B9B000214693858402228597000000E780207647
:10B9C0001763FFFF670043731763FFFFE702A36E70
:10B9D000397197F00000E780E0B49305400661E913
:10B9E00097800000E78000606302051497A7FF1F9F
:10B9F00083C7C73713B7170097A6FF1F2388E636FC
:10BA0000014499CFC16417A9FF1F1309295793094E
:10BA1000400EFD1497000000E78020836342A40AD3
:10BA200097F0FFFFE78060094169B7290900096ABB
:10BA3000FD7A2A8B81447D199389F97B130A0A7157
:10BA4000938A8AC797000000E780208063D7A40408
:10BA50001304400EB387840217A7FF1F1307075272
:10BA60000324070B3E948357C4016382270B1840BD
:10BA70003307EB4063EAE900834744008507B38757
:10BA80004703D6976365F70801468145094597F056
:10BA9000FFFFE780C04AAA8B29E597400000E780B6
:10BAA000808385476317F50689659385057117A51A
:10BAB000FF1F1305E52997100100E780A04F95A00F
:10BAC000B30734030327090BBA9703D7C7016308E9
:10BAD000970003C75700A38207002382E7000504ED
:10BAE00015BF9305C500228597000000E78080E61A
:10BAF0005E852286976501009385C5E997F0FFFF73
:10BB0000E780404F5E8597100000E780608A8504DB
:10BB100015BF97A7FF1F938767469C478D83858B2B
:10BB2000C1F721611763FFFF6700635C014685452C
:10BB3000094502D002D202D402D697F0FFFFE78077
:10BB40000040AA8479DD97F00000E780E09C13892B
:10BB5000C4002A8481454A8597000000E780005F81
:10BB60000C4041464A8597000000E780405B8329EE
:10BB700044006385090C4E8502D802DA02DC02DE3D
:10BB800097300100E780E0382ACE141005462C08D3
:10BB900008184ECC97500000E780E00A1375F50FA7
:10BBA00051ED8355840093E525004A8597000000F8
:10BBB000E780E05E11460C104A8597000000E780A0
:10BBC0000056014697650100938545DD268597F06F
:10BBD000FFFFE7802042268597000000E780407D38
:10BBE0005C40A1D3014685450D4597F0FFFFE780F6
:10BBF0000035AA841DD548401389C4009730010040
:10BC0000E78020312AC64A8597000000E780404C33
:10BC10003246636FC5004C404A8597000000E780BC
:10BC2000005001468145268597F0FFFFE780803C64
:10BC3000268597000000E780A077E5B5835584004E
:10BC4000ADB71763FFFFE702834997A7FF1F9387ED
:10BC5000E7329C471DC193E7870017A5FF1F130517
:10BC6000250F17A7FF1F232FF73097100100E7803C
:10BC700040321763FFFF6700C348DD9B17A7FF1F14
:10BC80002322F73097300000E780E0647DF117A5AC
:10BC9000FF1F1305E50B97100100E780E033D1BFCC
:10BCA0001763FFFFE70223414169AA892E8AB28AFE
:10BCB000368BBA8B814417ACFF1F130C2C2C930CC2
:10BCC000400E7D1997F0FFFFE780205863C4A40061
:10BCD00001443DA03384940383270C0B3E94835787
:10BCE000C401638627055A87D6865286CE851305FA
:10BCF000040397000000E780E0BB01C923800B002C
:10BD000022851763FFFF6700833E8347F40185C3E5
:10BD10005A87D6865286CE85130594089700000070
:10BD2000E78040B909C585472380FB00D1BF850462
:10BD300051BF835745006380071E1763FFFFE7026B
:10BD4000633801112A8497000000E780C04D09C9BB
:10BD500085476309F50605611763FFFF6700C3396F
:10BD600097E00000E780007C7DF583574400494759
:10BD7000ED9BE392E7FEC145228597000000E78036
:10BD80004033AA84228597000000E780204F0357A4
:10BD9000440002CE91472A89631AF7002285970052
:10BDA0000000E780A0513C082ACC3ECE97E000007E
:10BDB000E78080765C55C5D374084A86A68505451C
:10BDC000829751BF03574400D147E3F6E7F8032AAF
:10BDD0000400C169014997AAFF1F938A2A1A130B0D
:10BDE000400EFD1997F0FFFFE7802046634FA90E34
:10BDF0002285032A040097000000E780C042A14585
:10BE00002A89228597000000E780A02AAA8422853B
:10BE100097000000E780804A14402A86AA897808A3
:10BE20002685CA8597000000E780C0E7AA8405D56B
:10BE300003C7F40189476315F7008347C10181DF18
:10BE40005546D2851385640097300100E780E0E70E
:10BE5000014597800000E780C01901C583D7C40160
:10BE6000A5E797A7FF1F938767119C479355190074
:10BE7000858913D73700058B01CF8983858B63991B
:10BE8000B70001452EC697000000E780C0DBB24531
:10BE90004E8597800000E780601F0346C1012A8419
:10BEA00093751900268597900000E780E03935C129
:10BEB000268597800000E780E018268511C001459F
:10BEC00097800000E780004C97300000E780A0409A
:10BED0008547E312F5E883C754001307F00FE38C9E
:10BEE000E7E68507A382F400BDB5B304690383A721
:10BEF0000A0BBE9483D7C401638B37015546D285A4
:10BF00001385640097300100E780C0D955DD05092D
:10BF1000D1BD5DD86DB782801763FFFFE702831A3A
:10BF200097800000E780000C05C1C164014417A997
:10BF3000FF1F1309A9049309400EFD1497F0FFFF9A
:10BF4000E780A030634EA40017A5FF1F130545E04E
:10BF500097100100E780E0031763FFFF6700C31934
:10BF6000330534038327090B3E958357C501638846
:10BF700097002312050097800000E780A00C0504BD
:10BF800075BF97A7FF1F938767FF9C478D83858B9E
:10BF90008DE31763FFFFE702831417A5FF1F130547
:10BFA00025DB97100100E78020031763FFFF670080
:10BFB000431582801763FFFFE702631297050000B5
:10BFC0009385C5A017A5FF1F130585D897100100FD
:10BFD000E78020EE1763FFFF6700A3121763FFFFE0
:10BFE000E702E30F8841B7E70400BC5B05054205A3
:10BFF0004181829709C585472300F5000505176330
:10C00000FFFF6700031083C7F5FF2E858507A38F09
:10C01000F5FE828083C7F5FFFD1793F7F70FA38F17
:10C02000F5FE99EF1763FFFFE702630BB7E7040024
:10C03000BC571385F5FF82971763FFFF6700630CFA
:10C0400082801C41035745008D8FBA951CC1231275
:10C05000B5003E85828093D78500A2051441DD8D11
:10C06000835745001387E6FF18C189072312F5009F
:10C0700013D685004111238FB6FEA38FC6FE410162
:10C08000828018419307F7FF1CC18357450085073D
:10C090002312F500A30FB7FE8280835745008D8FD2
:10C0A0002312F5001C41BE950CC12E858280AA8703
:10C0B00003D7470008410D8FAA952392E7008CC350
:10C0C0008280184108453305A74082808357450088
:10C0D000035765001D8F1C4108453385A740330574
:10C0E000A74082801763FFFFE70263FF41112EC65E
:10C0F0002A8497000000E780A0FDB2456373B50075
:10C1000001A0835744000840BE952312B4003E9519
:10C1100041011763FFFF6700C3FE1763FFFFE702DC
:10C1200003FC41112E84B28532C697000000E780DF
:10C13000A0FB3246A28597300100E78000B941019B
:10C140001763FFFF6700E3FB1763FFFFE70223F9B5
:10C150002E84854597000000E78000F923008500C4
:10C160001763FFFF6700E3F91763FFFFE70223F799
:10C1700041112317B100894597000000E780C0F600
:10C180008347E1002300F5008347F100A300F50099
:10C1900041011763FFFF6700C3F61763FFFFE70264
:10C1A00003F493D78500A2054111DD8D2317B1005B
:10C1B000894597000000E78020F38347E1002300D2
:10C1C000F5008347F100A300F50041011763FFFF6D
:10C1D000670023F31763FFFFE70263F013978501FE
:10C1E00093D78501C166938606F0D98F13D7850052
:10C1F000758FD98FA2053707FF00F98D4111DD8DAD
:10C200002EC6914597000000E78000EE6C001146B5
:10C2100097300100E78060AB41011763FFFF6700C3
:10C2200043EE1763FFFFE70283EB1C41854503C420
:10C23000070097000000E78080E622851763FFFF74
:10C24000670023EC1763FFFFE70263E91C4141111C
:10C25000894503C7070083C717002307E100A30729
:10C26000F10097000000E78080E30355E100410101
:10C270001763FFFF6700E3E81763FFFFE70223E6AA
:10C280001C414111894503C7070083C717002307D5
:10C29000E100A307F10097000000E78040E083572A
:10C2A000E100410113D58700A2075D8D4205418160
:10C2B0001763FFFF6700E3E41763FFFFE70223E272
:10C2C0000C4141112A841146680097300100E78033
:10C2D000C09F9145228597000000E78040DCB2476F
:10C2E000C166938606F01397870113D58701598D90
:10C2F00013D78700758F598DA2073707FF00F98F75
:10C300005D8D41011763FFFF6700A3DF1C45BE95EC
:10C310000CC18280AE87944391E6584101EF0CC175
:10C320005CC1828003C7570013671700A382E70030
:10C33000B687D5B70CC3EDB7AA87084119CD184108
:10C34000D44398C36313D500D8C32A870346570044
:10C350009376160081E6232007008280944381CAE9
:10C360008C4203A847008CC363930601CCC3799A1F
:10C3700014C3A302C7003687D1BF1C45DC471D8DFF
:10C38000B777DBB6938777DB09853305F50242057E
:10C3900041818280F147B385F50248452E95828020
:10C3A0008347450085072302F50082801763FFFF5E
:10C3B000E702E3D22A8409E41763FFFF670063D42E
:10C3C00083474400F5DBFD1793F7F70F2302F400D2
:10C3D000E5F71C4403D7270005072391E700DC435A
:10C3E00099C3228582974C4889CD83475400898B15
:10C3F00099E71C4422859C479C439C478297232AAB
:10C4000004000040232004007DB71763FFFFE7020C
:10C4100003CD8357250041112EC681EB01442285AF
:10C4200041011763FFFF6700C3CD03570500814734
:10C43000F146E305F7FEB385D702404585072E9404
:10C440008345440008C4F5F5B247AA8481E7232A4E
:10C45000040009A81C456C0022859C439C438297DC
:10C4600048C84DDD85472312F400B247232004005D
:10C47000231804002319F4005C485CC483D724000B
:10C48000FD172391F40061BF1763FFFFE70223C587
:10C4900097A7FF1F9387C78D884323260500232472
:10C4A0000500410597100100E78000B31763FFFF07
:10C4B000670023C51763FFFFE70263C217A4FF1FCE
:10C4C0001304048B1C40411199CF9C472300B500F5
:10C4D0002AC65CC197000000E78040FB1C40DC439B
:10C4E00099C33245829741011763FFFF670063C11B
:10C4F0000347450029E3584DAA877D551DCF176393
:10C50000FFFFE702C3BD1CC3DC4797A6FF1F23A1A3
:10C51000E686F156130507012390D7009705000022
:10C520009385050297100100E780A09801451763E5
:10C53000FFFF670003BD7D55828082801763FFFF88
:10C54000E702E3B901116146814528009760FFFFCA
:10C55000E780E0BB97A7FF1F938787819C43280054
:10C560009305F00FDC473EC697000000E780C0F45B
:10C5700005611763FFFF6700C3B89797FF1F938795
:10C58000277F9C43D847A1679387C702631EF70A9A
:10C59000397106DE22DC26DA80004AD84ED652D423
:10C5A00056D23285B28497000000E780C0C7AA89BE
:10C5B000268597000000E78020C92318A4FC268563
:10C5C00097000000E78040C82319A4FC2685970047
:10C5D0000000E78060C783D744000A8A231AA4FCBE
:10C5E000858393F7F70F230EF4FC8607BD0793F7B7
:10C5F000073F3301F1408A8A01498347C4FD6367DD
:10C60000F902CE85130584FC232C54FD970000000D
:10C61000E78080EA5281130104FCF2506254D25444
:10C620004259B259225A925A216182802685970036
:10C630000000E78060C193171900D6970509239081
:10C64000A7001379F90F55BF82809797FF1F938733
:10C6500027729C43D847A1679387A702631AF70AFA
:10C66000397106DE22DC26DA80004AD84ED652D452
:10C6700056D23285B28497000000E780C0BAAA89FA
:10C68000268597000000E78020BCFD572318A4FCF6
:10C6900026852319F4FC97000000E780E0BA83D7D1
:10C6A00044000A8A231AA4FC858393F7F70F230E0C
:10C6B000F4FC8607BD0793F7073F3301F1408A8AF0
:10C6C00001498347C4FD6367F902CE85130584FCE5
:10C6D000232C54FD97000000E78000DE52811301F7
:10C6E00004FCF2506254D2544259B259225A925A1E
:10C6F00021618280268597000000E780E0B49317CF
:10C700001900D69705092390A7001379F90F55BF93
:10C7100082809797FF1F9387A7659C43D847A1679F
:10C7200089076310F70A397106DE22DC26DA8000F9
:10C730004AD84ED652D456D232853289970000005C
:10C74000E78060AEAA894A8597000000E780C0AF05
:10C75000835749000A8A2318A4FC858393F7F70FAF
:10C76000230CF4FC8607BD0793F7073F3301F14024
:10C770008A8A8144834784FD63E7F402CE851305EA
:10C7800084FC232A54FD97000000E780E0D2528108
:10C79000130104FCF2506254D2544259B259225A45
:10C7A000925A216182804A8597000000E780C0A9E3
:10C7B00093971400D69785042390A70093F4F40F61
:10C7C00055BF82809797FF1F9387875A9C43D8470E
:10C7D000A1679387E704631EF70A397106DE22DC3E
:10C7E00026DA80004AD84ED652D456D23285B28448
:10C7F00097000000E78020A3AA8926859700000003
:10C80000E78080A42318A4FC268597000000E78019
:10C81000A0A3231AA4FC268597000000E780C0A2ED
:10C8200083D744000A8A2319A4FC858393F7F70F62
:10C83000230EF4FC8607BD0793F7073F3301F14051
:10C840008A8A01498347C4FD6367F902CE851305CF
:10C8500084FC232C54FD97000000E780E0C5528142
:10C86000130104FCF2506254D2544259B259225A74
:10C87000925A21618280268597000000E780C09C43
:10C8800093171900D69705092390A7001379F90F7C
:10C8900055BF82809797FF1F9387874D9C43D8474A
:10C8A000A1679387C704631AF70A397106DE22DC91
:10C8B00026DA80004AD84ED652D456D23285B28477
:10C8C00097000000E7802096AA892685970000003F
:10C8D000E7808097FD572318A4FC2685231AF4FCD3
:10C8E00097000000E780409683D744000A8A231906
:10C8F000A4FC858393F7F70F230EF4FC8607BD078E
:10C9000093F7073F3301F1408A8A01498347C4FD09
:10C910006367F902CE85130584FC232C54FD970030
:10C920000000E78060B95281130104FCF2506254A8
:10C93000D2544259B259225A925A21618280268594
:10C9400097000000E780409093171900D6970509DB
:10C950002390A7001379F90F55BF82809797FF1F87
:10C96000938707419C43D847A167DD076317F70406
:10C970001753FFFFE702A37679713285328497005F
:10C980000000E780408A2AC6228597000000E780E1
:10C99000A08B2311A102228597000000E780A088C8
:10C9A000B2452300A102280897000000E780C0B02C
:10C9B00045611753FFFF6700C37482809797FF1F7D
:10C9C0009387073B9C43D847A167938787046317E6
:10C9D000F7041753FFFFE7028370797132853284C1
:10C9E00097000000E78020842AC622859700000077
:10C9F000E78080852311A102228597000000E7804F
:10CA00008082B2452300A102280897000000E78039
:10CA1000A0AA45611753FFFF6700A36E8280979716
:10CA2000FF1F9387E7349C43D847A1679387A704E8
:10CA30006312F7021753FFFFE702636A0111280030
:10CA4000814597000000E78020A705611753FFFF8D
:10CA50006700236B82809797FF1F938767319C4302
:10CA6000D847A167938757026319F7021753FFFF4F
:10CA7000E702E3660111328597F0FFFFE780A07AB5
:10CA80002308A1008145280097000000E780C0A28C
:10CA900005611753FFFF6700C36682809797FF1FEA
:10CAA0009387072D9C43D847A1679387E702631BB1
:10CAB000F7041753FFFFE7028362011132853284C6
:10CAC00097F0FFFFE7804078AA84228597F0FFFF68
:10CAD000E7808077854709E9228597F0FFFFE780A7
:10CAE00080744205B337A0002800814523189100C7
:10CAF0003ECA97000000E780209C05611753FFFFA6
:10CB00006700236082809797FF1F938767269C4367
:10CB1000D84799476313F7081753FFFFE702235CD1
:10CB200079713285328497F0FFFFE780C06F2AC6A3
:10CB3000228597F0FFFFE78020712310A102228554
:10CB400097F0FFFFE780206E2301A102228597F076
:10CB5000FFFFE780406DA301A102228597F0FFFF50
:10CB6000E780606C2302A102228597F0FFFFE78037
:10CB7000806B2313A102228597F0FFFFE780A06A54
:10CB8000B2452314A102280897000000E780C09254
:10CB900045611753FFFF6700C35682809797FF1FB9
:10CBA0009387071D9C43D847A1679387C7036313E7
:10CBB000F7081753FFFFE7028352797132853284F9
:10CBC00097F0FFFFE78020662AC6228597F0FFFFD7
:10CBD000E78080672310A102228597F0FFFFE7809E
:10CBE000A0662311A102228597F0FFFFE780A063D2
:10CBF0002302A102228597F0FFFFE780C062A30213
:10CC0000A102228597F0FFFFE780E0612303A102E4
:10CC1000228597F0FFFFE7800061B245A303A102E0
:10CC2000280897000000E780208945611753FFFF1F
:10CC30006700234D82801753FFFFE702434A01112B
:10CC40002A8497F0FFFFE780005EAA84228597F090
:10CC5000FFFFE780605F228597F0FFFFE780C05EFF
:10CC6000035744008D4763F7E700228597F0FFFFE5
:10CC7000E780805D228597F0FFFFE780E05C280079
:10CC8000A68597000000E780208305611753FFFF0A
:10CC9000670023479797FF1F9387870D9C43D847CB
:10CCA000A167FD07631FF7001753FFFFE702234348
:10CCB000328597000000E78040F81753FFFF6700B8
:10CCC000434482809797FF1F9387870A9C43D847E6
:10CCD000A167E5076315F7081753FFFFE702234035
:10CCE00079713285328497F0FFFFE780C0532AC6FE
:10CCF000228597F0FFFFE7802055228597F0FFFF00
:10CD0000E78080542310A102228597F0FFFFE7807F
:10CD1000A053520551812311A10222852302010251
:10CD200097F0FFFFE7802050A302A102228597F031
:10CD3000FFFFE780404F2303A102228597F0FFFF0A
:10CD4000E780604EB245A303A102280897F0FFFFD9
:10CD5000E780807645611753FFFF6700833A828042
:10CD60009797FF1F9387C7009C43D847A167938776
:10CD7000E703631FF7001753FFFFE70243363285CF
:10CD800097000000E78060EB1753FFFF67006337F1
:10CD900082809797FF1F9387A7FD9C43D847A16781
:10CDA00093874704631EF7021753FFFFE7022333FD
:10CDB00079713285328497F0FFFFE780C0462AC63A
:10CDC000228597F0FFFFE7802048B245280897F0BA
:10CDD000FFFFE780606E45611753FFFF6700633216
:10CDE00082809797FF1F9387A7F89C43D847A16736
:10CDF000938787026310F7041753FFFFE702232E80
:10CE000079713285328497F0FFFFE780C0412AC6EE
:10CE1000228597F0FFFFE7800041B2452300A10281
:10CE2000280897F0FFFFE780206945611753FFFF4F
:10CE30006700232D82801753FFFFE702432A011169
:10CE400097F0FFFFE780203EAA85280097F0FFFFBC
:10CE5000E780806605611753FFFF6700832A979775
:10CE6000FF1F9387E7F09C43D847A167D107631F53
:10CE7000F7001753FFFFE702832632859700000073
:10CE8000E780A0FB1753FFFF6700A32782809797D7
:10CE9000FF1F9387E7ED9C43D847A167C507631F32
:10CEA000F7001753FFFFE702832332859700000046
:10CEB000E780A0F81753FFFF6700A32482809797AD
:10CEC000FF1F9387E7EA9C43D847A167B907631F11
:10CED000F7001753FFFFE702832032859700000019
:10CEE000E780A0F51753FFFF6700A3218280979783
:10CEF000FF1F9387E7E79C43D847A167AD07631FF0
:10CF0000F7001753FFFFE702831D328597000000EB
:10CF1000E780A0F21753FFFF6700A31E8280979758
:10CF2000FF1F9387E7E49C43D84789476318F702BC
:10CF30001753FFFFE702A31A0111328532C897F099
:10CF4000FFFFE780402EAA85280097F0FFFFE780CB
:10CF5000A05605611753FFFF6700A31A82809797B9
:10CF6000FF1F9387E7E09C43D847A1678D076311B4
:10CF7000F7041753FFFFE70283160111328532844D
:10CF800097F0FFFFE780202A13066100AA844C0077
:10CF9000228597300000E780C0232800A68597F0FF
:10CFA000FFFFE780605105611753FFFF67006315BE
:10CFB00082809797FF1F9387E7DB9C4381CFDC43F9
:10CFC00091CB1753FFFFE702831182971753FFFF9F
:10CFD0006700231382801753FFFFE7024310797124
:10CFE0003C08AE843ED2A165B7070A002A843ED42D
:10CFF00048103C08DD053ED636C432C63AC297D04A
:10D00000FFFFE780402C12474810BA8597F0FFFFDA
:10D01000E780C01332464810B28597F0FFFFE780E3
:10D02000E014A2464810B68597F0FFFFE780001293
:10D03000501001478146A685228597D0FFFFE780E3
:10D04000E04D45611753FFFF6700A30B1753FFFF28
:10D05000E702E30801117C000329C501AE843ECA42
:10D06000A165B70707002A843ECC48087C00C505A7
:10D070003ECE97D0FFFFE78000258345D9004808C2
:10D0800097F0FFFFE780800C500801478146A68596
:10D09000228597D0FFFFE780604805611753FFFFA7
:10D0A000670023061753FFFFE702630383C795005A
:10D0B00093F7F707A384F50097000000E78040F995
:10D0C0001753FFFF6700E3031753FFFFE702230136
:10D0D00079713C08AE843ED2A165B70709002A8465
:10D0E0003ED448103C08938545043ED632C636C42B
:10D0F00097D0FFFFE780201DA2464810B68597F025
:10D10000FFFFE780A00432464810B28597F0FFFF8A
:10D11000E780C005501001478146A685228597D03B
:10D12000FFFFE780A03F45611753FFFF670063FDE6
:10D130001753FFFFE702A3FA83C7950041112A8422
:10D1400093F7F707A384F50032852EC697F0FFFF0B
:10D15000E780800F85672AC46370F502977000002E
:10D16000E78020E92246B24509ED11478146228534
:10D1700097000000E78060E641011753FFFF67005A
:10D1800043F801478346F501DDB71753FFFFE70278
:10D1900063F301113C003ECAB7070A003ECC3C00D5
:10D1A0003ECE83C79500AA89328593F7F707A384FB
:10D1B000F5002E8497F0FFFFE78000098567637D07
:10D1C000F504A165AA8493858504480897D0FFFFDC
:10D1D000E780600F268597700000E78080E12A894C
:10D1E00029E19145480897F0FFFFE78020F6A685E2
:10D1F000480897F0FFFFE78060F7CA85480897F076
:10D20000FFFFE780A0F4014781465008A2854E85C4
:10D2100097D0FFFFE780803005611753FFFF67005D
:10D22000A3ED8145480897F0FFFFE78020F203490E
:10D23000090275BF1753FFFFE702C3E879711C109D
:10D240003ECAB7070F003ECC404D1C10AA84AE89E1
:10D250004808994532C636893ECE97D0FFFFE78011
:10D26000800632464808B28597F0FFFFE78000EE5F
:10D27000630C0902A545480897F0FFFFE780C0E668
:10D280002546CA8597200100E78020A45008014761
:10D290008146CE85268597D0FFFFE780202845610F
:10D2A0001753FFFF670043E58355C402480897F012
:10D2B000FFFFE780A0EB0355E402814505C58547E4
:10D2C00085456301F502C167FD179305F00F630BF8
:10D2D000F5007D1597700000E780208E93051500FE
:10D2E00093F5F50F480897F0FFFFE78020E68345A8
:10D2F0000403480897F0FFFFE78040E583451403E7
:10D30000480897F0FFFFE78060E48355240348084E
:10D3100097F0FFFFE78080E583554403480897F0C6
:10D32000FFFFE780A0E49DB71753FFFFE70223DB71
:10D3300083C795008146014693F7F707A384F5005C
:10D3400097000000E78040EF1753FFFF670063DBA3
:10D350001753FFFFE702A3D879713E841C103ECA21
:10D360002E89B7070F00A1653ECCFD051C10AA84CD
:10D37000480842C03AC23ECE36C432C697D0FFFFFC
:10D38000E78060F432464808B28597F0FFFFE780F7
:10D39000E0DBA2464808B68597F0FFFFE78000DD96
:10D3A00012474808BA8597F0FFFFE78020DC024863
:10D3B000630C08029145480897F0FFFFE780C0D250
:10D3C0001146A28597200100E78020905008014770
:10D3D0008146CA85268597D0FFFFE78020144561E6
:10D3E0001753FFFF6700E3D18945480897F0FFFF17
:10D3F000E78080CF834704002300F50083471400B3
:10D40000A300F500E1B71753FFFFE702A3CB83C7E3
:10D41000950001112A8A93F7F707A384F500328556
:10D42000AE8432C697F0FFFFE78000E232462A89D9
:10D43000328597F0FFFFE78000DF85676373F902AD
:10D44000AA894A8597700000E780A0BA2A8419ED5E
:10D45000114781464A86A685528597000000E780DD
:10D46000C0B705611753FFFF670003C99387E9FF42
:10D4700093F7F70F0547E366F7FE8347F50195EB52
:10D480008947E380F9FE8346F401528501474A86C5
:10D49000A68597000000E78040B4A167D907480837
:10D4A0003ECC230A010002CE97000000E780A0B026
:10D4B0004DBF639EE7008947639EF90093071020E4
:10D4C000231FF50097700000E780C0B76DBF0947C4
:10D4D000E39BE7FA8D47E398F9FA228597700000FD
:10D4E000E78080DF9797FF1F9387C7A79C4399E743
:10D4F0009797FF1F9387C7909C4399C703D5040054
:10D5000097800000E780A0CE231F040022855DBF26
:10D510001753FFFFE702A3BC01113C003ECAB70747
:10D520000B003ECC3C003ECE83C795002A89328555
:10D5300093F7F707A384F500AE8497F0FFFFE78029
:10D54000A0D093170501C187635AF006A1652A840C
:10D550009385E502480897D0FFFFE780C0D6A285F3
:10D56000480897F0FFFFE78060C09797FF1F9387F9
:10D5700027899C43A9EB01449375F40F480897F061
:10D58000FFFFE780A0BC9355844093F5F50F480852
:10D5900097F0FFFFE78080BB9355044193F5F50FAB
:10D5A000480897F0FFFFE78060BA014781465008BE
:10D5B000A6854A8597D0FFFFE78040F6056117539F
:10D5C000FFFF670003B4416585460546A2857D15CA
:10D5D00097500000E78060BD59DD510597000100BC
:10D5E000E780808F130440063344850271B71753D8
:10D5F000FFFFE702C3AE0111B70706003EC683C7AF
:10D60000950021642A8993F7F707A384F500AE8477
:10D6100028009305A4040AC40AC897D0FFFFE78036
:10D6200080CA300001478146A6854A8597D0FFFF12
:10D63000E780C0EE97E0FFFFE780E0111304940459
:10D64000480822CC230A010002CE97000000E780A0
:10D65000809605611753FFFF6700A3AA1753FFFFCA
:10D66000E70243A6C1642A8901449799FF1F938961
:10D67000E990130A8002FD1497E0FFFFE780E0BD08
:10D680006347A40001451753FFFF6700E3A6B307F4
:10D69000440303A7C90ABA9703D707006306970094
:10D6A00083D72700638427010504F9B70545E1BF47
:10D6B0001753FFFFE70203A12A8A2E8999C123A0ED
:10D6C000050081498144978AFF1F938AEA6A614B6A
:10D6D00097E0FFFFE780A0BE63C7A4004E85175305
:10D6E000FFFF670063A13384640383A70A003E94AD
:10D6F0008357040099E76304090023208900850407
:10D70000C1BF4146D2851305440097100100E78050
:10D71000605975F5A289E5B71753FFFFE702839AB1
:10D7200039717C083ED4B7070A003ED67C083ED843
:10D7300083C795002A8A328593F7F707A384F500FB
:10D740002E8932C697F0FFFFE78000B085676373CC
:10D75000F5083246AA84328597F0FFFFE780A0AC37
:10D760008547AA8963E8A706A165938585042810E3
:10D7700097D0FFFFE78020B5268597700000E780EF
:10D7800040872A8429ED9145281097F0FFFFE78014
:10D79000E09BA685281097F0FFFFE780209DCE85AF
:10D7A000281097F0FFFFE780609A0147814630100C
:10D7B000CA85528597D0FFFFE78040D6A16793873F
:10D7C000770448183EDC230A010202DE97F0FFFFCF
:10D7D000E780607E21611753FFFF6700E391814579
:10D7E000281097F0FFFFE7806096A685281097F035
:10D7F000FFFFE780A0979797FF1F9387E7AE9C43B3
:10D8000081CB22856389090097D00000E7804024FE
:10D810008345040271B797D00000E780C022CDBFD6
:10D820001753FFFFE702038A83C795004111AA89B6
:10D8300093F7F707A384F5003285AE84328A97F018
:10D84000FFFFE78060A08567637FF5022A89976004
:10D850000000E780007A2A84914631C58347F501AC
:10D8600005476387E70291C70D476366F704AD4636
:10D870001DA89305050303250A00414697100100E2
:10D88000E78040420DE941011753FFFF6700C3865F
:10D890009305950803250A00414697100100E7808B
:10D8A0006040814669F54A86A6854E85970000004E
:10D8B000E780C081C9BF83250A00130594089770CB
:10D8C0000000E780A02919C1C146F1BF9787FF1F5B
:10D8D000938747699C4399E79787FF1F9387475230
:10D8E0009C4399C7228597800000E780208A69FDC4
:10D8F0008547A30FF400228597B00000E78060847D
:10D90000228597600000E780E0734E8581464A8655
:10D91000A68597F0FFFFE780607BA1679387570498
:10D9200048003EC42302010002C697F0FFFFE780D3
:10D93000806891BF1743FFFFE702E37783C7950035
:10D940004111AA8993F7F707A384F50032852E8940
:10D95000B28A97F0FFFFE780208F85676374F50E2A
:10D96000AA8497600000E780C0682A840DED416BAF
:10D97000014A978BFF1F938B6B60130C400E7D1B2E
:10D9800019A833048A0383A70B0B3E948357C40161
:10D9900063836705050A97E0FFFFE780008BE3429A
:10D9A000AAFE95460DA08357C5016396970293057D
:10D9B000050303A50A00414697100100E780802E69
:10D9C000994611E181462686CA854E8597F0FFFF6C
:10D9D000E780C06F85A883A50A001305040397702C
:10D9E0000000E780A017C14679FD2285231E940020
:10D9F00097A00000E780E074228597600000E78030
:10DA000060649797FF1F9387278E9C43A9C32300C9
:10DA10000402228597D00000E78040F04E858146C1
:10DA20002686CA8597F0FFFFE780406AA167938743
:10DA3000070448003EC42302010002C697F0FFFF1E
:10DA4000E780605741011743FFFF6700436A89473A
:10DA50002300F402E1B7397106DE22DC4AD88000E7
:10DA600052D456D25AD026DA4ED65ECE2E8A32897B
:10DA70002A8B97D0FFFFE780407A06057105419910
:10DA80008A8A3301A140232224FC231404FC97D06A
:10DA9000FFFFE780807883479A000605350593F7F6
:10DAA000F7072315A4FCA304FA004A85232624FCC7
:10DAB00097E0FFFFE780407993170501C187634036
:10DAC000F0025681130104FCF2506254D2544259C0
:10DAD000B259225A925A025BF24B21618280AA8487
:10DAE0004A8597E0FFFFE7802076AA894A8597E07C
:10DAF000FFFFE7806075A1659385C5022A8913053C
:10DB000044FC97C0FFFFE780007C268597C0FFFF9D
:10DB1000E7804070854511C94A86CE8597C0FFFFD2
:10DB2000E780C069AA8B21E98945130544FC97E089
:10DB3000FFFFE780A061A685130544FC97E0FFFF87
:10DB4000E780C062CE85130544FC97E0FFFFE780C5
:10DB5000E061CA85130544FC97E0FFFFE7800061A0
:10DB600001478146130644FCD2855A8597D0FFFFB2
:10DB7000E780C09AB9B78145130544FC97E0FFFFE1
:10DB8000E780C05CA685130544FC97E0FFFFE780B3
:10DB9000E05DCE85130544FC97E0FFFFE780005D64
:10DBA000CA85130544FC97E0FFFFE780205C8144B1
:10DBB00097D0FFFFE7806066E3D4A4FA83A70B0148
:10DBC00013971400BA9783D5070099C5130544FC31
:10DBD00097E0FFFFE78080598504D9BF797106D6A9
:10DBE00022D44AD000184ECE52CC56CA26D25AC899
:10DBF000AE893289AA8A97D0FFFFE78000620605C6
:10DC0000690541990A8A3301A140232A24FC231C77
:10DC100004FC97D0FFFFE780406083C799000605AA
:10DC20002D0593F7F707231DA4FCA384F9004A856B
:10DC3000232E24FC97E0FFFFE78000619317050186
:10DC4000C187634FF0005281130104FDB25022548A
:10DC500092540259F249624AD24A424B456182804B
:10DC6000AA844A8597E0FFFFE780005EA16593855F
:10DC7000A5022A89130544FD97C0FFFFE780A06431
:10DC8000268597C0FFFFE780E058854509C9CA850A
:10DC900097C0FFFFE78080552A8B29E1894513054E
:10DCA00044FD97E0FFFFE780604AA685130544FD29
:10DCB00097E0FFFFE780804BCA85130544FD97E09E
:10DCC000FFFFE780A04A01478146130644FDCE8549
:10DCD000568597D0FFFFE7806084B5B7814513056F
:10DCE00044FD97E0FFFFE7806046A685130544FDED
:10DCF00097E0FFFFE7808047CA85130544FD97E062
:10DD0000FFFFE780A046814497D0FFFFE780E05007
:10DD1000E3DBA4FA83270B0113971400BA9783D58A
:10DD2000070099C5130544FD97E0FFFFE780004415
:10DD30008504D9BF1743FFFFE702633A83474500D5
:10DD4000404DD5EFFD575DC483469400094763639A
:10DD5000D70A0346B400854663EEC6088306E4008E
:10DD600063CA06085C45F9562390D7009787FF1FC2
:10DD700083C7C70099E3A304E4009787FF1F938735
:10DD800027089C4381E78947A306F4009787FF1F74
:10DD9000938787559C4381E789472306F4009705BD
:10DDA000000093854506AA841305040197F000003E
:10DDB000E7802010FD57231AF40281471CDC01483C
:10DDC0009787FF1F23A887FA9787FF1F9387C7FAB4
:10DDD000232E040304C0804397D0FFFFE780204E2A
:10DDE00061463306C502814522859740FFFFE780E3
:10DDF000003281473E851743FFFF67008330FD57A0
:10DE0000D5BF1743FFFFE702832D2A840355450240
:10DE100097600000E780E01D19E5231E040017430A
:10DE2000FFFF6700032E8357E401F5DB930504FF32
:10DE300017450100130545F097E00000E780E01466
:10DE4000F9BF1743FFFFE70283292E89A16541111E
:10DE50009385E5032A8436C432C6BE843AC297C08D
:10DE6000FFFFE780404612472285BA8597E0FFFF13
:10DE7000E780C02D32462285B28597E0FFFFE7801C
:10DE8000E02EA2462285B68597E0FFFFE780002EB0
:10DE9000630309029145228597E0FFFFE780C024D4
:10DEA0001146A68597100100E78020E24101174343
:10DEB000FFFF670003258945228597E0FFFFE78084
:10DEC000A02283C704002300F50083C71400A30029
:10DED000F500E9BF1743FFFFE702632083C7950002
:10DEE000444D054793F7F707A384F5001C42411101
:10DEF00083C707006367F7062E842A89B1C003C76A
:10DF0000D400630FF7021787FF1F130767EF18434B
:10DF100005C3A386F40097A00000E780404A83C7AA
:10DF2000D40099E741657D1597400000E7804030B7
:10DF300083D72403918B89C797E00000E780C01343
:10DF40004A85A28597F0FFFFE7808010A167C1078F
:10DF500048003EC42302010002C697F0FFFFE7809D
:10DF6000800541011743FFFF6700A3191743FFFF17
:10DF7000E702E31603D745008D47AA8441112E849A
:10DF800032892E8563E3E70297E0FFFFE780C02B2D
:10DF9000AA8523000900268597C0FFFFE78000259A
:10DFA00041011743FFFF6700C31597E0FFFFE780BC
:10DFB000A0292AC6228597E0FFFFE780E028B24526
:10DFC00085472A862300F900268597C0FFFFE78052
:10DFD000E01EF9B7397106DE22DC26DA80004ED663
:10DFE00052D456D24AD85AD05ECEAE89B284AA8ACA
:10DFF00097D0FFFFE78060210605130525024199B0
:10E000000A8A3301A140232224FC231404FC97D064
:10E01000FFFFE780801F83C7990006054D0593F732
:10E02000F7072315A4FCA384F9002685232624FCE6
:10E0300097E0FFFFE780402193170501C187634008
:10E04000F0025281130104FCF2506254D25442593E
:10E05000B259225A925A025BF24B21618280AA8BFA
:10E0600003AB040097C0FFFFE780C01A51E583D7D8
:10E07000440001498544F11793B71700A301F4FC4C
:10E08000834734FCA165C9C79385E504130544FCA7
:10E0900097C0FFFFE7802023A685130544FC97E087
:10E0A000FFFFE780A00ADE85130544FC97E0FFFF31
:10E0B000E780C00B834734FC114691E30946DA85BB
:10E0C000130544FC97E0FFFFE78060058144630A85
:10E0D0000900416B7D1B97D0FFFFE780001363CCE5
:10E0E000A40201478146130644FCCE85568597C09D
:10E0F000FFFFE780A042B1B7A685130634FC970066
:10E100000000E780E0E6933415002A8986048DBF7D
:10E110009385C504A5BF8327C90013971400BA9738
:10E1200083D5070063886501130544FC97E0FFFF72
:10E13000E780C003850445B71743FFFFE702A3F755
:10E1400079711C103EC4B7070F003EC61C103EC8B4
:10E1500083C79500AA8A328593F7F707A384F50051
:10E16000AE89328497E0FFFFE780000E9317050128
:10E17000C187635AF0062A8A228597E0FFFFE7806D
:10E18000A00C2A895285032B040097C0FFFFE7806B
:10E19000600839ED8357440081440544F11793B773
:10E1A0001700A303F10083457100DA872287CA862E
:10E1B0005286280097000000E780E0C801478146AA
:10E1C0003000CE85568597C0FFFFE7802035A167D8
:10E1D0009387D70348083ECC230A810026CE97F0C8
:10E1E000FFFFE78040DD45611743FFFF670023F035
:10E1F000A2851306710097000000E78060D7AA840B
:10E20000094455D13544E30055FB4A8597F0FFFF9B
:10E21000E78000450D4441D9014497D0FFFFE780D6
:10E22000C0FE634DA400C16B0144FD1B97D0FFFFEE
:10E23000E780A0FD634EA4001544B5B7DC44131776
:10E240001400BA9783D70700638327030504F1B747
:10E25000D84493171400BA9703D70700631B7701BC
:10E2600023902701268597A00000E78080DB0144EA
:10E270001DBF050465BF1743FFFFE702A3E483C783
:10E28000950041112A8A93F7F707A384F500328598
:10E290002E89328497E0FFFFE78000FB931705018A
:10E2A000C1876353F006AA89228597E0FFFFE780C4
:10E2B000A0F92311A1004E85832A040097C0FFFF17
:10E2C000E78040F539E58357440085440144F11760
:10E2D00093B71700A300F100034811000357210072
:10E2E000D6875285CE862686CA8597F0FFFFE780BF
:10E2F0006006A167F10748003EC42302910022C6D0
:10E3000097F0FFFFE78020CB41011743FFFF670035
:10E31000A3DEA2851306110097000000E78040C528
:10E320002A84894455D98357210011678544BA97B7
:10E33000C2071167C1831307F7EFE36FF7F89787F9
:10E34000FF1F938727C29C4381CB8545130521007E
:10E3500097500000E7802075835521002285814475
:10E3600097C0FFFFE780A0E125D923100500228593
:10E3700097A00000E78040CD85B71743FFFFE70275
:10E3800083D383C7950041112A8B93F7F707A384A2
:10E39000F50032852E8A328497E0FFFFE780C0EADD
:10E3A00093170501C1876351F006AA8A228597E079
:10E3B000FFFFE78060E92A895685832B040097C018
:10E3C000FFFFE78020E531E58357440081440544A1
:10E3D000F11793B71700A301F10003483100DE875E
:10E3E0005A854A87D6862286D28597F0FFFFE78036
:10E3F00060F6A167ED0748003EC42302810026C6EF
:10E4000097F0FFFFE78020BB41011743FFFF670044
:10E4100003CEA2851306310097000000E78040B5C7
:10E42000AA8409445DD99167CA97C2071167C1835D
:10E430001307F7EF0544E362F7FACA8597C0FFFFB9
:10E44000E780E0D3014451F9814997D0FFFFE7808D
:10E45000C0DC63DBA900984893971900BA9703D7EB
:10E46000070005EF2390270197D0FFFFE780E0DA50
:10E470001544E384A9F6268597A00000E780C0BC78
:10E480009787FF1F938707AE9C430144B9D74A85FE
:10E4900097500000E780C05889B785097DB71743BA
:10E4A000FFFFE70223C279713E847C083EC82E8AB2
:10E4B000B7071400A1653ECAE5057C08AA890808CB
:10E4C00036C4428932C6BA8AC6843ECC97C0FFFFA2
:10E4D000E78060DFCA85080897E0FFFFE78000C794
:10E4E00032460808B28597E0FFFFE78020C8A246C1
:10E4F000630A09049D45080897E0FFFFE780C0BE56
:10E500001D4681459740FFFFE78060C063890A0888
:10E510009145080897E0FFFFE78000BD1146A685FA
:10E5200097000100E780607A100801478146D28594
:10E530004E8597C0FFFFE78060FE45611743FFFFF0
:10E54000670083BBB685080897E0FFFFE78000C23D
:10E550001C400808D8439355C70185891207518389
:10E56000B205D98D97E0FFFFE78040C01C40080846
:10E5700083C5870097E0FFFFE78040BD1C40080887
:10E5800083C5A70097E0FFFFE78040BC1C40080858
:10E5900083C5970097E0FFFFE78040BB85BF8945B3
:10E5A000080897E0FFFFE78020B483C7040023003A
:10E5B000F50083C71400A300F500BDB71743FFFFA4
:10E5C000E70243B083C795004111AA8993F7F70783
:10E5D000A384F5003285AE84328497E0FFFFE780A4
:10E5E000A0C693170501C187635DF0042A89032A39
:10E5F000040097C0FFFFE780E0C119E9835744009A
:10E600000548F11793B71700A307F100814631A819
:10E610001306F100A28597000000E78060951DC5F4
:10E620001C459DC783D6470001480347F100930767
:10E630008500D2884A86A6854E8597000000E7802F
:10E6400040E641011743FFFF670003AB09487DBF68
:10E650001D486DBF1743FFFFE702C3A665715C0845
:10E660003EC4B7077B013EC65C083EC883C7950021
:10E670002A8A328593F7F707A384F500AE8997E0DD
:10E68000FFFFE78040BA8357E100E1C789452800D2
:10E6900097C0FFFFE78020C38145280097E0FFFF78
:10E6A000E780C0AA97C0FFFFE78000C99787FF1FD8
:10E6B000938787C39C431774FF1F0344246CAA8469
:10E6C0003334800099C3136424009777FF1F938726
:10E6D00027739C4399C3136444009787FF1F938754
:10E6E00067889C4399C31364840083D50400280081
:10E6F000014997E0FFFFE78060A783D52400280049
:10E7000097E0FFFFE78080A683D54400280097E0CC
:10E71000FFFFE780A0A597D0FFFFE78000AB931530
:10E720000501C181280097E0FFFFE78020A4A285B2
:10E73000280097E0FFFFE78060A39C446360F90234
:10E74000014781463000CE85528597C0FFFFE780A4
:10E75000E0DC59611743FFFF6700039ADC441314A0
:10E76000490028003E9497E0FFFFE78060968347CA
:10E7700044000347540089070607BA978607E36AEF
:10E78000F5FC835524002800814A97E0FFFFE780CD
:10E79000E09D83454400280097E0FFFFE780009B51
:10E7A00083455400280097E0FFFFE780209A8347C5
:10E7B000440063C9FA00814A8347540063C1FA02E6
:10E7C0000509A5BF1C4413975A002800BA9783D5A2
:10E7D0000700850A97E0FFFFE7804099C9BF032B38
:10E7E000C40093975A0028003E9B83552B00850A4E
:10E7F00097E0FFFFE780809783550B00280097E0A4
:10E80000FFFFE780A0964DBF1743FFFFE702238D70
:10E810005C4993E717005CC997A00000E78020B629
:10E820001743FFFF6700E38D1743FFFFE702238BCA
:10E830002E84814597F0FFFFE780C0E705C5835729
:10E840000500FD172310F50009C483572500231088
:10E85000F40097000000E78060FB01451743FFFFCD
:10E860006700238A31457DD823100400C5BF1743B4
:10E87000FFFFE702238583C7950041112A8A93F79A
:10E88000F707A384F50032852E89328497E0FFFFD5
:10E89000E780809B93170501C1876356F006AA891C
:10E8A000C145228597E0FFFFE780A0802A8B4E8537
:10E8B000832A040097C0FFFFE780C09531E98357A2
:10E8C0004400231101000544F11793B71700A3007A
:10E8D000F10081440348110003572100D687528577
:10E8E000CE862286CA8597F0FFFFE780A0A6A167A3
:10E8F0009387170248003EC42302810026C697E092
:10E90000FFFFE780406B41011733FFFF6700C37EC5
:10E9100013061100A28597F0FFFFE7806065AA84C7
:10E9200009E523110100094475B7930521005A85B3
:10E9300097000000E78080EF835721002A84D9DB0D
:10E940009777FF1F938707629C4381CB854513050B
:10E95000210097500000E78000158355210026858F
:10E96000314497C0FFFFE78080812DD5231005003B
:10E97000268597900000E780206D0144A1BF1733E2
:10E98000FFFFE702C37541112E896C00AA8402C6FD
:10E9900097F0FFFFE78000D20DC103570500050780
:10E9A0002310E50097000000E78040E681473E85A0
:10E9B00041011733FFFF6700C3743247954765DB9A
:10E9C000CA85268597300000E780400DC147E340A7
:10E9D00005FE3244854741462310F4008357090061
:10E9E000A685130544002311F40097000100E78079
:10E9F000C02D228545BF1733FFFFE702A36C83C7F5
:10EA000095004111AA8A93F7F707A384F500328590
:10EA1000AE89328497E0FFFFE780008393170501FA
:10EA2000C1876356F0062A8AC145228597D0FFFF29
:10EA3000E7802068AA845285032B040097B0FFFF6B
:10EA4000E780407D31E9835744002311010085446C
:10EA5000F11793B71700A300F10001440348110018
:10EA600003572100DA875685D2862686CE8597F011
:10EA7000FFFFE780208EA1679387070248003EC40E
:10EA80002302910022C697E0FFFFE780C0524101B8
:10EA90001733FFFF67004366A2851306110097F046
:10EAA000FFFFE780E04C2A8409E523110100894437
:10EAB00075B726859305210097000000E78060EC7C
:10EAC000AA8449FD83552100228597B0FFFFE78086
:10EAD000006B49F5014997C0FFFFE7800074635D53
:10EAE000A900184893171900BA9703D707000DEF2C
:10EAF000035721002390E70097C0FFFFE780E071F4
:10EB0000630625039777FF1F9387C7459C4399C7E3
:10EB10000355210097500000E78080F022859790F0
:10EB20000000E78060521DBF050975B795443DB7E9
:10EB300005C19307F00F630FF500C547630CF5009F
:10EB40009307F5FF05453315F500420541818280A5
:10EB50000145828041657D158280B9E91733FFFF49
:10EB6000E702E35703450603328497000000E7807D
:10EB700060FC9305803EB305B502C205C18181CD1D
:10EB80000357E402854763F8E7001305040197E0A3
:10EB90000000E78020428357E40241677D176385C8
:10EBA000E700FD172317F4021733FFFF67006355D3
:10EBB00082801733FFFFE7020350004283C79500AE
:10EBC000444D0349140093F7F707A384F5008347E6
:10EBD0000400220911673369F900A167B347F900FE
:10EBE00041112A8BAE8A63ECE70E8347240013079A
:10EBF000C00EB91793F7F70F6373F710034734008C
:10EC0000C14763EEE70E834744001307E00793C74D
:10EC100007086371F70C8349840083477400A209D5
:10EC2000B3E9F900856763F7F90A034A640083478B
:10EC300054004E85220A336AFA0097500000E7809C
:10EC4000403B61C123962403834B3400137AFA00BE
:10EC5000239A34032388740323994403938904017A
:10EC6000631C090023A60402239804024E8597E042
:10EC70000000E78060363DA0034924004A859700E4
:10EC80000000E78020EB2397A402834744004E85D1
:10EC9000A388F402E38D0BFCE30B09FC97E0000072
:10ECA000E780202F97900000E7800073814601469F
:10ECB000D6855A8597E0FFFFE7800058A1679387C4
:10ECC00097033EC423020100480002C697E0FFFFFD
:10ECD000E780602E41011733FFFF67004341854401
:10ECE000A2862686D6855A8597E0FFFFE780C05426
:10ECF000A167938797033EC423029100F1B7BD44F7
:10ED0000C5B79144F1BF1733FFFFE702A33B0111E1
:10ED10001C08404D3EC2B7070F003EC41C083EC64B
:10ED20002A89AE8997C0FFFFE78000D7585C1C5C3A
:10ED30006346B70E6394E50063E2A70E3385A740F0
:10ED4000B3B7A700B305B7401306803E81469D8D3B
:10ED500097000100E78080B793140501C180A16589
:10ED60009385C503480097B0FFFFE780C0558145F4
:10ED7000480097D0FFFFE780603D835504044800BA
:10ED800097D0FFFFE780803E83552404480097D04A
:10ED9000FFFFE780A03D814589CCC167FD17930542
:10EDA000F00F6388F400268597500000E780E0E0CC
:10EDB000AA85480097D0FFFFE780403903554404F7
:10EDC000814501CDC167FD179305F00F6307F5007D
:10EDD00097500000E78060DEAA85480097D0FFFFCB
:10EDE000E780C03683456404480097D0FFFFE78082
:10EDF000E03583457404480097D0FFFFE780003575
:10EE0000500001478146CE854A8597B0FFFFE780D5
:10EE1000E07005611733FFFF6700032E814481B75F
:10EE20001733FFFFE702A32B83C7950093F7F7077C
:10EE3000A384F50097000000E78020ED1733FFFF63
:10EE40006700232C1733FFFFE702C32783C7950012
:10EE50004111404D93F7F707A384F5002A8A3285C4
:10EE6000B284AE8997D0FFFFE780003E2A8B2685CB
:10EE700097D0FFFFE780403D2A89268597D0FFFF86
:10EE8000E780603A93170B0163CA0702E177CA97DC
:10EE9000C207C183116763E3E70293070910C20742
:10EEA000C1831307B00F637BF70093170901C18774
:10EEB000AA8A634AF000C54763FE57014101173330
:10EEC000FFFF6700632397B0FFFFE7802025E3176C
:10EED00025FFD5B763080B026306090281446389E5
:10EEE0000A02B7077F0023106405231124057CC0A4
:10EEF000568597000000E780E0C39304803EB3048A
:10EF0000950239A0B7077F00232004047CC0814408
:10EF10000355240497E00000E780A0A3A1C497C094
:10EF2000FFFFE78060B7269593D7F441333795000C
:10EF3000AE97BA9708DC5CDCCE855285970000005E
:10EF4000E780A0DC99E023220404A1679387B7033C
:10EF500048003EC42302010002C697E0FFFFE7809D
:10EF60008005A9BF814701481CDC232E0403E9B7B3
:10EF70001733FFFFE702A31697C0FFFFE780203497
:10EF8000E1473305F502914597500000E78000C541
:10EF9000E55711C59777FF1F23A0A7DE81473E8560
:10EFA0001733FFFF6700E31585471777FF1F230718
:10EFB000F7DC82801733FFFFE70263129777FF1FAA
:10EFC000938747DB80433DC0835704046390A706C3
:10EFD00083572404639CB7043689B28497C0FFFF2B
:10EFE000E78080AB5C5C63C3B7046395B7001C5CCF
:10EFF00063EEA7028347640463F3F400A687230348
:10F00000F4048347740463F39700A687A303F4040E
:10F010008357440441677D176385E7008507231202
:10F02000F4043C4481C7CA85268582971733FFFFC5
:10F030006700230D9777FF1F9387C7D39C43014534
:10F0400099C303C5870082801733FFFFE7022309B6
:10F050000111B70707003EC683C79500584D0AC483
:10F0600093F7F7070AC8A384F5002A89AE8411CB69
:10F070001C4283C707002304F70097900000E78035
:10F080000034216493055402280097B0FFFFE78005
:10F09000802397000000E78020FAAA85280097D0F7
:10F0A000FFFFE780A00A300001478146A6854A8518
:10F0B00097B0FFFFE780804613044402480822CC43
:10F0C000230A010002CE97E0FFFFE780C0EE056152
:10F0D0001733FFFF6700E3021733FFFFE702230048
:10F0E00001117C003ECAB70707003ECC7C003ECE33
:10F0F00083C795002E84AA8493F7F707A384F500AD
:10F10000A16593855502480897B0FFFFE780A01BD3
:10F1100097000000E78040F2AA85480897D0FFFFDB
:10F12000E780C002500801478146A285268597B036
:10F13000FFFFE780A03E05611733FFFF670063FC18
:10F140009777FF1F938707C39C43094599C303C55E
:10F15000970082809777FF1F9387C7C19C4309451B
:10F1600099C303C5D70082809777FF1F938787C015
:10F170009C43014599C303C5A70082801733FFFF55
:10F18000E70243F40111B70708003EC683C79500A4
:10F19000404D0AC493F7F7070AC8A384F5002A89EB
:10F1A000AE8429C41442854703C7060063E0E70A1A
:10F1B00083479400094681496380C702B307F7403B
:10F1C000A304E400B339F00083C716002305F4005C
:10F1D00097900000E780A01E03572403058B19C7F2
:10F1E0006386090097D00000E78000E92164930559
:10F1F0008402280097B0FFFFE780E00C9700000032
:10F20000E78040F4AA85280097D0FFFFE78000F44C
:10F2100097000000E78080F5AA85280097D0FFFFBF
:10F22000E780C0F2014781463000A6854A8597B045
:10F23000FFFFE780A02E13047402480822CC230AA3
:10F24000010002CE97E0FFFFE780E0D605611733AB
:10F25000FFFF670063EA1733FFFFE70243E801118E
:10F260007C003ECAB70708003ECC7C003ECE83C778
:10F2700095002E84AA8493F7F707A384F500A1656F
:10F2800093858502480897B0FFFFE780C003970089
:10F290000000E78020EBAA85480897D0FFFFE780B1
:10F2A000E0EA97000000E78060ECAA85480897D064
:10F2B000FFFFE780A0E9500801478146A285268527
:10F2C00097B0FFFFE780802505611733FFFF6700D8
:10F2D00043E39777FF1F9387E7A99C43014599C3B1
:10F2E00003C5B70082801733FFFFE70243DF011138
:10F2F000B70707003EC683C79500404D0AC493F781
:10F30000F7070AC8A384F5002A89AE8405C81C4201
:10F31000054783C707006368F7060347B400630F18
:10F32000F700A305F40097900000E78040098347A9
:10F33000B400B9CF97D0FFFFE78040BE21649305AA
:10F34000B400280097B0FFFFE780E0F797000000C7
:10F35000E78060F8AA85280097D0FFFFE78000DFEC
:10F36000014781463000A6854A8597B0FFFFE780B8
:10F37000E01A2904480822CC230A010002CE97E0B3
:10F38000FFFFE78040C305611733FFFF670063D7C6
:10F3900097D0FFFFE78020BF55B71733FFFFE70285
:10F3A00003D401117C003ECAB70707003ECC7C00A5
:10F3B0003ECE83C795002E84AA8493F7F707A384D3
:10F3C000F500A165AD05480897B0FFFFE780A0EF05
:10F3D00097000000E78020F0AA85480897D0FFFF3B
:10F3E000E780C0D6500801478146A285268597B0A0
:10F3F000FFFFE780A01205611733FFFF670063D0AE
:10F400009777FF1F938707979C43094599C303C5C7
:10F41000C70082801733FFFFE70263CC01117C0035
:10F42000AE843ECAA165B70707002A843ECCD10549
:10F430007C0048083ECE97B0FFFFE780C0E8970009
:10F440000000E78020FCAA85480897D0FFFFE780EE
:10F45000E0CF500801478146A685228597B0FFFF7F
:10F46000E780C00B05611733FFFF670083C91733BF
:10F47000FFFFE702C3C683C7950093F7F707A3848E
:10F48000F50097000000E78020F91733FFFF6700C1
:10F4900043C71733FFFFE702E3C283C79500032981
:10F4A000C501411193F7F707A384F5001C4283C9F6
:10F4B0000700854763E637079777FF1F9387C7E203
:10F4C0009C432E84AA8485CF97000000E78080F3B8
:10F4D00089476306F502630409028347C900638014
:10F4E00037032306390197900000E78040ED8357EA
:10F4F0002903898B89C797D00000E780E0B726856C
:10F50000A28597000000E78020F1A167CD074800A1
:10F510003EC42302010002C697E0FFFFE780A0A9D6
:10F5200041011733FFFF670023BD9777FF1F9387C4
:10F5300067849C431D4599C303C5E7008280173348
:10F54000FFFFE702C3B90111B70707003EC683C733
:10F550009500584D0AC493F7F7070AC8A384F5002D
:10F560002A89AE8415C71C4283C70700939687017A
:10F57000E18663C4060685466381D7068346E700B5
:10F580006388F6002307F70097900000E78020E3E8
:10F5900021649305E400280097B0FFFFE780A0D224
:10F5A00097000000E780A0F8AA85280097D0FFFF09
:10F5B000E780C0B9014781463000A6854A8597B0EB
:10F5C000FFFFE780A0F53504480822CC230A01009C
:10F5D00002CE97E0FFFFE780009E05611733FFFF33
:10F5E000670023B21733FFFFE70263AF01117C000E
:10F5F0003ECAB70707003ECC7C003ECE83C79500CD
:10F600002E84AA8493F7F707A384F500A165B905B2
:10F61000480897B0FFFFE78000CB97000000E78025
:10F6200000F1AA85480897D0FFFFE78020B2500874
:10F6300001478146A285268597B0FFFFE78000EE4F
:10F6400005611733FFFF6700C3AB1733FFFFE70206
:10F6500063A7AA8401441769FF1F1309E971E149EF
:10F6600097C0FFFFE780A0C56344A400014519A827
:10F6700033053403832709003E958357250063979C
:10F68000970011051733FFFF670003A70504C9BFE3
:10F69000032E8500630A0E121773FF1F1303838C5A
:10F6A0000323030063150300294363900612032319
:10F6B0004E01631503001D43639907101733FFFFC5
:10F6C000E702639FC689428A3E89BA8AB684328B32
:10F6D000AE8B2A84B5E103554E0019E501431A8526
:10F6E0001733FFFF6700A3A0A167A98F116763FB12
:10F6F000E70097000000E78080F5814597F0FFFF65
:10F70000E780C0120844B70700E05841F98F184558
:10F710005CC1B707001FF98F1CC55C4991C7610523
:10F7200097E00000E780408BE38A09FA22859790F2
:10F730000000E78060C65DB7328597C00000E780B3
:10F7400040430D4349DD1C44116703D54700A167C1
:10F75000A98F63FBE70097000000E78040EF814539
:10F7600097F0FFFFE780800C0323840093164B0182
:10F77000D1828347B300035663008588FD8BA305C0
:10F78000F300FD777D8E558EFD76FD16B204F18E69
:10F7900083274301C58E231273012313D30023044F
:10F7A000530123052301A3044301BDDF228597B044
:10F7B000FFFFE78080C9AA850844B5D1610597D0CD
:10F7C0000000E780207F8DB71D431A8582801733A4
:10F7D000FFFFE702238F0569AA84AE89328A0144BC
:10F7E000FD5A7D1997C0FFFFE78020A26347A40060
:10F7F00001451733FFFF67002390D8449317140087
:10F80000BA9703D70700631F370323905701630795
:10F810000A00268597900000E780A0809C449DC345
:10F8200083D76700B3F72701639E3701D288014869
:10F8300081470147814601468145268597000000A2
:10F84000E78040E5050479BF1733FFFFE7028387B0
:10F8500079711C103EC4B7070F003EC61C103EC88D
:10F8600083C79500AA8A328593F7F707A384F5002A
:10F870002E89328497D0FFFFE780009D9317050102
:10F88000C187635AF006AA89228597D0FFFFE780D7
:10F89000A09B2A8A4E85032B040097B0FFFFE780C8
:10F8A000609739ED8357440081440544F11793B7BD
:10F8B0001700A303F10083457100DA872287D286FF
:10F8C0004E86280097E0FFFFE780E057014781461A
:10F8D0003000CA85568597B0FFFFE78020C4A16736
:10F8E0009387F70348083ECC230A810026CE97D0A1
:10F8F000FFFFE780406C45611723FFFF6700C37F70
:10F90000A2851306710097E0FFFFE7806066AA8476
:10F91000094455D1528597E0FFFFE78060D40D443C
:10F9200059D90546D285268597000000E78060EA10
:10F930002A8451B71723FFFFE702637A8355070034
:10F940000346270041112A842E8532C62EC497E033
:10F95000FFFFE780E0D001C93246A245228597002B
:10F960000000E78000E741011723FFFF670063798C
:10F970001723FFFFE702237483C795004111AA8A6A
:10F9800093F7F707A384F5003285AE89328497D0C8
:10F99000FFFFE780608B93170501C1876357F00A6B
:10F9A000C1452A8A228597C0FFFFE78080702A8D93
:10F9B000228597D0FFFFE78020892A89228597D06A
:10F9C000FFFFE7804086930705F893F7F70F1307CB
:10F9D000E007AA8B637BF706228597D0FFFFE780BD
:10F9E00080842A8C228597D0FFFFE780C083AA8C71
:10F9F0005285032B040097B0FFFFE780A08139E90F
:10FA000083574400231101008144F11793B7170075
:10FA1000A300F1000544034711008356210093879A
:10FA200084005685DA8822885286CE8597F0FFFFBB
:10FA3000E78020A7A167E90748003EC423028100B0
:10FA400026C697D0FFFFE780005741011723FFFF2D
:10FA50006700E36913061100A28597E0FFFFE780C6
:10FA60002051AA8409E52311010009446DB79305CB
:10FA700021006A8597F0FFFFE780A0F02A8441FD0E
:10FA8000835521009356C90013164901854866889D
:10FA9000E2875E87858A5182268597000000E7808D
:10FAA00060BF2A848DBF1723FFFFE702C36083C7AF
:10FAB000950041112A8B93F7F707A384F50032854F
:10FAC000AE89328497C0FFFFE78000789317050165
:10FAD000C1876352F00A2A8A228597C0FFFFE78018
:10FAE000A076AA8A228597C0FFFFE780E0752A8961
:10FAF000228597C0FFFFE7800073930705F893F70F
:10FB0000F70F1307E0072A8C6377F706228597C063
:10FB1000FFFFE7804071AA8C228597C0FFFFE78036
:10FB200080702A8D5285832B040097A0FFFFE78009
:10FB3000606E39E58357440085440144F11793B75B
:10FB40001700A301F10003473100930784005A8591
:10FB5000DE882688D6865286CE8597F0FFFFE7801E
:10FB600040948D4748003EC42302910022C697D09E
:10FB7000FFFFE780404441011723FFFF6700235741
:10FB8000A2851306310097E0FFFFE780603E2A84DC
:10FB9000894455D99356C9001316490185486A8886
:10FBA000E6876287858A5182D68597000000E780C4
:10FBB00060AEAA8449BF1723FFFFE702A3502A893A
:10FBC00081440144617A916A176BFF1F130B8B39D3
:10FBD00097B0FFFFE780606463C7A4002285172306
:10FBE000FFFF670063518327090093991400CE97A4
:10FBF00003D5070033074501420741836364570378
:10FC000005C103270B0019C785453E8597400000B5
:10FC1000E78060E9832709000504CE972390070059
:10FC200085047DB797000000E78060A28327090064
:10FC30000504CE972390070065D5814597F0FFFF17
:10FC4000E780C0BEF1BF1723FFFFE702A34783C7CA
:10FC5000950041112A8A93F7F707A384F5003285AE
:10FC60002E89328497C0FFFFE780005E931705015D
:10FC7000C187635AF004AA89832A040097A0FFFF72
:10FC8000E780405931E58357440085440144F1172A
:10FC900093B71700A301F10003483100D6875285BE
:10FCA0000147CE862686CA8597D0FFFFE780806A07
:10FCB000A167F50748003EC42302910022C697D0F1
:10FCC000FFFFE780402F41011723FFFF6700C3427A
:10FCD000A2851306310097E0FFFFE78060292A84A0
:10FCE00089445DD99767FF1F9387C7279C4381CFBE
:10FCF000044997B0FFFFE7804052AA8526859740C8
:10FD00000000E78040DA1305040197000000E78057
:10FD1000C0EA228597800000E78000338144ADBFB0
:10FD20001723FFFFE702233983C795004111AA8AF1
:10FD300093F7F707A384F5003285AE893284231147
:10FD4000010097C0FFFFE780205093170501C1878E
:10FD50006354F0062A8AC145228597C0FFFFE780D9
:10FD60004035AA8B5285032B040097A0FFFFE78044
:10FD7000604A21E98357440085440144F11793B751
:10FD80001700A300F1000348110003572100DA8790
:10FD90005685D2862686CE8597D0FFFFE780805B8A
:10FDA000A1679387270248003EC42302910022C620
:10FDB00097D0FFFFE780202041011723FFFF670056
:10FDC0000333A2851306110097E0FFFFE780401A76
:10FDD0002A8489444DD99767FF1F9387A7189843B2
:10FDE0003E8901CF044997B0FFFFE7800043AA8511
:10FDF000268597400000E78000CB1305040197009B
:10FE00000000E78080DB97B0FFFFE780004195446A
:10FE10003DD9930521005E8597F0FFFFE78060B62E
:10FE2000AA8435F11C480357210022852390E7005E
:10FE300097800000E780402183270900A9D7035558
:10FE4000210097400000E780A0BD35BF1723FFFFCA
:10FE5000E702632683C795004111AA8A93F7F70743
:10FE6000A384F5003285AE89328497C0FFFFE78016
:10FE7000A03D93170501C1876351F0062A8A2285A8
:10FE800097C0FFFFE780403C2A895285032B04007E
:10FE900097A0FFFFE780003831E583574400854491
:10FEA0000144F11793B71700A301F1000348310093
:10FEB000DA8756854A87D2862686CE8597D0FFFF79
:10FEC000E7804049A167F90748003EC4230291003A
:10FED00022C697D0FFFFE780000E41011723FFFFE6
:10FEE0006700E320A2851306310097E0FFFFE7805B
:10FEF00020082A8489445DD99167CA97C20711678F
:10FF0000C1831307F7EF8544E362F7FA9767FF1F92
:10FF1000938747059843BE8B01CF044997B0FFFFF5
:10FF2000E780A02FAA85268597400000E780A0B72C
:10FF30001305040197000000E78020C897B0FFFF79
:10FF4000E780A02D95443DD11C4822858144239013
:10FF5000270197800000E780200F83A70B00B9D707
:10FF60004A8597400000E780A0AB89B71723FFFFC1
:10FF7000E702E3162A844105B28497000000E78077
:10FF8000C0C311C5228597800000E780E00B814641
:10FF90000146A685228597800000E780C04E1C4C54
:10FFA00089C7DC4799C3228582971723FFFF670023
:10FFB00043159767FF1F9387E7DB9C43014599C370
:10FFC0001385070182809767FF1F9387A7DA88430D
:10FFD00082801723FFFFE70283109317C600DD8D91
:10FFE000C2054111C1812A8432C697C0FFFFE78054
:10FFF000E0173246228511829375F60F97C0FFFFF6
:020000040001F9
:10000000E780C01441011723FFFF6700830F172308
:10001000FFFFE702230B79713C083ED2B7070C00C3
:100020003ED43C083ED683C79500AE842A8993F718
:10003000F707A384F500A16593853504481097A0C0
:10004000FFFFE7804028C165FD150144176AFF1FC7
:10005000130ACAF2930A400EAE892E8B2EC697B0B1
:10006000FFFFE780801E4205931704014181C18391
:10007000B24563E9A702C167FD176387F500481021
:1000800097C0FFFFE780800E501001478146A6858C
:100090004A8597A0FFFFE780604845611723FFFF6F
:1000A000670083053307540383270A0BBA9703D6E7
:1000B000C701630A3601638A3501481097000000C2
:1000C000E78060F1DA85050451BFB285EDBF1723E3
:1000D000FFFFE70243FE79717C083EC8B7071100B5
:1000E0003ECA7C083ECC83C79500AA89328593F727
:1000F000F707A384F5002E8997C0FFFFE780C0149F
:1001000085676378F504A165AA848905080897A026
:10011000FFFFE780401B268597400000E78060EDE9
:10012000133415000A04A285080897C0FFFFE78072
:10013000E001A685080897C0FFFFE780200325CCD3
:10014000014781461008CA854E8597A0FFFFE780CA
:10015000E03C45611723FFFF670063F9B3075403D1
:100160000327CA0ABA9703D70700631C970003D670
:10017000270063806505080897000000E780A0E578
:10018000DE8505042EC697B0FFFFE780000D42050F
:10019000931704014181C183B245E3E1A7FCC16724
:1001A000FD17E38FF5F8080897C0FFFFE78000FC14
:1001B00041BFB285F9B7C165FD150144176AFF1F3C
:1001C000130ACADB930A80022E8BAE8B65BF1723FE
:1001D000FFFFE702C3F0184183471700834607007B
:1001E000A207D58FD207D1832390F500834727003C
:1001F000034717008D45A207D98F91832310F6007E
:1002000097C0FFFFE780A0E91723FFFF670063EFB8
:100210001723FFFFE70203EBC16401441769FF1FC7
:100220001309C9D593098002FD1497B0FFFFE78039
:10023000C0026347A40001451723FFFF6700C3EB1B
:10024000330534038327C90A3E9583570500E385A8
:1002500097FE0504D9BF1723FFFFE702A3E62A8A0A
:10026000AE89B284B68A97400000E78080D819E54D
:1002700091473E851723FFFF670003E82A894E85D3
:1002800097C00000E780E08E2A84638E0A048D47C1
:100290006DD103570500C547E31D47FD0347F9012D
:1002A0008546AD47E317D7FC8347450081CF4146DC
:1002B000A6855D0597F00000E780C09E814755D96F
:1002C000AD4745BF130965012302E500CA852685B0
:1002D00097100000E780606231C1A547E38B0AF800
:1002E0002302040079B705C183570500E39247F95B
:1002F0004146A685190597F00000E780A09A81473E
:100300002DD99947BDB74E8597000000E78080F052
:100310002A84954739DD130955004DBF4146A6850E
:1003200023104401231134011305190097F0000034
:10033000E780A099228597800000E780A0EA8147A6
:100340000DBF1723FFFFE70283D979717C003ECCF4
:10035000B7070A003ECE7C003ED083C79500B2842A
:100360002E8493F7F707A384F5001306A1002A89CA
:100370002C00268597000000E780A0E5A1652808ED
:100380008D0597A0FFFFE78000F490408355A10002
:1003900003558100854697000000E78000ECAA84A1
:1003A000AA85280897C0FFFFE78040DA0356A1001E
:1003B00083558100280897000000E780C0C13008FD
:1003C00001478146A2854A8597A0FFFFE780001577
:1003D000854748103ED42302910202D697D0FFFFF2
:1003E000E78060BD45611723FFFF670083D11723B6
:1003F000FFFFE702C3CE79717C003ECCB7070A004D
:100400003ECE7C003ED083C79500B2842E8493F705
:10041000F707A384F5001306A1002A892C0026857E
:1004200097000000E780E0DAA16528088D0597A015
:10043000FFFFE78040E990408355A100035581000C
:10044000814697000000E78040E1AA84AA85280839
:1004500097C0FFFFE78080CF0356A100835581003E
:10046000280897000000E78000B730080147814660
:10047000A2854A8597A0FFFFE780400A4810230223
:10048000910202D402D697D0FFFFE780C0B2456147
:100490001723FFFF6700E3C61723FFFFE70223C40C
:1004A00097000000E78060DB1723FFFF670063C54C
:1004B0009767FF1F9387478C884382801723FFFF2E
:1004C000E702E3C1835725004111AE842A84230744
:1004D000B10017F5FFFF130525466C002316F10048
:1004E00097A0FFFFE780804591C422859780000098
:1004F000E780E0D6FD572310F40013062002814563
:10050000130554009720FFFFE78060C041011723C7
:10051000FFFF670003BF1723FFFFE702A3BA79714C
:100520007C003ECCB7070A003ECE7C003ED083C79D
:100530009500AA89AE8493F7F7073285A384F50066
:100540001306A1002C0097000000E78080C8035527
:100550008100114497400000E780A0A915C503550C
:10056000A100014497B00000E780A06011CD0357BF
:1005700005008357810045446318F70085459700BF
:100580000000E780E0F30144216993053900280861
:1005900097A0FFFFE78020D3A285280897C0FFFF20
:1005A000E780C0BA0356A100835581002808970050
:1005B0000000E78040A2300801478146A6854E85AD
:1005C00097A0FFFFE78080F548104AD423028102FC
:1005D00002D697D0FFFFE780009E45611723FFFFFB
:1005E000670083B11723FFFFE702C3AD9757FF1FD3
:1005F000938747782A8488432E8915C50357450376
:100600008357C4016311F70223260502231805024C
:10061000410597D00000E780209C63060900978081
:100620000000E78060DB81449769FF1F938909958B
:10063000130A800297B0FFFFE78020C263C4A404BE
:100640009757FF1F9387C77B9C4399C70355C401E6
:1006500097200000E780C0BD6307090022859780CE
:100660000000E780C0A01306400E81452285972038
:10067000FFFFE780C0A9FD57231EF4001723FFFFEB
:10068000670083A73385440383A7C90A3E950357B0
:1006900005008357C4016317F700CA85970000005F
:1006A000E78000E2850479B71723FFFFE70283A103
:1006B00083C795004111AA8993F7F707A384F50032
:1006C0003285AE8497C0FFFFE78000B88567637806
:1006D000F5042A8997400000E780A091014401CDEC
:1006E00083D70400314463882701854597000000C3
:1006F000E78080EF01444E85A2864A86A68597D082
:10070000FFFFE780A09CA1679387170448003EC4C1
:100710002302810002C697D0FFFFE780C089410114
:100720001723FFFF6700439D1723FFFFE70283990D
:100730009757FF1F93870764804329C4014597C0DB
:100740000000E780002181470148C1641CDC232EA2
:100750000403232004041769FF1F1309298201449D
:100760009309400EFD1497B0FFFFE78000AE634F82
:10077000A400814517F5FFFF1305857F97A0FFFFB4
:10078000E780C01B1723FFFF67000397330534037F
:100790008327090B3E958357C501638797008545DD
:1007A00097000000E78040E4050475BF93570501FA
:1007B00013D78700A380F50093170501C183A18398
:1007C0002380E5002381F500A381A5008280172303
:1007D000FFFFE702C3902300050083C71500A300B5
:1007E000F50083C725002301F50083C73500A30169
:1007F000F50083C745002302F50083C75500A30217
:10080000F50083C7650093059500A3030500230346
:10081000F50023040500328597000000E78040F9C9
:100820001723FFFF6700E38D1723FFFFE70283898C
:100830004111E9540DCD85CD93F9C5FF2E842A8948
:10084000AA84338AA900B7EA040063189A020D88C3
:10085000854411CCB7E704009C5F82972AC62286A4
:100860006C003305390197E00000E78000462685DB
:1008700041011723FFFF6700238883A78A039104A0
:10088000829793170501C183A183A38EF4FE93572A
:100890000501238FF4FEA183238EA4FEA38FF4FE13
:1008A0006DB763E6D5021723FFFFE7024383B287E4
:1008B00041113686BE8536C697E00000E780E040ED
:1008C000B246410136851723FFFF670083838146C7
:1008D00036858280838705001387F5003D05FD87F7
:1008E00093F77708834607007D158606B58FA3002A
:1008F000F5006307B7007D17834717009D83DDB7B9
:1009000082801713FFFFE702837DB7E7040083A708
:10091000070932872A863A858297133515001713FF
:10092000FFFF6700037E15C181478DC11713FFFFCD
:10093000E702E37A414697E00000E7800039854707
:100940003E851713FFFF6700C37B81473E8582808A
:100950001DCD1713FFFFE7028378414681452A84A6
:100960009710FFFFE780A07A4146814513050403F5
:100970009710FFFFE780A0790147C1672322040495
:1009800038C87CC805451713FFFF6700837701450A
:10099000828081473DCDB5CD1713FFFFE702237459
:1009A000B2842E891306800581452A849710FFFFA3
:1009B000E780E075CA8524C4268597000000E7809B
:1009C000C0F64146814522859710FFFFE7802074DD
:1009D0003044A285228597000000E780C0F293048E
:1009E0000401A285268597000000E780E0EEA68539
:1009F0001305040297000000E78000EE22859700AF
:100A00000000E78020F585473E851713FFFF67004C
:100A1000436F3E8582801713FFFFE702A36A4111EF
:100A2000E9540DCD85CD93F9C5FF2E842A89AA847A
:100A3000338AA900B7EA0400639844030D8881440F
:100A400011CCB7E704009C5F82972AC622866C000F
:100A50003305390197E00000E78020272685410112
:100A60001713FFFF6700436983A78A0391048297E6
:100A700093170501C183A183A38EF4FE935705014B
:100A8000238FF4FEA183238EA4FEA38FF4FE6DB703
:100A900065CD1713FFFFE702E362B28411E6054557
:100AA0001713FFFF670043652A842E890145EDD99E
:100AB0003C487848B3E6E700E5D69386F7FFB3B73E
:100AC000F6007D17032A4404BA9734C87CC863052E
:100AD0000A06C14913050A03B38949412295637D7A
:100AE0003601B2862E86A68597000000E780A0DB3F
:100AF0007C40BE9464C065B7CE862E86CE859700B6
:100B00000000E78040DAC114D2944E9923220404F5
:100B1000A2879306040103C7070003C607038507DE
:100B2000318FA38FE7FEE398F6FE3044A28522853D
:100B300097000000E78020DD2699C14933069940DF
:100B400063EC9900A9DCA686A6851305040397002B
:100B50000000E78040D579BF8147B306F400330732
:100B6000F6000347070083C5060085072D8F238005
:100B7000E600E39437FF3044A28522859700000009
:100B8000E78060D8C1145DBF014582800DC1171395
:100B9000FFFFE702C3541306800581459710FFFF4E
:100BA000E780E05605451713FFFF670083550145B1
:100BB0008280814749C5C1C51713FFFFE702235251
:100BC000FC4141462E84AA846399C704138605011B
:100BD000A2878146C14503C7070003C507038507F0
:100BE000298F3305D600034505008506298FA38F7D
:100BF000E7FEE392B6FE3044A2852685970000000A
:100C0000E78060D0228597000000E78060F8854784
:100C10003E851713FFFF6700C34E138507031D8E24
:100C2000814522959710FFFFE780604E7C401307B7
:100C300000F813060402A2972388E70251BF3E85FD
:100C400082801713FFFFE70283496D712E84B284FF
:100C5000AA8590102800368997000000E780A0D36D
:100C600009EDD55725A050400C4028009700000002
:100C7000E78040E27DD5FD142104F5F42C004A857F
:100C800097000000E78020F3814761DD3E855161D8
:100C90001713FFFF6700E3461713FFFFE702234424
:100CA00041112EC432C62C00054697000000E78093
:100CB00080F941011713FFFF6700A3441713FFFFDB
:100CC000E702E34101112A842EC602C802CA02CCFF
:100CD00002CE97E00000E780C023B2462A86A285B4
:100CE000080897000000E78060FB1375F50F0561A9
:100CF0001713FFFF6700E3401713FFFFE702233ED0
:100D00007971B2872A8421462308B10013051101A5
:100D1000BE853AC436C697E00000E78000FBB246C5
:100D200093059101368597000000E78060A8228531
:100D3000141035460C0897000000E78020F62A843E
:100D4000224701E921460C103A8597E00000E78030
:100D5000C0F7228545611713FFFF6700833A171319
:100D6000FFFFE702C3377171AE84AA850A8532841A
:100D700097000000E78060BB11C90A86A68522851E
:100D800097000000E78020B8814711E1C5473E8504
:100D90004D611713FFFF6700C3361713FFFFE7020C
:100DA00003311D712A8AB289BE84354685471305F1
:100DB00011012E8CB68A3A8BC28C468D2308F10025
:100DC00097E00000E78060F010100C085285231FA8
:100DD000010097000000E780C0F82A843DEDA1479C
:100DE0006313FD089307900591E0E5473546E285DA
:100DF0001305110113990A012308F1001359090180
:100E000097E00000E78060EC1357890093978A0011
:100E1000D98F90080C085285231FF100970000001D
:100E2000E78020F42A8415E9A1E49387FA009183EE
:100E30001379F9003EC6631309004149668B81446A
:100E4000C14B854DB247639F970C6A868C003385F2
:100E50005C0197E00000E78040E7228525611713D9
:100E6000FFFF6700832893079004C9F0A547BDBF23
:100E7000834701050947C14B2308F100834711054A
:100E8000A58FA308F10093872400814463E1FB044C
:100E9000014714083386E6008C08B386E400BA954F
:100EA000DA9683C6060083C505000507AD8E2300CC
:100EB000D600E390E7FE4147639CE70490080C08E6
:100EC000528597000000E780C0E925D181A0B306D4
:100ED0009B00BA871008B305F60090083E9603C53C
:100EE00006000346060085078506298E2380C50077
:100EF000E39277FF998F90080C085285BE94970073
:100F00000000E78000E68947014749D12A84B1B74C
:100F100090083E96034606001408BE962380C6003D
:100F2000850759BFB247850463879714814718081E
:100F3000B306F70098083E973386F9000347070089
:100F4000034606008507318F2380E600E39177FF93
:100F500090080C08528597000000E78080E05DF55E
:100F60003546E285130511012308B10197E0000021
:100F7000E780A0D5139704014183939784002183D0
:100F8000D98F10180C085285231FF100970000001C
:100F9000E78020DD25FD814710183387F9003E9654
:100FA0000347070003460600B306FB008507318FA1
:100FB0002380E600E39277FF65A81808B306F700E0
:100FC00098083E973386F90003470700034606005A
:100FD0008507318F2380E600E3E127FFCA87639E00
:100FE000770990080C08528597000000E78060D7C9
:100FF00011FD81479800B306F700900818103E973E
:101000003E9603470700034606008507318F23807D
:10101000E600E39177FF3546E285130511012308C9
:10102000B10197E00000E78040CA139704014183B3
:10103000939784002183D98F10180C085285231FA1
:10104000F10097000000E780C0D1E31105EC814773
:1010500010183387F9003E96034707000346060041
:10106000B306FB008507318F2380E600E3E227FF0C
:10107000C109410BC1BB814785B79408BE9683C6A1
:10108000060018083E972300D700850789BF6380B4
:1010900006321713FFFFE702830159712A84BE89C4
:1010A000B28B85473546130511022E8B468C42893B
:1010B000BA8A368A2300F10297E00000E780E0C098
:1010C00010180C1022852317010297000000E780FA
:1010D00040C963180512A147631FFC0693079005DA
:1010E00063930900E5473546DA8513051102931429
:1010F0000A012300F102C18097E00000E780E0BC14
:1011000093178A0013D78400D98F90080C1022857A
:101110002317F10297000000E780A0C47DE16392ED
:1011200009049307FA00BD88918391E0C144C20786
:10113000C183DE8C814A3EC6414DB24763E2FA0E5E
:101140006286B3854B01881097E00000E78080B588
:101150004DC93D557DA093079004E39609F8A54736
:1011600059B7834701050947C14C2300F102834762
:101170001105B3C7F900A300F10293872900814943
:1011800063E1FC04814618103306D7008C083387CE
:10119000D900B69556970347070083C50500850615
:1011A0002D8F2300E600E390D7FE41476390E706CA
:1011B00090080C10228597000000E78080BA35D196
:1011C00089A0B3863A01BA871010B305F6009008DB
:1011D0003E9603C506000346060085078506298E50
:1011E0002380C500E39297FF3387EC4090080C10F2
:1011F0002285BA9997000000E780A0B68947014789
:1012000041D165611713FFFF670023EE90083E96FA
:10121000034606001410BE962380C600850779B7E2
:10122000B247850A93990A01939D8A0093D90901CF
:101230006391570F85473546DA8513051102230060
:10124000F10293D9890097E00000E78000A8B3ED90
:101250003D0190000C1022852317B1039700000078
:10126000E78020B059FD8147A68963EA9706268664
:101270000C084A8597E00000E78020A581471810F8
:10128000B306F700100898083E973E9603470700FC
:10129000034606008507318F2380E600E3E197FED1
:1012A000639FA90590080C10228597000000E78035
:1012B00040AB21F981479810B306F7009008181841
:1012C0003E973E9603470700034606008507318F89
:1012D0002380E600E391A7FF4109C10CB9BD1808BE
:1012E0009000B306F7003E963387FC0003470700E3
:1012F000034606008507318F2380E600B5B79808BE
:101300004E97034707001C10CE972380E7008509FE
:1013100041BF85473546DA85130511022300F102E6
:1013200093D9890097E00000E780209AB3ED3D0152
:1013300090000C1022852317B10397000000E7806E
:1013400040A2E31005EC814718089000B306F700AF
:101350003E963387FC0003470700034606008507D7
:10136000318F2380E600E391A7FF41460C084A85B0
:1013700097E00000E780609581471810B306F700FA
:10138000100898083E973E9603470700034606005C
:101390008507318F2380E600E391A7FF90080C10AA
:1013A000228597000000E780C09B1DD599BD7D5523
:1013B00082801713FFFFE70283D201112A842E8552
:1013C00093055100328902C002C202C402C69304CE
:1013D000740097F0FFFFE780A03D1D46A68513052A
:1013E000910097E00000E780408E10088A854A85CA
:1013F00097000000E780E09619ED930714001808A5
:1014000083C607000346070085070507B18EA38F33
:10141000D7FEE397F4FE05611713FFFF670063CE65
:101420001713FFFFE70203CA2E848C414111AA89DA
:10143000838715003289914463D30700A1449757ED
:10144000FF1F938767EA9C43A1C7C1CA8D4723103A
:10145000F10083C725004A852301F10083C73500C9
:10146000A301F10083C745002302F10083C75500A3
:10147000A302F10083C7650093059100A303010057
:101480002303F1002304010097F0FFFFE7804032BF
:101490000C404A860A8597F0FFFFE78080330328D7
:1014A000040083564400A6881D0881470147E516BD
:1014B00042868A854E8597000000E780408E2A8903
:1014C00019E5A685228597B0FFFFE780E0C14A8530
:1014D00041011713FFFF670023C24A860A8597F070
:1014E000FFFFE780002F6DB71713FFFFE70283BDF3
:1014F0002E848C414111AA89838715003289914439
:1015000063D30700A1449757FF1F9387E7DD9C43F0
:10151000A1C7C1C68D472310F10083C725004A85A6
:101520002301F10083C73500A301F10083C7450003
:101530002302F10083C75500A302F10083C76500B1
:1015400093059100A30301002303F100230401008C
:1015500097F0FFFFE780C0250C404A860A8597F088
:10156000FFFFE780002783564400032804008A8594
:10157000858EC2061D08C1822312D400A688814729
:101580000147E51642864E8597000000E78060B06F
:1015900041011713FFFF670023B64A860A8597F0BB
:1015A000FFFFE78000234DBF1713FFFFE70223B3C0
:1015B000B335B000011185052A891315F60133658D
:1015C00015012308B1009305110136843AC632C0D3
:1015D0003EC442C297F0FFFFE780801DA247124839
:1015E000425593D68700230BF10093059101935741
:1015F0008800A30AD100A30BF100230C010197F08E
:10160000FFFFE780E01A3247024603280400B337A1
:10161000E000835644009207914411C2A1444A85D8
:10162000A68842860C0897F0FFFFE78040772A895A
:1016300019E5A685228597B0FFFFE780E0AA4A85D5
:1016400005611713FFFF6700C3AB1713FFFFE70226
:1016500063A701113EC68647B335B0008505AA8948
:101660001315F6015D8D2308B10093051101368431
:101670003A89B28442C446C297F0FFFFE780401324
:1016800022489248164593578800A30AF100930513
:10169000910193D78800230B0101A30BF100230CC8
:1016A000110197F0FFFFE780A010324710408356EA
:1016B0004400B337E000920703280900914891C025
:1016C000A1480C084E8597000000E780809CAA8402
:1016D00001E9835544004A8597B0FFFFE780C0A029
:1016E000268505611713FFFF670003A1AA959307DD
:1016F000F00F170701001307A7676317B50013C59D
:10170000F7FF1375F50F828005058346F5FFB58F4A
:10171000BA9783C70700D5B703574500144193070D
:10172000F00F170601001306A6643697420741839F
:10173000139506014181631BE500AD8FB29703C588
:101740000700130515F3133515008280850603C5C0
:10175000F6FFA98FB29783C70700D9BF1713FFFF02
:10176000E702E397B28736842E86BA86AA853E853D
:10177000BA8497F0FFFFE7806052634F050022852F
:1017800097D00000E780E0782A86A686A285268585
:1017900097F0FFFFE78080501713FFFF6700639605
:1017A0001713FFFFE70203925D712A8BAE8A1705BC
:1017B0000100130565592C00B284368ABA893E8926
:1017C00097F0FFFFE780C04F2A845DE13410414667
:1017D000DA85280097F0FFFFE780404C2A8449E92A
:1017E0008547A303F100A6C2930771002408BEC475
:1017F000A68685470D462C18281002DC02DED6C0CE
:10180000BEC697F0FFFFE78000442A8435E1834796
:101810007102A6860D4693F7F7072300FA00C14729
:101820003EDE2C188947281026DCA303F10097F030
:10183000FFFFE78040412A8405ED4146A6854E859D
:1018400097D00000E78060488D47A6860D462C188B
:101850002810A303F10097F0FFFFE780C03E2A8421
:1018600001E94146A6854A8597D00000E780E0451A
:10187000228561611713FFFF670003881713FFFFBD
:10188000E702E38597F700009387C7A0984383C7D3
:10189000470079712A89AE84170501001305454B6D
:1018A0000C083AC42306F10097F0FFFFE78040419F
:1018B0002A8405ED14104146CA85080897F0FFFFF9
:1018C000E780C03D2A8415E1140815462C00081055
:1018D00097F0FFFFE780803C2A8401E921462C082D
:1018E000268597D00000E780403E2285456117138A
:1018F000FFFF670003811703FFFFE702437E97F7AF
:101900000000938727999C477971AA842E84170534
:101910000100130565440C083EC697F0FFFFE78001
:10192000203A0DE914104146A685080897F0FFFFFC
:10193000E780C03605E1140811466C00081097F0E6
:10194000FFFFE780A03519E58347F10193F7F7031F
:101950002300F40045611703FFFF6700837A170334
:10196000FFFFE702C3773688A14881470147E54674
:1019700097F0FFFFE780A0421703FFFF670063783F
:101980001703FFFFE702A3753688A1488147014787
:10199000E54697F0FFFFE780C06F1703FFFF670082
:1019A00043761703FFFFE702837301112A842E8514
:1019B0000C0832C697F0FFFFE780803009ED324710
:1019C000970601009386C6371008C1452285970007
:1019D0000000E780E0D805611703FFFF670063722E
:1019E0001703FFFFE702A36F4111C1472EC032C4A6
:1019F0008A8509463EC23EC697F0FFFFE780A024D5
:101A000041011703FFFF6700C36F1703FFFFE702E2
:101A1000036D4111AE8613061009AA850A8502C01E
:101A200002C202C402C697F0FFFFE78020274101EF
:101A30001703FFFF6700E36C1703FFFFE702236A4A
:101A40003287970601009386A6312E869305000201
:101A500097000000E780C0D01703FFFF6700636AAC
:101A60001703FFFFE702A3677971C1472ACC2ED085
:101A700032D42C080D4628003ECE3ED23ED602C4BB
:101A800002C602C802CA97F0FFFFE780C01B45618B
:101A90001703FFFF6700E3661703FFFFE7022364F6
:101AA0000111AA842E84170501001305E52B8A85F0
:101AB00097F0FFFFE780C02015E514084146A68592
:101AC0000A8597F0FFFFE780601D09ED8347E1017C
:101AD0000347F101A207D98FCA07C9836177D98F5C
:101AE0002310F40005611703FFFF6700836115CD24
:101AF0001703FFFFE702A35E9747FF1F9387472C5B
:101B000090439745FF1F9385E52B1745FF1F13054E
:101B1000252797D00000E78000C51745FF1F130554
:101B200025261703FFFF6700C35D1745FF1F130539
:101B3000252582808DCD1703FFFFE702435A974783
:101B4000FF1F9387E727944301112E840A86974548
:101B5000FF1F9385252797D00000E78040C60A85A0
:101B60000294014505611703FFFF670083597D5506
:101B700082801703FFFFE702835697D00000E780BB
:101B800080D19747FF1F23ADA72217F5FFFF13054D
:101B9000E5C997B00000E780C0741703FFFF670036
:101BA00043561747FF1F1307E723931715000843F2
:101BB0003E95FD572310F50082801703FFFFE702D3
:101BC00003522A84084009E51703FFFF67006353A7
:101BD0001C4158401CC06313E5005CC0834755009E
:101BE00023200500F99BA302F50097A0FFFFE780E3
:101BF000207CC9BF1703FFFFE702C34C9747FF1FB5
:101C00009387472098432A8411CB8347350093F765
:101C1000070289C70355050089450297130544014A
:101C200097B00000E780403B835504000355E40073
:101C300097300000E780A00C485819C597A0FFFF17
:101C4000E7800077232A040213058403970000002D
:101C5000E780E0F68144B1499790FFFFE780206A72
:101C600063CBA402834734002320040493F727FCAA
:101C7000A301F40000489790FFFFE7804069131626
:101C80001500814522859700FFFFE7804048170334
:101C9000FFFF67006346B387340303290403850409
:101CA0003E994A8597000000E78060F1230409000F
:101CB00065B78347350093F7070299E301458280B2
:101CC0008357E500E39CB7FEC167FD176316F60076
:101CD00005458280054599A81703FFFFE7022340C9
:101CE00093170601C187B2842A8401496359F0021F
:101CF000835705009DCB01456367F60003458400CB
:101D00003E953325A6001375F50F0DA01C4813173B
:101D10001900BA9783D70700E38E97FA05099790C1
:101D2000FFFFE780C05EE343A9FE01451703FFFF05
:101D30006700233D1703FFFFE702C338AE89AA847B
:101D40009790FFFFE78060522A8497D0FFFFE780DB
:101D5000A02EAA86014713068401970500009385EB
:101D600085E41745FF1F130525089790FFFFE780BF
:101D7000E0182A8925C98C441304C50022859E05D4
:101D800093F5050897A0FFFFE780403CCC40838790
:101D90007400E18163DD070493E50508228597A0BF
:101DA000FFFFE780A03A0D4693854400228597A067
:101DB000FFFFE780C03683D50400228597A0FFFF90
:101DC000E780E03D83D52400228597A0FFFFE780D0
:101DD000003D03D6490083A50900228597A0FFFF97
:101DE000E780E0334A851703FFFF6700E33093F590
:101DF000F5076DB71703FFFFE702632E01112A8471
:101E0000328532C697A0FFFFE780E0279780FFFF6B
:101E1000E780C030835704001747FF1F13070716DA
:101E20003246231BF100930700F8A30DF1001C4775
:101E30001843231AA1008983858BB307F740B28525
:101E400048083ECE231C0100230D0100970000002E
:101E5000E78080EE05611703FFFF6700832A170301
:101E6000FFFFE7022326004101453DC49304C4005F
:101E700026853289AE8997A0FFFFE780C02495456B
:101E80002A8A2685035B040197A0FFFFE7802021B3
:101E9000268597A0FFFFE780603E8D45AA8A2685AC
:101EA00097A0FFFFE780A01F268597A0FFFFE78090
:101EB000E03C5C48420A135A0A01D2975CC42318DA
:101EC0006401814763983A0146054D8133062541F7
:101ED0009337160013F5F70F1703FFFF6700C321B1
:101EE0001703FFFFE702231D89692A8BAE8B328A15
:101EF000B68A81440144314CFD199790FFFFE78079
:101F0000004063CDA4009790FFFFE7804042018D21
:101F100033B5AA001703FFFF6700631D33898403ED
:101F200083270B003E9963170A00834789008504C5
:101F30003E94E1B703560A00DE854A8533F6C900B0
:101F400097000000E780E0F16DD10545E1B7170388
:101F5000FFFFE702C31801112A847C000355E50046
:101F60003ECAB70707003ECC7C003ECE972000005B
:101F7000E78020082A898545480897A0FFFFE78069
:101F800020399945480897A0FFFFE780E015AA840B
:101F90004A8597200000E780A0082380A400974787
:101FA000FF1F9387A7FD9C434166130606F0939697
:101FB000870113D78701558F93D68700F18E558FF0
:101FC000A207B706FF00F58FD98F11462C001385A5
:101FD00014003EC497D00000E78020CF5008A382B1
:101FE00004008945228597000000E780E0E019C9D8
:101FF000AA851305840397A0FFFFE780E0313C40EA
:1020000085073CC005611703FFFF6700830F1703B7
:10201000FFFFE702C30C9790FFFFE78040312A845F
:1020200005049790FFFFE780802F3305A402F14756
:1020300091453305F50297200000E78020BA11E5AD
:1020400065551703FFFF6700C30B9747FF1F23A3C7
:10205000A7DA9790FFFFE780802D2A8405049790E8
:10206000FFFFE780C02B3305A402894506059720B2
:102070000000E780A0B669D59747FF1F23A4A7D625
:102080009790FFFFE780A02A2A8405049790FFFF1E
:10209000E780E0283304A4029747FF1F239687D4E4
:1020A0009790FFFFE780A0282A849790FFFFE780A2
:1020B0000027930714003385A7029747FF1F239635
:1020C000A7D2970701009387E78D1747FF1F2321AA
:1020D000F7D20145BDB71703FFFFE702A3FEAA84AD
:1020E0002E8901449749FF1F938949E9130A800605
:1020F0009790FFFFE780A0226347A40001451703E4
:10210000FFFF670063FF3305440383A709024A8684
:10211000A6853E9597000000E780E0B919E1050427
:10212000C1BF0545E9BF1703FFFFE702C3F8AA8A4D
:102130002E8BB28B368C3A8A814401448149974C6C
:10214000FF1F938CACE3130D80069790FFFFE78091
:10215000001D63C9A40011E085494E851703FFFFE8
:102160006700E3F83389A40383A70C025E86D68553
:102170003E994A8597000000E780E0B31DC1979023
:10218000FFFFE780C01A0544636D4501D286628671
:10219000DA851305090397000000E780A0D411C178
:1021A000854985045DB71703FFFFE702A3F1C1640A
:1021B00041112A8901449749FF1F938929DC130A99
:1021C0008006FD1436C632C42EC29790FFFFE7800A
:1021D000001592452246B2466348A40001454101DC
:1021E0001703FFFF670043F13305440383A7090288
:1021F0003E9509C683473500C18B9DC791C683476D
:10220000350093F707028DC3630699008357E500F5
:10221000639C27010357050001CB63E7E500834773
:102220008500BA97E3CDF5FA050469BF1703FFFFF0
:10223000E70243E9C1642A8901449749FF1F938952
:10224000E9D3130A8006FD149790FFFFE780200D65
:102250006346A4001703FFFF670003EA3305440346
:1022600083A709023E958357E500638A97006304BC
:1022700099006396270197000000E780E097050426
:10228000E1B71703FFFFE70283E289692A8AAE8A72
:10229000328BB68B8144174CFF1F130C2CCE930C42
:1022A0008006314DFD199790FFFFE780400763C618
:1022B000A4001703FFFF670043E3338994038327D8
:1022C0000C028355CA015A863E994A859700000040
:1022D000E780609E31C1814D15A03384AD03832713
:1022E000090303D60B00D68533F6C9003E94228538
:1022F00097000000E780E0B609E9850D9790FFFFA1
:10230000E780E0FFE3CBADFC01A822859700000049
:10231000E780E08A23040400850471B71703FFFFF8
:10232000E70263D94169AA8A014A174BFF1F130BC1
:10233000EBC47D19C14B054C9790FFFFE78020FE51
:102340006346AA001703FFFF670063DA930980065C
:10235000B3073A0383290B02BE9983D7E900638E42
:10236000270163842A01639A570103A4890301E8C2
:102370004E8597000000E780C0BD050A75BF8357F2
:102380000401639977099304C400268597A0FFFF91
:10239000E78060D385452A8D2685835C040197A05C
:1023A000FFFFE780C0CF268597A0FFFFE780A0E76B
:1023B00062056185635905048D45268597A0FFFF59
:1023C000E780E0CD8945268597A0FFFFE78020CDF7
:1023D0008945268597A0FFFFE78060CC8545268547
:1023E00097A0FFFFE780E0CC83470500094793F7FC
:1023F000F707639AE7009945268597A0FFFFE780D6
:1024000040CBA30285014848337D2D012318940158
:102410006A9548C40040A1BF1703FFFFE70223CC21
:1024200037E404008327041D82979747FF1F83C763
:10243000E7A11715FF1F13056511A300F5008327FA
:10244000441C82978327841C81461306F00F814524
:10245000014582971703FFFF6700A3CA1747FF1FB5
:102460001307C78E18439745FF1F83C5259E9747BF
:10247000FF1F9387279C8346870303469703639731
:10248000D5009747FF1F2383C79C828083C58701A0
:102490000347A7036317B6009747FF1F2388E79AF0
:1024A000828003C687016317C7009747FF1F238FEA
:1024B000D798828083C68701130750026319D7001B
:1024C000930760021747FF1F2302F798828083C695
:1024D0008701130660026315D60093077002DDB70B
:1024E00083C7870155BF9747FF1F9387A794D44B96
:1024F0000947638DE6081703FFFFE70243BE17494C
:10250000FF1F130969903E8483470900918B9DCF7B
:10251000B7E4040083A7041D829783A7441C1745D2
:10252000FF1F1305E58E829783A7841C81461746FB
:10253000FF1F0346E68F81450145829721C58347EA
:102540000900ED9B1747FF1F2300F78C834704000A
:1025500093F7F70F85CB91471747FF1F2326F78E79
:1025600097000000E78080EB97000000E78040EFD5
:10257000B7E70400BC4F414691451745FF1F03458F
:10258000E58B82971703FFFF6700A3B782801703CD
:10259000FFFFE702C3B48D4741116306F504C54749
:1025A0006308F50285476310F5029747FF1F2381F3
:1025B000A78AB7E70400BC4B930500101745FF1F1F
:1025C0000345C587829741011703FFFF670063B387
:1025D00085471747FF1F230DF786B7E70400BC4B5D
:1025E00093050020E1BF9747FF1F9387A784D44B33
:1025F0001147638DE600B7E7040083A7071D8297A4
:10260000B7E70400BC4B930500044DBF05491747CD
:10261000FF1F232B278383C7070032C62E8493F71F
:10262000F70FD5D3B7E4040083A7041D7D141374FA
:10263000F40F8297E37689FCB245994703C61500EB
:10264000E3F0C7FCFC4409061745FF1F130585800E
:102650008297BC48930500081735FF1F0345057E88
:10266000829779BF1703FFFFE70263A71737FF1FA2
:102670001307477C4047184B1C409736FF1F23A188
:10268000F67C6316E4001737FF1F232DF77A130536
:1026900084FE9790FFFFE78060A6035564FF978054
:1026A000FFFFE780E06E97A0FFFFE78060D0170391
:1026B000FFFF670003A51703FFFFE70243A2973759
:1026C000FF1F93872777D84BDC4789C79700000007
:1026D000E78080F985471737FF1F2327F77697375D
:1026E000FF1F9387A7669C43930500021735FF1FC2
:1026F0000345C57483C787031737FF1F2308F77483
:10270000B7E70400BC4B82971703FFFF6700639F86
:102710009737FF1F23A2A77282801703FFFFE702EC
:10272000639A37E404007C4CA1451735FF1F03452D
:10273000E57082977C48A1451735FF1F034505705A
:102740009734FF1F9384046F8297DC4489EB9700D2
:102750000000E78080D91703FFFF6700E39903D5E6
:1027600067FF9780FFFFE780A062AA896DD1D848F4
:1027700091476310F7027C4C91451735FF1F0345C5
:10278000E56B82977C4891451735FF1F0345056B24
:10279000829703A9490103D409018947B7E90400D5
:1027A0001737FF1F2322F76A83A7091D210442045C
:1027B000829783C784011715FF1F130525D9611957
:1027C0001717FF1FA304F7D883A7491C41808297DE
:1027D0009737FF1F238E076683A7C91C81460946CA
:1027E0009375F40F4A85829711E99737FF1F83C7C6
:1027F000677689C79700FF1FE780C03FB7E70400EF
:10280000BC4F2146A1451735FF1F0345256382971D
:1028100099B71703FFFFE702838C93F70520011197
:102820002E8481CF97000000E78020E91345042023
:1028300005611703FFFF6700C38C93F70510A9CF4D
:102840009734FF1F9384045FDC4897000000E78003
:1028500020C11737FF1F1307674F184383C7840131
:10286000034787036318F700DC4489C7970000001B
:10287000E78080DF85471737FF1F2327F75CB7E71F
:102880000400BC4B930500021735FF1F0345055B91
:1028900082971345041069BF93F70508BDC79737A2
:1028A000FF1F83C7375BE91719469735FF1F9385CD
:1028B000855A1305D10093F4F70F1739FF1F034909
:1028C000695997C00000E780404093970401C18395
:1028D0001737FF1F13078758231DF100231CF10032
:1028E0009737FF1F938707553ACE3ACAD843230636
:1028F000010009CBDC439315890154080D46E1859D
:10290000680082971345040825B793F72500A5C3EF
:102910009737FF1F93870752D84B89476306F70203
:102920009737FF1F83C7474E13F7270011EF918B8F
:1029300099CFB7E70400BC4F1306000A8945173545
:10294000FF1F0345A54F829713452400D5B5973740
:10295000FF1F9387A73F9C4383C787031737FF1F3A
:102960002306F74E97000000E78060DBF1BF93F786
:10297000050281CB97000000E78060DA134504026E
:1029800045BD93F7850081CB97000000E780E0D23A
:102990001345840071BD93F7150081CB97000000AB
:1029A000E780A0B41345140061B593F7450081CBCF
:1029B00097000000E78060B31345440095BD93F78E
:1029C000050495C39737FF1F83C7C74691CB970070
:1029D0000000E780A0A491471737FF1F2326F74682
:1029E00013450404B1B593F705010145E38207E4FB
:1029F0009737FF1F93870744D84B91476310F7041D
:102A00009737FF1F938747409C4313D72700858341
:102A1000D98F858B91E7B7E7040083A7071D8297BD
:102A2000B7E70400FC4F91451735FF1F03450541EB
:102A3000829785471737FF1F2328F7401345040166
:102A4000C5BB9737FF1F2387A750828017F3FEFF70
:102A5000E702E3689737FF1F23A4073E9737FF1F5E
:102A600023A2073E85471734FF1F1304242E173770
:102A7000FF1F232BF73C1C4083C787031737FF1F1B
:102A80002306F73C9790FFFFE780A08F29C5971793
:102A9000FF1F23A1A7AC1C40170500001305A5D7F5
:102AA00083C787031737FF1F2302F73A1717FF1F44
:102AB000A30EF7A89737FF1FA38E0736B7E70400CA
:102AC00083A7070882979737FF1F2389A73617F335
:102AD000FEFF67000363B7C7898E938767ED1717FB
:102AE000FF1F2329F7A645BF1737FF1F034787346A
:102AF000795555E79737FF1F9387C73303C71700EB
:102B000005079736FF1FA387E63203C717008D46D8
:102B10003377D7029736FF1FA38EE63083C61700A0
:102B20001737FF1F13078722184393F6F60FA9EEF6
:102B3000834787031737FF1F230AF7308547173767
:102B4000FF1F2309F72E9737FF1F9387E72B9C431F
:102B50000145998BA9E717F3FEFFE702435837E4D5
:102B600004007C48C1451735FF1F0345252D82977A
:102B70003C4885451735FF1F0345452C8297014585
:102B800017F3FEFF6700E35783C717008546639579
:102B9000F6008347970379BF8347A70361BF82800D
:102BA0009737FF1F83C70729A1CF17F3FEFFE7025F
:102BB000035337E404009737FF1F238D07267C4813
:102BC00085451735FF1F0345652782977C4C914546
:102BD0001735FF1F0345852682977C489145173599
:102BE000FF1F0345A52582973C48C1451735FF1FA8
:102BF0000345C5248297014517F3FEFF6700635024
